:100000000C94F3100C9482C60C94ADC60C94D8C614
:100010000C9403C70C942EC70C9459C70C9484C736
:100020000C94AFC70C9424110C9424110C9424113B
:100030000C9424110C94A6CF0C9424110C9424112C
:100040000C9424110C94C98B0C9424110C9424113D
:100050000C9424110C9424110C9451980C94DAC72C
:100060000C9424110C9426110C9424110C9424113A
:100070000C9424110C9424110C9424110C9424112C
:100080000C9424110C9424110C9424110C9424111C
:100090000C9424110C9424110C9424110C9424110C
:1000A0000C9424110C9424110C9424110C942411FC
:1000B0000C9424110C9424110C9424110C942411EC
:1000C0000C9424110C9424110C9424110C942411DC
:1000D0000C9424110C9424110C94094A0C94474A52
:1000E0000C942411D331F3310B3239325B329B3211
:1000F0002A335D33033467349C34B9347836CB34D7
:10010000D534DF34E934FA34223548356635AC3538
:10011000E835F235FC350636103678362C3678362A
:1001200078367836783635362C973C975B976B97D0
:1001300086978B978E97939796979B979E97A39763
:10014000AD975CC626C62EC63AC647C668C675C6F3
:100150001BC920C925C92FC939C9B2C943C94BC94F
:1001600053C95DC967C971C980C98AC9B2C994C96F
:100170009EC9A8C9D4C9D7C9C6C9CAC9D0C90ECAD7
:10018000DBC9DFC9E5C9E9C9EDC9F3C9F7C9FBC9CD
:100190000ECA01CA05CA09CA084AD73B3BCE016E3E
:1001A00084BCBFFDC12F3D6C74319ABD56833DDACE
:1001B0003D00C77F11BED9E4BB4C3E916BAAAABEDD
:1001C000000000803F05A84CCDB2D44EB93836A906
:1001D000020C50B9918688083CA6AAAA2ABE000043
:1001E00000803F004A313800446F6E6520736176AD
:1001F000696E672066696C652E0A004D32390020F1
:1002000020506C616E6E65724275666665724279E9
:100210007465733A20002046726565204D656D6FE8
:1002200072793A2000436F6D70696C65643A204DB5
:10023000617220313520323031380A00207C204173
:100240007574686F723A20284A6F6C6C792C20782C
:10025000787878787878782E434F2E290A003230D3
:1002600031362D31322D30362031323A30300020C7
:100270004C61737420557064617465643A20003178
:100280002E312E302D5243380A0056312E312E3267
:100290000A0020536F66747761726520526573653A
:1002A000740A00205761746368646F672052657335
:1002B00065740A002042726F776E206F7574205249
:1002C000657365740A002045787465726E616C20F0
:1002D00052657365740A00506F77657255700A0035
:1002E0004A3132004A31370073746172740A005027
:1002F00072696E7465722068616C7465642E206B1F
:10030000696C6C28292063616C6C6564210A004B60
:10031000494C4C45442E20004B494C4C45442E2022
:100320000020746F6F206C6F6E6720657874727533
:1003300073696F6E2070726576656E7465640A000D
:1003400020636F6C6420657874727573696F6E20BA
:1003500070726576656E7465640A006F6B00526535
:1003600073656E643A20004F66667365747320612E
:1003700070706C696564004572723A20546F6F202A
:100380006661722100546F6F206661722066726F21
:100390006D207265666572656E636520706F696E4B
:1003A000740A0043290A0061626C656420286D6943
:1003B0006E2074656D702000436F6C6420657874E6
:1003C000727564657320617265200020643A0020B4
:1003D000693A0020703A00205A0020590058002045
:1003E000204D61783A2000205A0020590058002002
:1003F000204D696E3A20004F6666004F6E20005314
:100400006F667420656E6473746F70733A20005A5F
:1004100020456E6473746F702041646A7573746DE7
:10042000656E742073657420746F20286D6D293A91
:100430000053657474696E672054726176656C2030
:10044000416363656C65726174696F6E3A20005335
:10045000657474696E6720526574726163742041BB
:100460006363656C65726174696F6E3A20005365F1
:100470007474696E67205072696E7420416363659D
:100480006C65726174696F6E3A20005365747469AB
:100490006E67205072696E7420616E6420547261C0
:1004A00076656C20416363656C65726174696F6E1B
:1004B0003A20004D31343520533C696E6465783EF6
:1004C000206F7574206F662072616E67652028301A
:1004D0002D31290A004649524D574152455F4E4140
:1004E0004D453A4D61726C696E20312E312E302DA2
:1004F00052433820284769746875622920534F5544
:100500005243455F434F44455F55524C3A687474BB
:1005100070733A2F2F6769746875622E636F6D2F41
:100520004D61726C696E4669726D776172652F4DAF
:1005300061726C696E2050524F544F434F4C5F565E
:10054000455253494F4E3A312E30204D4143484990
:100550004E455F545950453A3344205072696E7489
:1005600065722045585452554445525F434F554E8D
:10057000543A3120555549443A63656465326132D5
:10058000662D343161322D343734382D39623132B1
:100590002D6335356336326633363766660A003387
:1005A00044205072696E746572204F66662E004258
:1005B000656420646F6E652E004A3039003F0A0082
:1005C00020573A004265642048656174696E672E61
:1005D000004A3038004A3033004A3034004A30375D
:1005E0000048656174696E6720646F6E652E003F18
:1005F0000A0020573A004A30360048656174696E37
:10060000672E2E2E003344205072696E746572205E
:1006100072656164792E006F6B004B494C4C454408
:100620002E20004543484F00494E464F0045525248
:100630004F52530044525952554E00434F4D4D5561
:100640004E49434154494F4E006F666600230628C9
:10065000062D0634063B0644454255473A00486598
:100660006174696E672E2E2E003344205072696EBD
:100670007465722072656164792E002569730025A6
:10068000696D20256973002569682025696D20251D
:10069000697300256964202569682025696D202516
:1006A00069730025697920256964202569682025FA
:1006B000696D20256973005072696E742074696DCC
:1006C000653A2000456E642066696C65206C69732C
:1006D000740A00426567696E2066696C65206C6902
:1006E00073740A004E6F206D6F76652E00334420C0
:1006F0005072696E7465722072656164792E005261
:100700006573756D696E67207072696E74005761EC
:10071000697420666F7220757365722E2E2E00200C
:10072000453A00205A3A0020593A00583A00576199
:10073000726E696E673A20486F6D696E6720427508
:100740006D702044697669736F72203C20310A0015
:100750004A303400536C6565702E2E2E0047322FC0
:1007600047332062616420706172616D65746572E7
:10077000730A004163746976652045787472756404
:1007800065723A20002042403A0020403A00202F73
:100790000020423A00202F0020543A00556E6B6E24
:1007A0006F776E20636F6D6D616E643A202200205A
:1007B000496E76616C6964206578747275646572DF
:1007C000200053442072656164206572726F720A62
:1007D00000446F6E65207072696E74696E67206682
:1007E000696C650A004B494C4C45442E200053541B
:1007F0004F505045442E20005072696E746572202F
:1008000073746F707065642064756520746F206503
:1008100072726F72732E2046697820746865206545
:1008200072726F7220616E6420757365204D393964
:100830003920746F20726573746172742E2028548D
:10084000656D70657261747572652069732072657B
:100850007365742E20536574206974206166746515
:10086000722072657374617274696E67290A004E32
:100870006F204C696E65204E756D626572207769D8
:10088000746820636865636B73756D2C204C6173AD
:1008900074204C696E653A20004E6F204368656392
:1008A0006B73756D2077697468206C696E65206E56
:1008B000756D6265722C204C617374204C696E6595
:1008C0003A2000636865636B73756D206D69736DA5
:1008D000617463682C204C617374204C696E653AB6
:1008E00020004C696E65204E756D626572206973DB
:1008F000206E6F74204C617374204C696E65204EBD
:10090000756D6265722B312C204C617374204C69BB
:100910006E653A20004D31313000656E7175657538
:1009200065696E672022004731205A2B323000471C
:100930003931004A31300056312E312E32004A33DF
:100940003320004A3032004A313200473930004704
:1009500031204525694635303000473120452D305E
:100960002E314625690047312045302E3146256914
:10097000004731205A2569462569004731205A2D04
:10098000302E31462569004731205A302E31462518
:1009900069004731205925694625690047312059AA
:1009A0002D302E314625690047312059302E3146F1
:1009B00025690047312058256946256900473120BF
:1009C000582D302E314625690047312058302E31C0
:1009D0004625690047393100473238004732382010
:1009E0005A004732382059004732382058004132E7
:1009F000305620004A3036004D3834004A3034003A
:100A00004A3136004A303500454E4400464E2000FB
:100A10004A3032003939393A393939004D00480005
:100A20004137562000413656202D2D2D0041365697
:100A300020005A3A2000593A2000583A2000413507
:100A40005600413456200041335620004132562092
:100A500000413156200041305620004D31313000E8
:100A60004A3132004A3033004A3135004A323300CD
:100A7000FFFFFF0000A0400000A040000000400079
:100A8000005C430000574300004E430000A0C0003C
:100A90000000000000000000005743000057430022
:100AA000004E430000A0C000000000000000004F06
:100AB0004B0045525220006563686F3A00457272E0
:100AC0006F723A007C3C3E5E2B3D3F2F5B5D3B2CC2
:100AD0002A225C004A3134004D3331004D38342035
:100AE000582059205A20450043616E6E6F7420656E
:100AF0006E746572207375626469723A2000617564
:100B0000746F25692E67006572726F722077726943
:100B100074696E6720746F2066696C650A004E6F99
:100B200074205344207072696E74696E670A0053B2
:100B300044207072696E74696E67206279746520F2
:100B40000044656C6574696F6E206661696C6564EC
:100B50002C2046696C653A200046696C6520646506
:100B60006C657465643A006F70656E206661696CCF
:100B700065642C2046696C653A2000577269746977
:100B80006E6720746F2066696C653A20004A3231C6
:100B9000006F70656E206661696C65642C20466923
:100BA0006C653A20004A3231006F70656E206661D4
:100BB000696C65642C2046696C653A20004A3230C5
:100BC0000046696C652073656C65637465640A0032
:100BD0002053697A653A200046696C65206F70651C
:100BE0006E65643A20004A3231006F70656E20668F
:100BF00061696C65642C2046696C653A200020664A
:100C0000696C653A20004E6F7720002220706F7368
:100C1000002220706172656E743A22005355425270
:100C20004F5554494E452043414C4C2074617267E6
:100C300065743A22004B494C4C45442E2000747296
:100C400079696E6720746F2063616C6C20737562C4
:100C50002D67636F64652066696C657320776974BE
:100C60006820746F6F206D616E79206C6576656C9D
:100C7000732E204D4158206C6576656C2069733A5F
:100C8000004A3032004A31360047393000473120BF
:100C90005A2D3230004D3234004D3233202573004E
:100CA00053442063617264206F6B0A006F70656E3D
:100CB000526F6F74206661696C65640A00766F6CB0
:100CC000756D652E696E6974206661696C65640A6C
:100CD00000534420696E6974206661696C0A0020C3
:100CE000204D3230302044300A0020204D32303048
:100CF0002044002044697361626C65640A0046699F
:100D00006C616D656E742073657474696E67733A97
:100D10000020440020490020204D33303120500075
:100D20005049442073657474696E67733A0A0020F1
:100D3000460020420020480020204D313435205309
:100D4000004D6174657269616C20686561747570CD
:100D500020706172616D65746572733A0A002020BB
:100D60004D363636205A005A3220456E6473746F01
:100D7000702061646A7573746D656E7420286D6D82
:100D8000293A0A00205A0020590020204D323036DE
:100D9000205800486F6D65206F6666736574202863
:100DA0006D6D290A00204500205A00205900205866
:100DB0000020420020540020204D323035205300C6
:100DC000416476616E636564207661726961626C0C
:100DD00065733A20533D4D696E20666565647261A6
:100DE000746520286D6D2F73292C20543D4D696E3C
:100DF0002074726176656C206665656472617465E5
:100E000020286D6D2F73292C20423D6D696E696D10
:100E1000756D207365676D656E742074696D6520EE
:100E2000286D73292C20583D6D6178696D756D2092
:100E30005859206A65726B20286D6D2F73292C20FC
:100E4000205A3D6D6178696D756D205A206A657212
:100E50006B20286D6D2F73292C2020453D6D617806
:100E6000696D756D2045206A65726B20286D6D2F48
:100E700073290A0020540020520020204D323034C3
:100E8000205000416363656C65726174696F6E73B5
:100E90003A20503D7072696E74696E672C20523D25
:100EA0007265747261637420616E6420543D747263
:100EB0006176656C0A00204500205A002059002008
:100EC000204D3230312058004D6178696D756D20AC
:100ED000416363656C65726174696F6E20286D6D26
:100EE0002F7332293A0A00204500205A0020590069
:100EF00020204D3230332058004D6178696D756D7A
:100F00002066656564726174657320286D6D2F734A
:100F1000293A0A00204500205A0020590020204D7F
:100F200039322058005374657073207065722075D3
:100F30006E69743A0A0048617264636F6465642084
:100F400044656661756C742053657474696E67736B
:100F5000204C6F616465640A00454550524F4D2036
:100F6000636865636B73756D206D69736D61746320
:100F7000680A00206279746573290A002073746F0F
:100F80007265642073657474696E6773207265742A
:100F9000726965766564202800206279746573291A
:100FA0000A0053657474696E67732053746F7265B9
:100FB000642028004572726F722077726974696EBE
:100FC0006720746F20454550524F4D210A007A32F8
:100FD0005F6D696E3A20007A5F6D696E3A20007924
:100FE0005F6D696E3A2000785F6D696E3A2000523D
:100FF00065706F7274696E6720656E6473746F706C
:10100000207374617475730A0020746F6F206C6FA5
:101010006E6720657874727573696F6E2070726583
:1010200076656E7465640A004A31330020636F6C24
:101030006420657874727573696F6E20707265765E
:10104000656E7465640A00205A3A0020593A0020FF
:10105000436F756E7420583A20004D383420582064
:1010600059205A20450024F4D43050C38E20C2A207
:101070004017828B7011127A910D816CD90AA86188
:10108000E108C7586607615143061E4B5D05C1451F
:10109000A7041A411104093D980371393103403600
:1010A000DB0265339102D4305402802E1D02632C82
:1010B000EE01752AC501B028A001102781018F25F6
:1010C00064012B244B01E0223401AC211F018D204F
:1010D0000D01801FFC00841EED00971DDF00B81C71
:1010E000D200E61BC600201BBC00641AB200B21975
:1010F000A8000A19A0006A189900D117910040179A
:101100008B00B516840031167E00B31579003A15B0
:101110007300C7146F0058146A00EE13660088133A
:10112000630025135E00C7125B006C125700151296
:101130005400C111510070114F0021114B00D61005
:1011400049008D1047004610440002104200C00FB5
:101150004000800F3E00420F3C00060F3B00CB0ECC
:101160003800930E37005C0E3500270E3400F30D67
:101170003200C10D3100900D3000600D2E00320D97
:101180002D00050D2C00D90C2B00AE0C2900850C70
:1011900029005C0C2700350C27000E0C2600E80BFC
:1011A0002400C40B2400A00B23007D0B23005A0B4A
:1011B0002100390B2100180B2000F80A1F00D90A62
:1011C0001E00BB0A1E009D0A1D00800A1D00630A46
:1011D0001C00470A1B002C0A1B00110A1A00F70901
:1011E0001A00DD091900C4091900AB091900920998
:1011F00017007B091800630917004C09160036090F
:101200001600200916000A091500F5081500E00867
:101210001400CC081400B8081400A40814009008A6
:1012200013007D0812006B081300580812004608CE
:1012300012003408110023081100120811000108DF
:101240001100F0071000E0071000D0071000C007E1
:101250001000B0070F00A107100091070E008307D0
:101260000F0074070F0065070E0057070E004907AF
:101270000E003B070D002E070E0020070D00130780
:101280000D0006070D00F9060C00ED060D00E00646
:101290000C00D4060C00C8060C00BC060C00B006FE
:1012A0000C00A4060B0099060C008D060B008206AC
:1012B0000B0077060B006C060B0061060A00570650
:1012C0000B004C060A0042060A0038060A002E06E9
:1012D0000A0024060A001A060A001006090007067A
:1012E0000A00FD050900F4050900EB050900E20507
:1012F0000900D9050900D0050900C7050900BE0588
:101300000900B5050800AD050800A50509009C0504
:101310000800940508008C050800840508007C0579
:101320000800740508006C050700650508005D05E8
:101330000700560508004E05070047050700400551
:10134000080038050700310507002A0507002305B6
:1013500007001C050600160507000F050700080515
:10136000060002050700FB040600F5040700EE0472
:101370000600E8040600E2040700DB040600D504CA
:101380000600CF040600C9040600C3040600BD041D
:101390000600B7040600B1040500AC040600A6046C
:1013A0000600A00405009B040600950405009004B7
:1013B00006008A04050085040500800406007A04FE
:1013C000050075040500700405006B040500660443
:1013D0000500610405005C04050057040500520483
:1013E00005004D04050048040500430405003E04C3
:1013F00004003A04050035040500300404002C0400
:10140000050027040400230405001E0404001A0438
:10141000040016040500110404000D04040009046E
:1014200005000404040000040400FC030400F803A5
:101430000400F4030400F0030400EC030400E803D8
:101440000400E4030400E0030400DC030400D80308
:101450000400D4030400D0030400CC030400C80338
:101460000300C503030024F404D9201BC40C5C0E44
:101470009804C4095F0265077101F405F900FB04D3
:10148000B30048048700C1036900580355000303F3
:101490004500BE023A008402310053022A002902AC
:1014A000250004022000E4011C00C8011900AF015E
:1014B00017009801140084011300710110006101EC
:1014C000100051010E0043010D0036010B002B01ED
:1014D0000B0020010B00150109000C01090003019C
:1014E0000800FB000800F3000800EB000700E40020
:1014F0000600DE000600D8000600D2000600CC0080
:101500000500C7000500C2000500BD000400B900C9
:101510000400B5000400B1000400AD000400A900FF
:101520000400A5000300A20003009F0004009B002C
:101530000300980003009500020093000300900050
:1015400003008D0002008B0003008800020086006B
:10155000020084000300810002007F0002007D0081
:1015600002007B0002007900020077000100760093
:1015700002007400020072000100710002006F009E
:1015800002006D0001006C0002006A0001006900A9
:1015900002006700010066000100650001006400B0
:1015A00002006200010061000100600001005F00B4
:1015B00002005D0001005C0001005B0001005A00B8
:1015C00001005900010058000100570001005600B9
:1015D00001005500010054000100530000005300B9
:1015E00001005200010051000100500001004F00B5
:1015F00001004E0000004E0001004D0001004C00B3
:1016000001004B0000004B0001004A0001004900AE
:1016100001004800000048000100470001004600AA
:1016200000004600010045000000450001004400A4
:10163000010043000000430001004200000042009E
:1016400001004100000041000100400001003F0096
:1016500000003F0001003E0000003E0001003D0090
:1016600000003D0001003C0000003C0000003C0088
:1016700001003B0000003B0001003A0000003A007E
:101680000100390000003900010038000000380076
:10169000000038000100370000003700010036006C
:1016A0000000360000003600010035000000350063
:1016B0000000350001003400000034000000340058
:1016C000010033000000330000003300010032004D
:1016D0000000320000003200010031000000310043
:1016E0000000310001003000000030000000300038
:1016F00001002F0000002F0000002F0000002F002D
:1017000001002E0000002E0000002E0001002D0020
:1017100000002D0000002D0000002D0001002C0015
:1017200000002C0000002C0000002C0001002B0009
:1017300000002B0000002B0000002B0001002A00FD
:1017400000002A0000002A0000002A0001002900F1
:1017500000002900000029000000290000002900E5
:1017600001002800000028000000280000002800D8
:1017700000002800010027000000270000002700CB
:1017800000002700000027000100260000002600BE
:1017900000002600000026000000260001002500B1
:1017A00000002500000025000000250000002500A5
:1017B0000000250001002400000024000000240097
:1017C000000024000000240001002300000023008A
:1017D000000023000000230000002300000023007D
:1017E000000023000100220000002200000022006F
:1017F0000000220000002200000022000100210061
:101800000000210000002100000021000000210054
:101810000000210000002100010020000000200045
:101820000000200000002000000020000000200038
:10183000000020000000200001001F0000001F0029
:1018400000001F0000001F0000001F0000001F001C
:1018500000001F0001001E0000001E0000001E000E
:1018600000001E0000004D494E54454D502074723A
:1018700069676765726564004572723A204D494E2A
:1018800054454D5020424544004572723A204D491E
:101890004E54454D50004D415854454D50207472A2
:1018A00069676765726564004572723A204D4158F8
:1018B00054454D5020424544004572723A204D41F6
:1018C0005854454D50006265640A002C20737973AA
:1018D00074656D2073746F70706564212048656154
:1018E0007465725F49443A200023646566696E65D9
:1018F000202044454641554C545F4B6420002364EE
:101900006566696E65202044454641554C545F4BE1
:1019100069200023646566696E6520204445464160
:10192000554C545F4B702000504944204175746FF2
:1019300074756E652066696E6973686564212050F0
:10194000757420746865206C617374204B702C2052
:101950004B6920616E64204B6420636F6E73746109
:101960006E74732066726F6D2062656C6F7720698C
:101970006E746F20436F6E66696775726174696F0C
:101980006E2E680A00504944204175746F74756E5C
:1019900065206661696C6564212074696D656F7589
:1019A000740A00504944204175746F74756E652047
:1019B0006661696C6564212054656D70657261743F
:1019C00075726520746F6F20686967680A00204B24
:1019D000643A2000204B693A2000204B703A2000E6
:1019E0000A20436C617373696320504944200A00E4
:1019F0002054753A2000204B753A2000206D617804
:101A00003A2000206D696E3A200020643A200020C0
:101A1000626961733A20001000C90210012C014074
:101A200001220170011801B0010E01F00104015002
:101A300002FA00B002F0003003E600D003DC0090B0
:101A400004D2007005C800A006BE000008B400B0B3
:101A500009AA00D00BA000600E960060118C000057
:101A600015820020197800C01D6E00A0226400B00D
:101A7000275A00902C500000314600E0343C001002
:101A8000383200903A2800603C1E00A03D140080CF
:101A90003E0A00203F000070012C0190012701B098
:101AA000012201C0011D01F00118011002130130D3
:101AB000020E016002090190020401C002FF000051
:101AC00003FA004003F5008003F000D003EB002090
:101AD00004E6007004E100E004DC004005D700C02B
:101AE00005D2004006CD00D006C8008007C30030F4
:101AF00008BE00F008B900C009B400B00AAF00B0D9
:101B00000BAA00D00CA500000EA000500F9B00C037
:101B10001096005012910000148C00C0158700B080
:101B2000178200B0197D00D01B7800001E730040A2
:101B3000206E0090226900F024640040275F00902E
:101B4000295A00E02B5500102E500020304B001079
:101B5000324600E033410090353C001037370070CA
:101B6000383200A0392D00B03A2800A03B23006095
:101B70003C1E00103D1900903D1400103E0F0070F7
:101B80003E0A00C03E0500003F00004A30310043DD
:101B90006172642072656D6F766564004A30300052
:101BA0004361726420696E73657274656400052E0A
:101BB0002E004D61696E0046696C2E204469612ECD
:101BC0000046696C2E204469612E004520696E2014
:101BD0006D6D33004F6666004F6E2000436F6E746C
:101BE000726F6C004573746570732F6D6D00457373
:101BF000746570732F6D6D005A73746570732F6DFB
:101C00006D005A73746570732F6D6D005973746530
:101C100070732F6D6D005973746570732F6D6D0047
:101C20005873746570732F6D6D005873746570739D
:101C30002F6D6D00412D74726176656C00412D74BD
:101C4000726176656C00412D726574726163740017
:101C5000412D7265747261637400416D6178204535
:101C600000416D6178204500416D6178205A004146
:101C70006D6178205A00416D6178205900416D6195
:101C800078205900416D6178205800416D617820BD
:101C900058005654726176206D696E005654726118
:101CA00076206D696E00566D696E00566D696E0026
:101CB000566D6178204500566D6178204500566D5F
:101CC0006178205A00566D6178205A00566D61780F
:101CD000205900566D6178205900566D6178205862
:101CE00000566D617820580056652D6A65726B004C
:101CF00056652D6A65726B00567A2D6A65726B00A7
:101D0000567A2D6A65726B0056792D6A65726B0082
:101D100056792D6A65726B0056782D6A65726B0074
:101D200056782D6A65726B00416363656C00416390
:101D300063656C00436F6E74726F6C0053746F72E6
:101D400065206D656D6F727900426564004265645F
:101D5000004E6F7A7A6C65004E6F7A7A6C65004639
:101D6000616E2073706565640046616E20737065F6
:101D700065640054656D70657261747572650050BC
:101D80007265686561742041425320636F6E66001E
:101D90005072656865617420504C4120636F6E66B7
:101DA000005049442D44005049442D4400504944BA
:101DB0002D49005049442D49005049442D500050B0
:101DC00049442D5000200220466163740020022007
:101DD00046616374002002204D6178002002204D8E
:101DE0006178002002204D696E002002204D696E4E
:101DF000004175746F74656D70004F6666004F6EBC
:101E0000200046616E2073706565640046616E2037
:101E100073706565640042656400426564004E6FDE
:101E20007A7A6C65004E6F7A7A6C6500436F6E74D7
:101E3000726F6C00526573746F7265206661696CB5
:101E400073616665004C6F6164206D656D6F7279BA
:101E50000053746F7265206D656D6F72790046690D
:101E60006C616D656E74004D6F74696F6E005465C2
:101E70006D7065726174757265004D61696E004DBB
:101E80006F766520302E316D6D004D6F7665203197
:101E90006D6D004D6F76652031306D6D005072654F
:101EA00070617265004578747275646572004D6F7B
:101EB0007665205A004D6F76652059004D6F766526
:101EC0002058004D6F7665206178697300457874FD
:101ED0007275646572004D6F7665205A004D6F769D
:101EE000652059004D6F7665205800436F6F6C6414
:101EF0006F776E00507265686561742041425300CF
:101F00005072656865617420504C41004D38340052
:101F100044697361626C6520737465707065727377
:101F2000004D6F7665206178697300536574206891
:101F30006F6D65206F666673657473004732380095
:101F40004175746F20686F6D65004D61696E00505A
:101F50007265686561742041425320426564005097
:101F6000726568656174204142530050726570610A
:101F70007265005072656865617420504C41204262
:101F80006564005072656865617420504C41005072
:101F900072657061726500466C6F7700466C6F7792
:101FA0000046616E2073706565640046616E207343
:101FB000706565640042656400426564004E6F7A36
:101FC0007A6C65004E6F7A7A6C6500537065656453
:101FD000005370656564004D61696E004D343238A0
:101FE000004E6F2053442063617264005072696E2A
:101FF000742066726F6D2053440053746F702070AC
:1020000072696E7400526573756D65207072696EC9
:1020100074005061757365207072696E7400436F4F
:102020006E74726F6C0050726570617265005475E9
:102030006E6500496E666F2073637265656E00257C
:10204000753A2530327500253032753A25303275B3
:10205000002D2D2D005344005A0059005800012036
:1020600000012000506C65617365207265736574B2
:10207000005052494E5445522048414C544544006A
:1020800000000A0B02090C0D0E08070304010000F2
:102090000000000000000000000000000000000040
:1020A00000000000000000000000000012111000FD
:1020B0000000000000000000000000000000000020
:1020C000000000000000010210202008081020403D
:1020D00010204080020102010804020101020408EC
:1020E000102040808040201008040201800402017A
:1020F00080402010080402010804020101020408C3
:1021000010204080010204081020408005050505CC
:10211000070508080808020202020A0A080804045F
:10212000040401010101010101010303030303038D
:102130000303040707070C0C0C0C0C0C0C0C02021C
:10214000020206060606060606060B0B0B0B0B0B19
:102150000B0B000020002300260029002C002F007C
:102160003200000100000301060109010000220005
:10217000250028002B002E00310034000201000051
:10218000050108010B0100002100240027002A009E
:102190002D003000330001010000040107010A0195
:1021A000024E414E494E495459494E46CDCCCC3D44
:1021B0000AD7233C17B7D13877CC2B329595E62434
:1021C0001FB14F0A000020410000C84200401C46D9
:1021D00020BCBE4CCA1B0E5AAEC59D747C30074B4A
:1021E000898511A19A3011241FBECFEFD1E2DEBF45
:1021F000CDBF00E00CBF14E0A0E0B2E0E4EFF7EBED
:1022000001E00BBF02C007900D92A03CB107D9F7C7
:1022100025E1A0ECB4E001C01D92AC3CB207E1F7AF
:1022200011E2C4EED1E200E006C022970109FE01EE
:102230000BBF0E947AD4CC3DD10780E00807A9F7F4
:102240000E9406D00C94E9DB0C9400001F920F92C0
:102250000FB60F9211240BB60F922F933F938F93CB
:102260009F93EF93FF932091C6009FB7F894E0915E
:10227000400581E08E0F8F7730914105831731F053
:10228000F0E0E054FB4F2083809340059FBFFF9117
:10229000EF919F918F913F912F910F900BBE0F90D7
:1022A0000FBE0F901F9018959B01AC01211581EE78
:1022B00038074105510549F182E08093C00060E094
:1022C00079E08DE390E00E944ED42150310941091C
:1022D0005109CA01B90122E030E040E050E00E941B
:1022E0004ED43093C5002093C4008091C10080611A
:1022F0008093C1008091C10088608093C10080916B
:10230000C10080688093C10008951092C00020E150
:1023100030E0E7CF3FB7F894209141058091400528
:10232000821759F0E22FF0E0E054FB4F808190E0FB
:102330002F5F2F772093410502C08FEF9FEF3FBFA4
:1023400008952FB7F89480914005909141052FBFD3
:10235000891B8F7708958FB7F894909141059093DA
:1023600040058FBF08959091C00095FFFCCF8093EA
:10237000C6000895AF92BF92CF92DF92EF92FF9284
:102380000F931F93CF93DF93CDB7DEB7A0970FB610
:10239000F894DEBF0FBECDBF6115710581059105B3
:1023A000A9F1B12CC42ED12CE12CF12CAA24A39498
:1023B000AB0C01E010E00C0F1D1F0B0D111DB7FC45
:1023C0001A95A70196010E942CD4F8016083B901E7
:1023D000CA01611571058105910511F41B2D11C00C
:1023E000BA2CE4CFE1E0F0E0EC0FFD1FE10FF11DAE
:1023F00017FDFA9580818A3038F490E3890FB3DFB6
:1024000011501F3F79F714C097E3F8CF80E3A096EF
:102410000FB6F894DEBF0FBECDBFDF91CF911F91F5
:102420000F91FF90EF90DF90CF90BF90AF909BCF38
:10243000A0960FB6F894DEBF0FBECDBFDF91CF914F
:102440001F910F91FF90EF90DF90CF90BF90AF90D2
:1024500008954115510511F4862F85CF8BCFCF926A
:10246000DF92EF92FF926B017C0197FF0AC08DE231
:102470007ADFF094E094D094C094C11CD11CE11C8C
:10248000F11C4AE0C701B601FF90EF90DF90CF90BA
:1024900071CF4115510511F4862F65CF4A30510592
:1024A00009F4DDCF67CFAB01BC01882777FD8095AC
:1024B000982FEFCF8DE057DF8AE055CFAB01BC01FD
:1024C00080E090E0C6DFF6CF8F929F92AF92BF92EE
:1024D000CF92DF92EF92FF92CF936B017C01B42EEB
:1024E00020E030E0A9010E94EED087FF06C08DE217
:1024F0003ADFF7FAF094F7F8F094C0E060E070E0AB
:1025000080E09FE3CB1541F02DEC3CEC4CEC5DE31F
:102510000E942CD3CF5FF6CF9B01AC01C701B6015F
:102520000E9415D06B017C010E9462D14B015C01BD
:102530004AE020DFCC2381F1C501B4010E948ED195
:102540009B01AC01C701B6010E9414D06B017C0154
:102550008EE209DF20E030E040E251E4C701B6013D
:102560000E942CD36B017C010E945DD14B01AA24F7
:1025700097FCA094BA2CC501B40171DFC501B40168
:102580000E9490D19B01AC01C701B6010E9414D0FA
:102590006B017C01C150F1F6CF91FF90EF90DF907D
:1025A000CF90BF90AF909F908F9008958DCFFC01FA
:1025B00065917591859194910895CF93DF93EBE2A6
:1025C000F7E08491EF012196882319F0CCDEFE011B
:1025D000F8CF6091EB077091EC078091ED07909137
:1025E000EE0742E050E0E2DFE7E2F7E08491EF013E
:1025F0002196882319F0B7DEFE01F8CF6091EF072E
:102600007091F0078091F1079091F20742E050E05D
:10261000CDDFE3E2F7E08491EF012196882319F002
:10262000A2DEFE01F8CF6091F3077091F40780916C
:10263000F5079091F60742E050E0B8DFEFE1F7E0F0
:102640008491EF012196882319F08DDEFE01F8CFE9
:102650006091F7077091F8078091F9079091FA0758
:1026600042E050E0A3DFDF91CF910C94458D809143
:10267000D5149091D61490938C0A80938B0A8091F4
:10268000D1149091D21490938A0A8093890A8091F0
:10269000910A813049F50E946A925F9A1092D5079B
:1026A0008A9A479A1092D6079FB7F89480910801AA
:1026B0008160809308019FBF479A1092D707129AB2
:1026C0000E942A701092910A80918B0A90918C0A34
:1026D0009093D6148093D5148091890A90918A0A98
:1026E0009093D2148093D1140895CF92DF92EF92F9
:1026F000FF920F931F93CF93DF93EC010E9424C8A6
:102700000E811F81288539850115110521053105A7
:1027100059F53C853323A9F12A8531503C8731E0B6
:10272000320F3A874D85341301C01A86FE0134E01A
:10273000239FE00DF11D112406851785208931891D
:102740000A831B832C833D836B017C01C00ED11E49
:10275000E11CF11CCE82DF82E886F9868C819D81A6
:10276000892B79F0469A0DC06B017C01C01AD10A01
:10277000E20AF30AF7FC05C046981E821F821886FB
:102780001986DF91CF911F910F91FF90EF90DF900D
:10279000CF900895DC01ED91FC910190F081E02D46
:1027A00019940E9424C860931406709315068093B0
:1027B00016069093170608958091B80F9091B70F61
:1027C000891B8F700895CF92DF92EF92FF920F9343
:1027D0001F93CF93DF93EB01FC01608171818281B4
:1027E00093812CE3C22ED12CE12CF12CA701960170
:1027F0000E942CD4162F072FCA01B901A7019601F8
:102800000E942CD4F62EE72ECA01B90128E130E04F
:1028100040E050E00E942CD4FB01C9016DE671E05C
:102820000E9405D49B014F2D5E2D21153105D9F055
:102830000F931F93EF92FF92FF93EF939F938F93CA
:102840003F932F9383EA96E09F938F93DF93CF93E9
:102850000E940ED98DB79EB70E960FB6F8949EBF04
:102860000FBE8DBF5BC00097C9F00F931F93EF920F
:10287000FF92FF93EF939F938F9383E996E09F934B
:102880008F93DF93CF930E940ED9EDB7FEB73C969E
:102890000FB6F894FEBF0FBEEDBF40C03097B9F041
:1028A0000F931F93EF92FF92FF93EF9387E896E0C9
:1028B0009F938F93DF93CF930E940ED98DB79EB7CE
:1028C0000A960FB6F8949EBF0FBE8DBF27C0452B4A
:1028D000A9F00F931F93EF92FF928FE796E09F93DB
:1028E0008F93DF93CF930E940ED9EDB7FEB7389642
:1028F0000FB6F894FEBF0FBEEDBF10C00F931F932D
:102900008BE796E09F938F93DF93CF930E940ED92E
:102910000F900F900F900F900F900F90DF91CF912D
:102920001F910F91FF90EF90DF90CF900895EF925D
:10293000FF920F931F93CF93DF93EC017B018A01EA
:102940006C854D8564130AC0E881F9810190F0819E
:10295000E02DCE0119950E941091F2CFF701208150
:102960003181F801808191815B85FE0174E0579F80
:10297000E00DF11D11243E963183208393838283E1
:102980006F5F6C8781E0850F841711F08B8701C022
:102990001B86DF91CF911F910F91FF90EF900895CB
:1029A0000F931F93CF93DF931F921F92CDB7DEB784
:1029B000FC0184918F010F5F1F4F811102C08B01B9
:1029C00007C069837A83CFDCF80169817A81F1CF0E
:1029D000D8018D918D01882311F0C5DCF9CF0F90BE
:1029E0000F90DF91CF911F910F9108950F931F9337
:1029F000CF93DF93EB01FC0184918F010F5F1F4F99
:102A0000882319F0B0DCF801F7CF6AE070E0CE015E
:102A1000DF91CF911F910F9146CDCF92DF92EF9230
:102A2000FF92CF93DF936A017B01FC018491EF0158
:102A30002196882319F097DCFE01F8CF4AE050E098
:102A4000C701B601DF91CF91FF90EF90DF90CF905B
:102A500020CDCF92DF92EF92FF92CF93DF936A0166
:102A60007B01FC018491EF012196882319F07BDC26
:102A7000FE01F8CF42E050E0C701B601DF91CF91EF
:102A8000FF90EF90DF90CF9091CDCF92DF92EF92B9
:102A9000FF92CF93DF936A017B01FC018491EF01E8
:102AA0002196882319F05FDCFE01F8CF42E050E068
:102AB000C701B601DF91CF91FF90EF90DF90CF90EB
:102AC00075CDCF92DF92EF92FF92CF93DF936A01A1
:102AD0007B01FC018491EF012196882319F043DCEE
:102AE000FE01F8CF4AE050E0C701B601DF91CF9177
:102AF000FF90EF90DF90CF90ACCC60E08FE40E942D
:102B00000FCA61E08AE30E940FCA8C98089560E0C2
:102B100083E10E940FCA5A9A2FEF80E792E021507A
:102B200080409040E1F700C000000895CF93DF930C
:102B30008091C705811109C089B182FB882780F97E
:102B40008093BC0581E08093C70549B142FB4427CF
:102B500040F94093BB05242F30E08091BC059927B4
:102B600087FD9095821793070CF05AC08091B905A4
:102B70009091BA0501969093BA058093B905803873
:102B80009E4308F456C01092BA051092B9050E94EF
:102B90008E738091FE07882321F1ECE6FAE06491C0
:102BA000EF01662351F0772767FD70958FE29CE077
:102BB000F1DD2196FE016491F4CF6DE070E08FE2CB
:102BC0009CE0E8DD6AE070E08FE29CE0E3DD81E01C
:102BD00080938F0A8093BD058093EA0E1092FE07C2
:102BE0001AC0E8E6FAE06491EF01662351F0772716
:102BF00067FD70958FE29CE0CDDD2196FE0164912A
:102C0000F4CF6DE070E08FE29CE0C4DD6AE070E03C
:102C10008FE29CE0BFDD8091BB058093BC0509C0BD
:102C20002817390731F01092BA051092B905409370
:102C3000BC05DF91CF910895CF93DF939091260C3F
:102C40008091C605911131C0882309F479C0809123
:102C5000B5059091B605A091B705B091B80501965C
:102C6000A11DB11D8093B5059093B605A093B7053E
:102C7000B093B8051092C6050297A105B1050CF4F2
:102C80005FC081E08093260CE4E6FAE06491EF01F6
:102C9000662309F438C0772767FD70958FE29CE0C2
:102CA00079DD2196FE016491F3CF81113FC08091BF
:102CB000B5059091B605A091B705B091B8050196FC
:102CC000A11DB11D8093B5059093B605A093B705DE
:102CD000B093B8058135934CA105B1058CF11092E4
:102CE000C6051092260CE0E6FAE06491EF01662337
:102CF00051F0772767FD70958FE29CE04BDD2196C0
:102D0000FE016491F4CF6DE070E08FE29CE042DD63
:102D10006AE070E08FE29CE03DDD1092B505109214
:102D2000B6051092B7051092B8050AC01092B50505
:102D30001092B6051092B7051092B8051092C6050C
:102D4000DF91CF9108950E9424C860931406709378
:102D50001506809316069093170608958091960A9B
:102D60009091970A60E070E001960C948DD4682FE2
:102D7000772767FD70952091A20A3091A30A40E65B
:102D8000429FC001439F900D11248A55954F0E9488
:102D9000BCD89093970A8093960A21E0892B09F476
:102DA00020E0822F08958091FF07882389F01092F8
:102DB000E90E1092E80E81E0809338026AE070E03C
:102DC00080E090E00E9453C88CEF97E00E94985DED
:102DD0008091E80E9091E90E0895CF92DF92EF92E4
:102DE000FF926C01EE24D7FCE094FE2C1616170619
:102DF0008CF420E030E0A9018FE10E9472CCC70181
:102E0000B6010E9453C88FE1FF90EF90DF90CF9002
:102E10000C9493CFC701B601FF90EF90DF90CF9055
:102E20000C9453C88091BE0581111FC0659B02C0E0
:102E300038E001C030E090910901991F9927991F4E
:102E4000990F990F8091090186FF02C022E001C00D
:102E500020E089B183FB882780F9832B892B822B83
:102E60008093B40581E08093BE05659B02C028E095
:102E700001C020E080910901881F8827881F880FE2
:102E8000880F9091090196FF02C092E001C090E086
:102E900049B143FB442740F9422B482B492B40932F
:102EA000B305242F332727FD30958091B40599274A
:102EB00087FD9095281739079CF48091B2058F5FA4
:102EC0008093B2058A3F98F01092B20560ED77E0EA
:102ED0008CE390E082DF8091B3058093B405089580
:102EE0002817390721F01092B2054093B4050895D0
:102EF0000E9487710E942B718091EF0E8A3599F0A4
:102F00008AE58093EF0E0E94FE708DEC9CECACE4A1
:102F1000BEE38093290C90932A0CA0932B0CB093C2
:102F20002C0C0C944D718091EB0E9091EC0EA091B5
:102F3000ED0EB091EE0E8093290C90932A0CA09385
:102F40002B0CB0932C0C0895EAE0F1E080818062B4
:102F500080839FB7F894EBE0F1E080818F7D8083E0
:102F60009FBF089520E030E042E852E46091DD1414
:102F70007091DE148091DF149091E0140E94F1D2E0
:102F80009FB718162CF4F89480910B01806204C04E
:102F9000F89480910B018F7D80930B019FBF089562
:102FA0008CEF97E00C94075E27EF37E043EF57E094
:102FB0006FEE77E08BEE97E00C94B4838F929F9244
:102FC000BF92CF92DF92EF92FF920F931F93CF9316
:102FD000DF9300D01F92CDB7DEB7B22ED32E4C01B7
:102FE000880C991C880C991CC4018551984F7C0150
:102FF000FC01108211821282138249835A836B83EF
:103000007C83D2DF49815A816B817C81F7014083C7
:10301000518362837383C0901C0620E030E0A901D5
:10302000B8018B2D9D2D0E94EED0811108C0F401B6
:10303000E652FC4F90818181B280D38002C0902FF4
:10304000812FE92EF82E0B2D1D2D27EF37E043EFB2
:1030500057E06FEE77E08BEE97E00E94F6780E94E3
:103060006D8C10920A0F0F900F900F900F90DF91C0
:10307000CF911F910F91FF90EF90DF90CF90BF9075
:103080009F908F90089580914B0680934C061092EC
:103090004A06089520914B0630E0F901E153FA4FBA
:1030A0008083C90101968370992780934B06809194
:1030B0004A068F5F80934A060895CF93FC01C62F7E
:1030C00080818B3399F080914A06843078F4209186
:1030D0004B0630E6239FC0011124BF01835B994F4B
:1030E0000E94D0D88C2FD6DF81E001C080E0CF9144
:1030F00008950F931F93CF93DF93EC01DEDF8823B6
:10310000A9F0E7EBFAE084918F010F5F1F4F88234E
:1031100019F029D9F801F7CFBE018AE199E040DC26
:1031200082E221D98AE01FD981E001C080E0DF91ED
:10313000CF911F910F910895DF92EF92FF920F931D
:103140001F93CF93DF93CDB7DEB76E970FB6F8948A
:10315000DEBF0FBECDBF6091420670914306611580
:10316000710559F14DE150E08E010F5F1F4FC8010D
:103170000E945FD81E8EF8017F01E01AF10AD190FB
:10318000DD2019F08AE0D812F7CFF801EE0DFF1D0F
:10319000108260E0C801ADDF882379F0DD20B1F056
:1031A0008FEFE81AF80A80914206909143068E0D3F
:1031B0009F1D909343068093420681E02091420632
:1031C00030914306232B39F480E005C0109243066A
:1031D00010924206F2CF6E960FB6F894DEBF0FBE85
:1031E000CDBFDF91CF911F910F91FF90EF90DF90B6
:1031F000089590934306809342069ECF80914A069D
:103200008430E8F48091AF058F5F8093AF05813003
:1032100039F48FE299E090934306809342068CDF65
:103220008091AF05823059F487E299E0909343068C
:103230008093420681DF1092BD051092AF0508957C
:103240009898A09A08958F929F92AF92BF92CF9232
:10325000DF92EF92FF920F931F93CF93DF93CDB73F
:10326000DEB728970FB6F894DEBF0FBECDBF8091B2
:10327000FE07882309F485C180914A06811102C0A6
:1032800010924D059924939440917A0A50917B0AAB
:1032900060917C0A70917D0A8091760A9091770AFC
:1032A000A091780AB091790A481759076A077B07F5
:1032B00008F4912C00E010E0BB24B394F0E6AF2EAC
:1032C00090914A0680912E0C943008F0B1C0911074
:1032D000AFC090914D059111ABC08111A9C08091F3
:1032E000D1099091D209A091D309B091D4098093CA
:1032F0007A0A90937B0AA0937C0AB0937D0A89ECAA
:1033000099E00E941250882E99249394C0907A0AD2
:10331000D0907B0AE0907C0AF0907D0A4091760A7A
:103320005091770A6091780A7091790AC416D5068F
:10333000E606F706C0F4912C8F3F2FEF920751F16C
:103340004AE0841709F445C0ADE08A1709F441C08A
:10335000B3E28B1719F02AE3821350C020914C0579
:1033600021114CC031C0E1EDF7E084917F014FEFB6
:10337000E41AF40A882321F00E94B311F701F5CF73
:103380008CEF97E00E94A66661E08CEF97E00E94C8
:1033900085611AC0EDEBFAE084917F019FEFE91A95
:1033A000F90A882321F00E94B311F701F5CFE2EC6E
:1033B000F7E084917F01AFEFEA1AFA0A882321F03F
:1033C0000E94B311F701F5CFB3E28B1202C0B092A5
:1033D0004D0510924C050115110509F471CF80912E
:1033E0004B06F801A89EE00DF11D1124E35BF94F97
:1033F000108280E04FDE00E010E062CF0F35110553
:1034000008F05ECF2BE3821202C0B0924C052091EF
:103410004C05211155CF90914B06F801A99EE00D66
:10342000F11D1124E35BF94F80830F5F1F4F48CFDD
:10343000882309F4A6C0EDE4F6E02DEA36E08DE03D
:1034400097E06DE677E01192D9011D929D01DC01B4
:103450001D92CD01DB011D92BD01B6E0ED3AFB07E7
:1034600091F7C0901C0660912F027091300288275E
:1034700077FD8095982F0E9490D119821A821B8225
:103480001C8200E010E020EA30EC0D831E832F83C5
:1034900038877B018C0124EF3EE048EF5EE0BE01FF
:1034A0006F5F7F4FCE0105960E94F67864EF7EE055
:1034B00083E090E00E9470848091000F9091010F52
:1034C000A091020FB091030F8093DB079093DC076C
:1034D000A093DD07B093DE078091FC0E9091FD0E66
:1034E000A091FE0EB091FF0E8093DF079093E0074E
:1034F000A093E107B093E2072AE939E949E95EE3DD
:103500006091F3077091F4078091F5079091F607A9
:103510000E94F1D21816BCF42DEC3CEC4CEC5DE3AF
:103520006091F80E7091F90E8091FA0E9091FB0E59
:103530000E9414D06093F3077093F4078093F5070B
:103540009093F60710C08091F80E9091F90EA0911B
:10355000FA0EB091FB0E8093F3079093F407A093BB
:10356000F507B093F60785E595E5A5E0B2E480930D
:10357000310290933202A0933302B093340210923E
:103580002E0C28960FB6F894DEBF0FBECDBFDF918C
:10359000CF911F910F91FF90EF90DF90CF90BF9050
:1035A000AF909F908F9008950F931F93CF93DF93C9
:1035B000009144061091450665E470E0C8010E9440
:1035C000BCD8EC01C8010196209761F0188260E038
:1035D00070E00E948DD425E42883DF91CF911F9164
:1035E0000F91089560E070E0DF91CF911F910F91EE
:1035F0000C948DD480914406909145064AE050E0A9
:1036000060E070E001960C9426D78091440690917A
:1036100045064AE050E060E070E001960C94F5D574
:1036200080914406909145064AE050E060E070E0E9
:1036300001960E94F5D5CB010895809144069091A2
:1036400045064AE050E060E070E001960E9426D70F
:10365000CB01089580914406909145064AE050E0E0
:1036600060E070E001960E94F5D597FD20C0809142
:103670004406909145064AE050E060E070E0019613
:103680000E94F5D56F3F71058105910509F064F43D
:1036900080914406909145064AE050E060E070E079
:1036A00001960E94F5D501C06FEF862F089580E046
:1036B0000895E0914406F0914506218181E090E073
:1036C000203231F40196DF01A80FB91F2C91F8CFF9
:1036D0002D3211F02B3229F40196DF01A80FB91F0A
:1036E0002C912E3219F4E80FF91F218120532A3032
:1036F00038F4B0DF91E0811101C090E0892F089586
:1037000081E0089551CF50CF4FDF20E030E04AE70D
:1037100054E40E942CD30C9462D1682F772767FD64
:10372000709580914606909147060E94BCD8909370
:1037300045068093440621E0892B09F420E0822F7E
:1037400008950F931F93CF93DF93EC0184E5E5DF9A
:10375000882321F17FDF8823F9F0E7EBFAE08491F9
:103760008F010F5F1F4F882321F00E94B311F801D2
:10377000F6CF8DE40E94B3116AE070E0CE010E94A2
:10378000531268DF682F70E08FEA97E02FD98AE044
:103790000E94B31181E007C05DDF02C080911C066A
:1037A0008093E30580E0DF91CF911F910F91089501
:1037B000CF92DF92EF92FF920F931F93CF93DF93FD
:1037C000EC01CC0FDD1FCC0FDD1FFE01E15EF94FD8
:1037D00020E030E0A90160817181828193810E94A3
:1037E00015D0FE01E55DF94F208131814281538181
:1037F0000E9415D06B017C01CE018D55954F0E9422
:10380000D7128E01085E1D4FA70196010E9415D0A8
:10381000F8016083718382839383CE018956954F2B
:103820000E94D712C45FDD4FA70196010E9415D0F8
:10383000688379838A839B83DF91CF911F910F9156
:10384000FF90EF90DF90CF9008952F923F924F928C
:103850005F927F928F929F92AF92BF92CF92DF92B0
:10386000EF92FF920F931F93CF93DF9300D000D07E
:10387000CDB7DEB75C01FC01E059F54F74908230A2
:10388000910519F481E080938D144501880C991CF1
:10389000880C991CC4018158954F0E94D7121B01B6
:1038A0002C01672D772767FD7095872F972F0E9432
:1038B00090D16B017C0120E030E040EC5FE3C2017D
:1038C000B1010E942CD3A70196010E942CD3AB0119
:1038D000BC0100E010E09801C50170DBC4018D5807
:1038E000954F0E94D7129B01AC01C701B6010E94FF
:1038F0002CD36B017C0120E030E0A9010E94EED0C6
:10390000882309F458C000E010E09801B701A6012F
:103910007058C50153DB86E0E6E2F3E0DE01119664
:1039200001900D928A95E1F7F501EE0FFF1F81E0FE
:1039300090E08C0F9D1FE80FF91F608171811616B2
:103940001706D4F0E7EBFAE084918F010F5F1F4F69
:10395000882321F00E94B311F801F6CFEEE2F7E0E0
:1039600084918F010F5F1F4F882321F00E94B311B4
:10397000F801F6CF6AE070E0882777FD8095982FF0
:103980000E9490D19B01AC01F401E652FC4F608192
:103990007181828193810E94F5D01B012C01A701C6
:1039A0009601C701B6010E9415D0AB01BC0192017E
:1039B0008101C50103DB92E0A916B10409F03EC004
:1039C0006091DF057091E0058091E1059091E2053D
:1039D0006B017C01E894F7F8171474F4F7FAF0948B
:1039E000F7F8F0947724739420E030E0A9010E9466
:1039F000F1D218167CF009C07724739420E030E0EF
:103A0000A9010E94EED087FD05C0712C81E0809352
:103A1000881403C081E08093891400E010E09801CD
:103A2000B701A60182E090E0C9DA772019F0109280
:103A3000891402C01092881410928D14F501E85276
:103A4000F84F81E08083F501EB52F84F80838401C9
:103A5000055D194FF8011082118212821382C5018F
:103A6000A7DEC4018557954F0E94D71294012551B6
:103A7000384F7901F401E15EF94F208131814281B3
:103A800053810E9415D0F8012081318142815381F8
:103A90000E9415D0F701608371838283938384DA57
:103AA00094012552384FF70180819181A281B38121
:103AB000F90180839183A283B38326960FB6F8948D
:103AC000DEBF0FBECDBFDF91CF911F910F91FF9051
:103AD000EF90DF90CF90BF90AF909F908F907F90AE
:103AE0005F904F903F902F900895CF92EF92FF926A
:103AF0000F931F93E0903102F09032020091330255
:103B000010913402C0901C0627EF37E043EF57E0D6
:103B10006FEE77E08BEE97E00E94F6781F910F91A1
:103B2000FF90EF90CF900895CF92EF92FF920F9376
:103B30001F93C0901C067B018C0127EE37E043EEFB
:103B400057E06FED77E08BED97E00E94F6781F91DC
:103B50000F91FF90EF90CF90089580E1EBEDF7E0AB
:103B6000ABEEB7E001900D928A95E1F708952F92A0
:103B70003F924F925F926F927F928F929F92AF92FD
:103B8000BF92CF92DF92EF92FF920F931F93CF934A
:103B9000DF9300D01F92CDB7DEB75C014B018A01E5
:103BA0003C832B834090310250903202609033026C
:103BB00070903402FA01C080D180E280F380A701C6
:103BC00096016091F3077091F4078091F507909149
:103BD000F6070E94EED087FF2FC0EB81FC8120808A
:103BE0003180F281F983EB81FC81F381FA8320E05B
:103BF00030E0A901B10189819F2F0E94EED081118F
:103C000005C0212C312C30EC20E402C039812A81FE
:103C1000C101A32FB22F8093310290933202A0935F
:103C20003302B0933402C092F307D092F407E092CB
:103C3000F507F092F60759DFEB81FC81C080D18057
:103C4000E280F38020E030E0A901B601C7010E94C4
:103C5000EED0811105C055E545E535E023E404C00B
:103C60005C2D4D2D3E2D2F2D852F942FA32FB22F60
:103C70008093310290933202A0933302B0933402C6
:103C8000F50180819181A281B3818093EB079093AC
:103C9000EC07A093ED07B093EE07F40180819181CA
:103CA000A281B3818093EF079093F007A093F1076F
:103CB000B093F2071ADFF801C080D180E280F38070
:103CC000A70196016091F3077091F4078091F507C1
:103CD0009091F6070E94F1D2181664F5EB81FC81F1
:103CE000B08001811281A38020E030E0A9016B2D1A
:103CF000702F812F9A2D0E94EED0811105C0B12C1A
:103D000000E010EC20E401C02A2D8B2D902FA12F74
:103D1000B22F8093310290933202A0933302B0937A
:103D20003402C092F307D092F407E092F507F092C4
:103D3000F607DBDE0E946D8C409231025092320217
:103D400060923302709234020F900F900F900F9098
:103D5000DF91CF911F910F91FF90EF90DF90CF9067
:103D6000BF90AF909F908F907F906F905F904F909B
:103D70003F902F9008959B01AC016FEE77E08BEEA2
:103D800097E0F5CECF92DF92EF92FF920F931F93C1
:103D9000CF93DF9306EDE02E03E0F02E0BED17E05E
:103DA000CBEED7E088E3C82E86E0D82EF7018191CC
:103DB0007F01B3DC8823C9F0F7DBF60120812111F4
:103DC00004C020911B06222329F0288139814A81D1
:103DD0005B8103C020E030E0A9010E9415D0F8010A
:103DE000608371838283938309C088819981AA81CA
:103DF000BB81F80180839183A283B3830C5F1F4F43
:103E00002496FFEFCF1ADF0A8AEDE81683E0F80662
:103E100069F686E482DC8823B9F0C6DB20E030E076
:103E2000A9010E94F1D218167CF4BEDB20E030E03C
:103E300040E752E40E94F5D0609331027093320261
:103E40008093330290933402DF91CF911F910F91B1
:103E5000FF90EF90DF90CF900895CF93DF93E7EB43
:103E6000FAE08491EF012196882321F00E94B3119A
:103E7000FE01F7CF60914806709149068CE997E002
:103E80000E94D01482E20E94B3118AE0DF91CF91A8
:103E90000C94B311CF93DF938C9A80918D0A882371
:103EA000E9F0E0E5F7E06491EF01662359F0772748
:103EB00067FD70958FE29CE00E94CA132196FE0177
:103EC0006491F3CF6DE070E08FE29CE00E94CA1332
:103ED0006AE070E08FE29CE00E94CA13809189152D
:103EE0008823D9F10E94C0708091F00E9091F10E5C
:103EF000A091F20EB091F30E85369105A105B105A2
:103F00005CF00597A109B1098093F00E9093F10E32
:103F1000A093F20EB093F30E4091F00E5091F10E7B
:103F20006091F20E7091F30E40937A0A50937B0ADF
:103F300060937C0A70937D0A89EC99E00E94DF50BF
:103F400081E080932E0C8093900A1092891582EB69
:103F500090E090931E0680931D06669B0DC081E045
:103F60008093910A41E050E067E373E1809136026B
:103F7000DF91CF910C9411C6DF91CF910895EF920C
:103F8000FF920F931F93CF93DF9300D01F92CDB773
:103F9000DEB70E946D8C8091310290913202A09127
:103FA0003302B091340280933E0690933F06A09373
:103FB0004006B093410680912F0290913002909379
:103FC0003D0680933C0684E690E090933002809317
:103FD0002F020E94D113EE24E394E092390288E587
:103FE0009CDBF82E89E599DB182F8AE596DB082FF4
:103FF000F11005C0111107C0982F9E2505C011238F
:1040000011F0982F01C090E09093060280E1EBEE52
:10401000F7E0ABEDB7E001900D928A95E1F79111D1
:1040200004C0F11002C01123B1F120E030E040E8FB
:104030005FE3609127067091280680912906909190
:104040002A060E9415D02091330630913406409103
:104050003506509136060E9415D06093E3077093A1
:10406000E4078093E5079093E6072091F3073091EA
:10407000F4074091F5075091F6070E94F1D2181607
:1040800054F419821A821B821C82BE016F5F7F4F1B
:1040900083EE97E070DE80910602811102C0FF205E
:1040A00019F080E090E0D1DB80910602811102C01E
:1040B000112319F081E090E0C8DB809106028111A4
:1040C00002C0002319F082E090E0BFDB0E94D41709
:1040D00080910B0F8093390280913E0690913F06AC
:1040E000A0914006B0914106809331029093320234
:1040F000A0933302B093340280913C0690913D0628
:104100009093300280932F020E94D1130E94DD12FF
:104110000F900F900F900F90DF91CF911F910F9103
:10412000FF90EF9008958F929F92AF92BF92CF929F
:10413000DF92EF92FF920F931F93CF93DF9300D004
:104140001F92CDB7DEB785E4E8DAB82E811102C040
:104150000E946D8C96EDC92E93E0D92E2BE2E22EB3
:1041600026E0F22E0BEE17E0812C912CA12CF6010B
:1041700081916F01D2DA882351F1F80120813181D8
:104180004281538129833A834B835C830DDAF801A2
:10419000608371838283938329813A814B815C811F
:1041A000F3E08F16A1F00E9414D09B01AC01F7013F
:1041B00060817181828193810E9415D0F7016083B3
:1041C000718382839383C401F3DAAA24A394FFEF5B
:1041D0008F1A9F0A84E0E80EF11C0C5F1F4FE4E089
:1041E0008E16910421F6AA2019F00E94D41708C057
:1041F000BB2031F067EF77E083E090E00E947084AD
:104200000F900F900F900F90DF91CF911F910F9112
:10421000FF90EF90DF90CF90BF90AF909F908F90E6
:104220000C94DD120F931F93CF93DF93CDB7DEB7BE
:1042300069970FB6F894DEBF0FBECDBF82E096E05F
:104240000E94F38D6E8B7F8B888F998FBE016F5F7D
:104250007F4FCE0146960E94E31360E0CE010196A7
:104260000E94E49FE7EBFAE084918F010F5F1F4FFC
:10427000882321F00E94B311F801F6CFBE016F5FD1
:104280007F4F87EB96E00E94D0148AE00E94B31122
:1042900080913E0F8823E1F010923E0F6091D5147B
:1042A0007091D614882777FD8095982F0E9490D121
:1042B00020916E0230916F02409170025091710214
:1042C0000E94F1D2181624F41092D6141092D5142C
:1042D00069960FB6F894DEBF0FBECDBFDF91CF91C8
:1042E0001F910F9108951F93CF93DF938091FE0745
:1042F00081110E946D8CC0914606D091470661E203
:1043000070E0CE010E94BCD8009711F0EC0121961C
:1043100080E503DA882341F011E080914406909112
:1043200045068C179D0708F010E08091FF07882351
:1043300079F1212F41E0BE018CEF97E00E94F362FA
:1043400083E5EBD9882339F08091440690914506A6
:104350008C179D0768F08CEF97E00E94135F111196
:1043600017C082E096E0DF91CF911F910C94208ED0
:104370004CD9AB01BC0140937A0A50937B0A6093FD
:104380007C0A70937D0A89EC99E00E94DF50E3CFAC
:10439000DF91CF911F91089588E690E0D2D98111E5
:1043A00035C08091FB0783FD31C083E5B6D98823F2
:1043B00059F1FAD80E945DD17093D6146093D51448
:1043C000F3D820E030E04AEA52E40E94EED018161A
:1043D0004CF082E096E00E94C68D60E089E696E0AF
:1043E0000E9428A0E1D82091DD143091DE14409184
:1043F000DF145091E0140E94F1D218162CF460E002
:104400008EE596E00E9428A00C9459850895CF93DC
:10441000DF93E8E9F7E08491EF012196882321F00A
:104420000E94B311FE01F7CF6091DD147091DE148C
:104430008091DF149091E01441E050E00E94D61288
:10444000E5E9F7E08491EF012196882321F00E94AD
:10445000B311FE01F7CF6091D5147091D61488275F
:1044600077FD8095982F0E9490D141E050E00E9406
:10447000D612E1E9F7E08491EF012196882321F03B
:104480000E94B311FE01F7CF6091D9147091DA1434
:104490008091DB149091DC1441E050E00E94D61230
:1044A000EEE8F7E08491EF012196882321F00E9445
:1044B000B311FE01F7CF6091D1147091D214882707
:1044C00077FD8095982F0E9490D141E050E00E94A6
:1044D000D612EAE8F7E08491EF012196882321F0D3
:1044E0000E94B311FE01F7CF8091E30590E00E9496
:1044F000EE8E6AE070E00E945312E5E8F7E08491E6
:10450000EF012196882321F00E94B311FE01F7CF1D
:104510008FEF9FEF0E94EE8E6AE070E0DF91CF9107
:104520000C945312DF92EF92FF920F931F93CF934D
:10453000DF9383E5F2D8882311F08CD801C080E0A6
:104540008093FB07E7EBFAE08491EF012196882343
:1045500021F00E94B311FE01F7CFE7E5F6E0849168
:10456000EF012196882321F00E94B311FE01F7CFBD
:104570008091FB07882381F10DE416E0C0E0D0E0D4
:1045800020E08091FB0790E00C2E02C09595879566
:104590000A94E2F780FF17C0DD24D394D20E2223C1
:1045A00019F08CE20E94B311F80125913491F901C0
:1045B00084917901FFEFEF1AFF0A882329F00E9406
:1045C000B3119701F4CFD22E21960E5F1F4FC53045
:1045D000D10569F02D2DD5CFE9E4F6E08491EF0106
:1045E0002196882321F00E94B311FE01F7CF8AE0C3
:1045F000DF91CF911F910F91FF90EF90DF900C947E
:10460000B311CF93DF9383E588D88823D9F008D8F6
:10461000C82F8230C0F0EDEBFAE08491EF012196D3
:10462000882321F00E94B311FE01F7CFE3EBF4E001
:104630008491EF012196882309F452C00E94B3119E
:10464000FE01F6CFC0E088E468D88823B9F00E9464
:10465000101BAC2FB0E08A3A910544F09C012F303A
:1046600081E038072CF02EE031E002C02AEA30E089
:10467000AA0FBB1FAB57BA4E2D933C9386E44DD87F
:104680008823A9F00E94101B8F3F910519F014F0A8
:104690008FEF90E0EC2FF0E0EE0FFF1FE358FA4EA3
:1046A0009C0197FF02C020E030E03183208382E448
:1046B00034D88823A9F00E94101BEC2FF0E085303D
:1046C000910534F0883891052CF087E890E002C01D
:1046D00085E090E0EE0FFF1FEF57FA4E9183808345
:1046E000DF91CF91089583E518D8882351F00CD835
:1046F00060930702709308028093090290930A0264
:10470000089588E50AD881110FC089E506D881117E
:104710000BC08AE502D8811107C085E40E948D1B79
:10472000811102C00C94028D0E946D8C88E50E945C
:104730008D1B882319F05F9A1092D50789E50E9496
:104740008D1B882321F08A9A479A1092D6078AE512
:104750000E948D1B882359F09FB7F894809108011F
:104760008160809308019FBF479A1092D70785E424
:104770000E948D1B882311F0129A089508957F924C
:104780008F929F92AF92BF92CF92DF92EF92FF9261
:104790000F931F93CF93DF9306ED13E0C7E9DFE09C
:1047A000712CF80181918F010E948D1B882309F4DF
:1047B0006CC0F3E07F1263C00E94D41A6B017C01CD
:1047C00020E030E040EA51E40E94EED087FF4EC086
:1047D000A70196016091A30F7091A40F8091A50F7E
:1047E0009091A60F0E94F5D04B015C019B01AC019A
:1047F00060914F0F7091500F8091510F9091520F17
:104800000E942CD360934F0F7093500F8093510FE1
:104810009093520FA50194016091B30F7091B40F62
:104820008091B50F9091B60F0E942CD36093B30F77
:104830007093B40F8093B50F9093B60F6091830F70
:104840007091840F8091850F9091860F0E948ED178
:10485000A50194010E942CD30E9462D16093830F22
:104860007093840F8093850F9093860FC092A30F4F
:10487000D092A40FE092A50FF092A60F06C00E945E
:10488000D41A688379838A839B837394249684E003
:10489000781287CFDF91CF911F910F91FF90EF900A
:1048A000DF90CF90BF90AF909F908F907F900C94AF
:1048B000358583E50E948D1B8823D9F00E94D41A88
:1048C000AB01BC0140935B0F50935C0F60935D0F95
:1048D00070935E0F4093530F5093540F6093550F96
:1048E0007093560F8BE894E00E9429158AE00E948D
:1048F000B31180E50E948D1B882399F00E94D41A81
:10490000AB01BC0140935B0F50935C0F60935D0F54
:1049100070935E0F8EE694E00E9429158AE00E9453
:10492000B31182E50E948D1B882399F00E94D41A4E
:10493000AB01BC014093570F5093580F6093590F30
:1049400070935A0F8FE494E00E9429158AE00E9428
:10495000B31184E50E948D1B882399F00E94D41A1C
:10496000AB01BC014093530F5093540F6093550F0C
:104970007093560F81E394E00E9429158AE00C940D
:10498000B311089583E50E948D1B882351F00E9486
:10499000D41A60935F0F7093600F8093610F9093B0
:1049A000620F84E50E948D1B882351F00E94D41A67
:1049B00060933F0F7093400F8093410F9093420F8D
:1049C00082E40E948D1B882351F00E94FA1A6093A2
:1049D000630F7093640F8093650F9093660F88E563
:1049E0000E948D1B882351F00E94D41A6093430FBC
:1049F0007093440F8093450F9093460F89E50E9472
:104A00008D1B882351F00E94D41A6093470F709336
:104A1000480F8093490F90934A0F8AE50E948D1B9F
:104A2000882351F00E94D41A60934B0F70934C0F5F
:104A300080934D0F90934E0F85E40E948D1B882329
:104A400051F00E94D41A60934F0F7093500F8093CF
:104A5000510F9093520F08958F929F92AF92BF92F1
:104A6000CF92DF92EF92FF920F931F93CF93DF933A
:104A700066EDC62E63E0D62E7BEEE72E77E0F72EAE
:104A80000FE116E0C0E0D0E0F60181916F010E94D5
:104A90008D1B882309F10E94D41A4B015C01F80197
:104AA00020813181428153810E9414D09B01AC014D
:104AB000F70160817181828193810E9415D0F70195
:104AC0006083718382839383F80180829182A282C2
:104AD000B382CE010E94D81B2196F4E0EF0EF11CA8
:104AE0000C5F1F4FC330D10579F60E94D417DF91B8
:104AF000CF911F910F91FF90EF90DF90CF90BF90DB
:104B0000AF909F908F900C94DD12CF93DF93E7EBE3
:104B1000FAE08491EF012196882321F00E94B311DD
:104B2000FE01F7CF83E50E948D1B882321F00E94B0
:104B3000591B80932402EFEFF3E08491EF0121965B
:104B4000882321F00E94B311FE01F7CF8091240247
:104B5000882319F0EBEFF3E002C0E7EFF3E0849174
:104B6000EF012196882321F00E94B311FE01F7CFB7
:104B7000EFEEF3E08491EF012196882321F00E946B
:104B8000B311FE01F7CF40911802509119026091C4
:104B90001A0270911B028DEE93E00E94291540913C
:104BA0001C0250911D0260911E0270911F028AEE3C
:104BB00093E00E94291540912002509121026091BA
:104BC00022027091230287EE93E00E942915EFEDF7
:104BD000F3E08491EF012196882321F00E94B31124
:104BE000FE01F7CF40910C0250910D0260910E0230
:104BF00070910F028DED93E00E94291540911002F3
:104C00005091110260911202709113028AED93E0AB
:104C10000E942915409114025091150260911602CC
:104C20007091170287ED93E00E9429158AE0DF91C9
:104C3000CF910C94B311CF92DF92EF92FF92CF936A
:104C4000DF9383E50E948D1B882321F00E94101BB7
:104C5000EC0102C0CEE6D0E080E50E948D1B8823E7
:104C600019F00E94101B02C088EE93E06C01EE2444
:104C7000D7FCE094FE2C1C161D06A4F420E030E0C6
:104C8000A901BE018FE10E9472CCC701B6010E944A
:104C900053C88FE1DF91CF91FF90EF90DF90CF90DD
:104CA0000C9493CFC701B601DF91CF91FF90EF90A5
:104CB000DF90CF900C9453C8CF93DF9385E40E948C
:104CC0008D1B811110C080E50E948D1B882399F0F7
:104CD0000E94D41A60939002709391028093920282
:104CE0009093930208C00E94101B181619065CF7D7
:104CF000EDEBFAE06FC089E40E948D1B882381F000
:104D00000E94D41A2CE933E549E45EE30E942CD3D7
:104D100060938C0270938D0280938E0290938F0229
:104D200084E40E948D1B882381F00E94D41A2CE910
:104D300033E549E45EE30E94F5D060938802709306
:104D4000890280938A0290938B020E94ED8EE7EB9A
:104D5000FAE08491EF012196882321F00E94B3119B
:104D6000FE01F7CF40919002509191026091920222
:104D70007091930283ED93E00E9429152CE933E5AD
:104D800049E45EE360918C0270918D0280918E0205
:104D900090918F020E94F5D0AB01BC018FEC93E0A3
:104DA0000E9445152CE933E549E45EE360918802F1
:104DB0007091890280918A0290918B020E942CD37B
:104DC000AB01BC018BEC93E00E94451510C00E9422
:104DD000B311FE018491EF0121968111F8CFCCE54A
:104DE000D3E08991882319F00E94B311FACF8AE0A9
:104DF000DF91CF910C94B311CF93DF9383E50E94A1
:104E00008D1BC82F8823A1F00E94D41A60938402BE
:104E1000709385028093860290938702D1E020E010
:104E200030E0A9010E94EED08111D0E0D093CE14E1
:104E300080E50E948D1B8823B1F020E030E0A901BD
:104E40006091840270918502809186029091870220
:104E50000E94EED0882319F00E94591B01C081E006
:104E60008093CE1439C0C11137C0E7EBFAE08491CA
:104E7000EF012196882321F00E94B311FE01F7CFA4
:104E80008091CE14882319F066E474E002C06DE6C8
:104E900073E088EB93E00E94D01420E030E040E023
:104EA0005FE3609184027091850280918602909107
:104EB00087020E9415D00E945DD187EA93E00E948C
:104EC000F614E3EAF3E08491EF012196882321F0C0
:104ED0000E94B311FE01F7CFDF91CF910895EF92B9
:104EE000FF920F93CF93DF9385E40E948D1B88235D
:104EF00021F00E94101BEC0102C0C0E0D0E083E46E
:104F00000E948D1B882321F00E94101B7C0103C08E
:104F1000E5E0EE2EF12C85E50E948D1B882321F023
:104F20000E94591B082F01C000E083E50E948D1BE1
:104F3000882319F00E94D41A06C0D7FD09C060E08A
:104F400070E086E193E4209739F41092E30504C001
:104F500060E070E08CE892E49701AE010E948B92D1
:104F6000DF91CF910F91FF90EF9008952F923F9294
:104F70004F925F926F927F928F929F92AF92BF9269
:104F8000CF92DF92EF92FF920F931F93CF93DF9315
:104F9000CDB7DEB72A970FB6F894DEBF0FBECDBFF0
:104FA00088ED97E098878F83FBEE2F2EF7E03F2E5A
:104FB000EFE1F6E0FE83ED8300E010E08F8198855D
:104FC000885D97409A878987EF81F8858191F88776
:104FD000EF83882309F4A3C0F801E45FFD4F20812B
:104FE000318142815381F801E85EFD4F608171811A
:104FF000828193810E9415D020E030E040E05FE3A1
:105000000E942CD39B01AC01F101608171818281EE
:1050100093810E94F1D2181634F4C8018557954F38
:105020000E94D71203C060E070E0CB01F101408024
:10503000518062807380ED81FE81C080D180E280EA
:10504000F380A70196010E9415D0F801E55DF94FA4
:1050500020813181428153810E9415D09B01AC0196
:10506000C301B2010E9414D04B015C0120E030E08A
:1050700040EA51EC0E94F1D2181664F520E030E0CD
:1050800040EA51E4C501B4010E94EED087FF22C07E
:10509000A5019401C701B6010E9414D04B015C0127
:1050A000A70196010E9414D09B01AC01C301B2017B
:1050B0000E9415D0F1016083718382839383ED8117
:1050C000FE8180829182A282B38289859A850E9424
:1050D000D81B25C0EDEBFAE084918F010F5F1F4FC5
:1050E000882321F00E94B311F801F6CFE5E8F3E040
:1050F00084918F010F5F1F4F882321F00E94B3110D
:10510000F801F6CF87E793E00E949EA088E290E046
:105110009A83898388EC90E09C838B832FC0F4E092
:105120002F0E311C0C5F1F4F8D819E8104969E8334
:105130008D830C30110509F041CF0E94D4170E94D5
:10514000DD1260E087E693E00E9428A083E992E008
:105150009A83898308EC10E01C830B83AE014F5FB8
:105160005F4FBE016D5F7F4F84EE95E00E94971404
:105170008AEB92E09A8389831C830B83AE014F5F95
:105180005F4FBE016D5F7F4F84EE95E00E949714E4
:105190002A960FB6F894DEBF0FBECDBFDF91CF9138
:1051A0001F910F91FF90EF90DF90CF90BF90AF9045
:1051B0009F908F907F906F905F904F903F902F9037
:1051C0000895CF93DF9380931C06E7EBFAE0849178
:1051D000EF012196882321F00E94B311FE01F7CF41
:1051E00060911C0670E083E797E00E94F6148AE065
:1051F000DF91CF910C94B311CF93DF930E94D11321
:10520000E0914C06F0E0E153FA4F8081882381F071
:10521000EBE5F3E08491EF012196882321F00E94D1
:10522000B311FE01F7CF8AE0DF91CF910C94B31157
:10523000DF91CF910895CF93DF930E94AB11EEE5FC
:10524000F3E08491EF012196882321F00E94B311AD
:10525000FE01F7CF6091CD077091CE078091CF0707
:105260009091D0076F5F7F4F8F4F9F4F4AE050E084
:105270000E9449128AE00E94B311DF91CF91BCCF06
:10528000EF92FF920F931F93CF93DF931F92CDB7AF
:10529000DEB7082F162FEDEBFAE084917F012FEF98
:1052A000E21AF20A882331F099830E94B311F701C0
:1052B0009981F3CFE02FF92F84917F019FEFE91AB5
:1052C000F90A882321F00E94B311F701F5CF60910C
:1052D000CD077091CE078091CF079091D0074AE01B
:1052E00050E00E9449128AE00E94B3111111A3DF1D
:1052F00010921906109218060F90DF91CF911F910E
:105300000F91FF90EF900895CF92DF92EF92FF926E
:10531000CF93DF93EC01C0901802D0901902E09077
:105320001A02F0901B02A7019601688179818A8197
:105330009B810E94EED087FF04C0C882D982EA8296
:10534000FB82C0901C02D0901D02E0901E02F090E3
:105350001F02A70196016C817D818E819F810E9431
:10536000EED087FF04C0CC82DD82EE82FF82C09047
:105370002002D0902102E0902202F0902302A701A7
:105380009601688579858A859B850E94EED087FF86
:1053900004C0C886D986EA86FB86C0900C02D090ED
:1053A0000D02E0900E02F0900F02A70196016881B5
:1053B00079818A819B810E94F1D2181624F4C882D7
:1053C000D982EA82FB82C0901002D0901102E09054
:1053D0001202F0901302A70196016C817D818E81EB
:1053E0009F810E94F1D2181624F4CC82DD82EE82D5
:1053F000FF82C0901402D0901502E0901602F09047
:105400001702A7019601688579858A859B850E9488
:10541000F1D2181624F4C886D986EA86FB86DF9175
:10542000CF91FF90EF90DF90CF90089580E090E0D3
:105430000E94EC8C6093D3057093D4058093D505BE
:105440009093D60581E090E00E94EC8C6093D705A4
:105450007093D8058093D9059093DA0582E090E0A7
:105460000E94EC8C6093DB057093DC058093DD0576
:105470009093DE050895CF93DF93EC01D7DFC43618
:10548000D10551F48CE0E3EDF5E0ABEEB7E001902F
:105490000D928A95E1F711C0CC0FDD1FCC0FDD1FF7
:1054A000FE01E551F84FCD52DA4F88819981AA81EA
:1054B000BB8180839183A283B383DF91CF910895D1
:1054C0000E94058D0E946D8C84E690E0D4DF0C94E0
:1054D000D417CF92DF92EF92FF928BED97E014DF1B
:1054E0000E94D1138091FB0783FD97C0C090E7070E
:1054F000D090E807E090E907F090EA072091F707DD
:105500003091F8074091F9075091FA07C701B601A9
:105510000E94EED0882309F480C08091CE148111BE
:1055200036C02091840230918502409186025091CC
:1055300087026091DD147091DE148091DF149091E8
:10554000E0140E94EED087FF22C0C092F707D092ED
:10555000F807E092F907F092FA07E7EBFAE0849196
:105560007F019FEFE91AF90A882321F00E94B31105
:10557000F701F5CFE0E4F3E084917F019FEFE91AB2
:10558000F90A882321F00E94B311F701F5CFC090EA
:10559000E707D090E807E090E907F090EA0720914C
:1055A000F7073091F8074091F9075091FA07C701C2
:1055B000B6010E9414D00E945DD197FF07C090955C
:1055C0008095709561957F4F8F4F9F4F693C710516
:1055D0008105910514F1C092F707D092F807E09287
:1055E000F907F092FA07E7EBFAE084917F019FEF69
:1055F000E91AF90A882321F00E94B311F701F5CFC7
:10560000E1E2F3E084917F019FEFE91AF90A882330
:1056100021F00E94B311F701F5CF2091DB07309103
:10562000DC074091DD075091DE076091EB07709138
:10563000EC078091ED079091EE070E94EED081116A
:105640001DC02091DF073091E0074091E1075091A4
:10565000E2076091EF077091F0078091F107909158
:10566000F2070E94EED0811109C060913102709161
:10567000320280913302909134021AC060912F025D
:1056800070913002882777FD8095982F0E9490D1E5
:105690002091310230913202409133025091340214
:1056A0000E942CD32AE037ED43E25CE30E942CD326
:1056B0000E94941DFF90EF90DF90CF900C94AD1D51
:1056C000CF92DF92EF92FF920F931F930E9424C814
:1056D000009148051091490520914A0530914B05EC
:1056E0006B017C01C01AD10AE20AF30AF7FC55C02B
:1056F0008B019C010C53164F2F4F3F4F00934805D1
:105700001093490520934A0530934B054F9B3CC0AD
:105710007A9B3AC02091060120FF36C02091D01418
:10572000211132C0029B30C0009144051091450503
:1057300020914605309147050115110521053105D8
:1057400099F0DC01CB01801B910BA20BB30B8056AF
:105750009A4EA109B1098827B7FD83959927AA27F1
:10576000BB27182F119501C010E0612F87E00E9420
:1057700048CA612F70E087E01F910F91FF90EF9072
:10578000DF90CF900C94F7C8609344057093450563
:105790008093460590934705C7CF1F910F91FF90C7
:1057A000EF90DF90CF900895CF92DF92EF92FF922B
:1057B0006B017C0180913706882351F120E030E0B5
:1057C000A901C701B6010E94EED0882309F12BED93
:1057D0003FE049E450E4C701B6010E942CD320E029
:1057E00030E040E05FE30E942CD3A70196010E94C5
:1057F0002CD320E030E040E05FE30E942CD39B01FB
:10580000AC0160E070E080E89FE30E94F5D004C046
:1058100060E070E080E89FE3FF90EF90DF90CF9032
:1058200008956091290270912A0280912B02909133
:105830002C02BADF60932502709326028093270220
:10584000909328020895CF93DF9388EC90E00E9414
:10585000A11B811142C084E40E948D1B8823E9F1C1
:105860000E94D41AC1E020E030E0A9010E94EED0ED
:10587000811101C0C0E0C0933706CC2359F1C0911B
:10588000E305D0E00E94D41AFE01EE0FFF1FEE0FD9
:10589000FF1FE75DFD4F608371838283938320E068
:1058A00030E0A9016091290270912A0280912B02B7
:1058B00090912C020E94EED081110CC080E090E00B
:1058C000A0EEBFE38093290290932A02A0932B02BB
:1058D000B0932C02DF91CF91A4CFDF91CF910895A7
:1058E0005F988A9847989FB7F894E8E0F1E0808144
:1058F0008E7F80839FBF4798129808955F9A109279
:10590000D5078A9A479A1092D6079FB7F894E8E08D
:10591000F1E08081816080839FBF479A1092D70712
:10592000129A0895EC01EDEBFAE084918F010F5F7C
:105930001F4F882321F00E94B311F801F6CFEFEE3C
:10594000F2E084918F010F5F1F4F882321F00E94A6
:10595000B311F801F6CFCE010E9465A164EF71E0AA
:1059600080E090E00E9453C8F8940E946A92C6DFDB
:10597000FFCF8F929F92AF92BF92DF92EF92FF92F2
:105980000F931F93CF93DF9380914A06843008F0E2
:105990002DC10E94A111882309F428C10E948A11F7
:1059A00020911806309119068A3019F08D3009F0CF
:1059B000F2C01092AE052115310531F3F901E25B19
:1059C000FA4F108210921906109218068EE495E094
:1059D0007C01FC01208101962032D1F3E7012E34B5
:1059E00011F0E12CF12C6AE270E0CE010E94BCD8EB
:1059F0008C01E114F10409F474C065E179E0CE0191
:105A00000E946ED8DD24D394892B11F4D12C09C0C7
:105A10006EE470E0CE0104960E94BCD8009709F0B5
:105A20007C014AE050E060E070E0C70101960E940E
:105A3000F5D56093D1077093D2078093D3079093E5
:105A4000D4078090CD079090CE07A090CF07B0905C
:105A5000D007FFEF8F1A9F0AAF0ABF0A68157905B2
:105A60008A059B0531F0D11004C061E082EE98E018
:105A70003DC00115110501F180E0F12CFE01E80F98
:105A8000F11D90819A3219F08F5FF926F7CF4AE025
:105A900050E060E070E0C80101960E94F5D50F2D3E
:105AA00010E020E030E0601771078207930741F0B3
:105AB00061E083EC98E01AC061E089E998E016C0E3
:105AC0008091D1079091D207A091D307B091D407CC
:105AD0008093CD079093CE07A093CF07B093D007C4
:105AE00011C0009779F060E08FE698E0DF91CF91E8
:105AF0001F910F91FF90EF90DF90BF90AF909F901C
:105B00008F90BECB80913502811122C067E470E096
:105B1000CE010E94BCD80097D9F04AE050E060E086
:105B200070E001960E94F5D56430710588F4E8EFC5
:105B3000F7E084918F010F5F1F4F882321F00E94AF
:105B4000B311F801F6CF60E08EEE97E00E9428A036
:105B500061E773E0CE010E94C7D8892B21F410922F
:105B60000B0210921A0666E773E0CE010E94C7D8B6
:105B7000892B19F485EE97E0D5DE6BE773E0CE0153
:105B80000E94C7D8892B09F49BDC61E08EE495E084
:105B90000E945D18F9CE2F3531050CF0F5CE8C350D
:105BA00081F40E94A111882309F4EECE0E948A118B
:105BB0009091AE059111E8CE20911806309119060A
:105BC00009C08B3319F491E09093AE059091AE0526
:105BD0009111DACEA9014F5F5F4F509319064093A0
:105BE0001806F901E25BFA4F8083CECEDF91CF91A8
:105BF0001F910F91FF90EF90DF90BF90AF909F901B
:105C00008F9008950E949C18811103C0B2DE0C94FD
:105C100023190895CF92DF92EF92FF920F931F9373
:105C2000CF93C82F0E9496150E94B21780914A0602
:105C3000843008F4E7DF0E9424C8C0901006D0909A
:105C40001106E0901206F0901306C114D104E1048D
:105C5000F104B9F000911406109115062091160672
:105C6000309117060C0D1D1D2E1D3F1D6B017C0173
:105C7000C01AD10AE20AF30AF7FC03C088E193E0F4
:105C80004AC0C0900702D0900802E0900902F0904C
:105C90000A02C114D104E104F10421F100911406B7
:105CA0001091150620911606309117060C0D1D1D3A
:105CB0002E1D3F1D6B017C01C01AD10AE20AF30AB6
:105CC000F7FC10C0C1110EC09091B80F8091B70FB2
:105CD000981308C08091EA0E811104C080912D0CA8
:105CE000882361F18091420590914305909902C00B
:105CF000019604C0181619062CF4019790934305D9
:105D00008093420580914205909143058E3E9240DA
:105D10001CF08FE093E006DED3DC8091EA0E811167
:105D200021C080912D0C81111DC0CF911F910F9129
:105D3000FF90EF90DF90CF900C94D8785F9A1092FC
:105D4000D5078A9A479A1092D6079FB7F894809100
:105D500008018160809308019FBF479A1092D7077E
:105D6000129AC0CFCF911F910F91FF90EF90DF90CB
:105D7000CF9008951F93CF93DF930E94201960E97D
:105D800070ED83E090E00E945411E8EEF2E084911F
:105D9000EF012196882321F00E94B311FE01F7CF75
:105DA000E7EBFAE08491EF012196882321F00E942D
:105DB000B311FE01F7CF40E052EC61E070E08FE2FA
:105DC0009CE00E94864A6DE070E08FE29CE00E94B9
:105DD000CA136AE070E08FE29CE00E94CA13E4EE0E
:105DE000F2E06491EF01662359F0772767FD709523
:105DF0008FE29CE00E94CA132196FE016491F3CFCA
:105E00006DE070E08FE29CE00E94CA136AE070E0EF
:105E10008FE29CE00E94CA136AE070E080E090E0AC
:105E20000E9453C8E0EEF2E06491EF01662359F05E
:105E3000772767FD70958FE29CE00E94CA13219638
:105E4000FE016491F3CF6DE070E08FE29CE00E9470
:105E5000CA136AE070E08FE29CE00E94CA130E94BD
:105E600078170E947D1514B710FF0BC0E7EDF2E024
:105E70008491EF012196882321F00E94B311FE0145
:105E8000F7CF11FF0BC0E6ECF2E08491EF01219611
:105E9000882321F00E94B311FE01F7CF12FF0BC03F
:105EA000E4EBF2E08491EF012196882321F00E9437
:105EB000B311FE01F7CF13FF0BC0E3EAF2E08491C8
:105EC000EF012196882321F00E94B311FE01F7CF44
:105ED00015FF0BC0E2E9F2E08491EF0121968823DF
:105EE00021F00E94B311FE01F7CF14BEEAE8F2E000
:105EF0008491EF012196882321F00E94B311FE01C5
:105F0000F7CF80E20E94B311EFE7F2E08491EF0156
:105F10002196882321F00E94B311FE01F7CF8AE079
:105F20000E94B311E7EBFAE08491EF0121968823F8
:105F300021F00E94B311FE01F7CFEFE6F2E0849169
:105F4000EF012196882321F00E94B311FE01F7CFC3
:105F5000EEE5F2E08491EF012196882321F00E9482
:105F6000B311FE01F7CFECE3F2E08491EF0121964B
:105F7000882321F00E94B311FE01F7CFE5E2F2E0A1
:105F80008491EF012196882321F00E94B311FE0134
:105F9000F7CFE7EBFAE08491EF012196882321F017
:105FA0000E94B311FE01F7CF0E944456BC0186E166
:105FB00092E00E94F61460E974E08FEF91E00E9495
:105FC000F6148AE00E94B31181E08093CF0580939C
:105FD000D0058093D1058093D2050E94746E8CE029
:105FE000EFE1F6E0ABEEB7E001900D928A95E1F7B4
:105FF0000E94D41781EE94E10E94CA910E94F08B16
:1060000080910101806180930101FFEF29EF80E021
:10601000F15020408040E1F700C000000E9453731F
:106020000E94F5A00E94A4170E94D0170E94871515
:10603000EFE3FCE93197F1F700C00000DF91CF9169
:106040001F91089526E034E0FC01318320832781ED
:10605000222319F004960C94C25108958F929F92B6
:10606000AF92BF92CF92DF92EF92FF920F931F9366
:10607000CF93DF938C0187539E4FE4DF68018FE657
:10608000C80ED11CC114D10421F178018BE5E81AA6
:106090008EEFF80AE70157018FE1A81AB10836E040
:1060A000832E34E0932ECC15DD0599F0FE01EE1918
:1060B000FF09EA0DFB1D91828082FE0178978081A5
:1060C000811102C06F97EFCFCE014B970E94C25152
:1060D000F9CFC801805B9F4FB5DFC8018F96DF9174
:1060E000CF911F910F91FF90EF90DF90CF90BF90D5
:1060F000AF909F908F90A6CF8CEF97E00E94075BA8
:1061000082E096E00E94B68DE4EEF5E08EEE93E03C
:106110009183808384E08093F1051092EF051092C3
:10612000EE051092F0053E9A469816821782108668
:10613000118608958CEF97E091CF8FE29CE00E944A
:10614000C1490C94A3162F923F924F925F926F9287
:106150007F928F929F92AF92BF92CF92DF92EF92F7
:10616000FF920F931F93CF93DF93CDB7DEB76E9758
:106170000FB6F894DEBF0FBECDBFBFEAAB2EBAE0BC
:10618000BB2E14ED212E19E0312E8E010F5F1F4F13
:1061900080E6482E8AEE582E612C712C8FE29CE00E
:1061A0000E9475491816190614F00C94483980910C
:1061B000A40A9091A50A049714F00C9448398FE230
:1061C0009CE00E94A14980939B0A2091990A3091FA
:1061D0009A0A8A3061F08D3051F08A3321F490911F
:1061E000980A992321F02F3531050CF49CC521150F
:1061F000310521F41092980A0C9448398091A00A34
:106200009091A10AA0E69A2E989E6001999ED00CCA
:106210001124F601E20FF31FEA55F54F1082209189
:10622000980A21117BC5FC01E456F54F1082C60186
:106230008A55954F7C016EE470E00E94BCD80097AF
:1062400009F450C09093970A8093960A8E199F097B
:106250008C0D9D1D4AE050E060E070E08955954F3F
:106260000E94F5D56093D1077093D2078093D3072E
:106270009093D4072091CD073091CE074091CF075E
:106280005091D0072F5F3F4F4F4F5F4FC090A00AF4
:10629000D090A10A621773078407950709F463C5B4
:1062A0009C9CC0019D9C900D11246BE57AE08A5561
:1062B000954F0E946ED8892B09F055C5E2EBFAE0A4
:1062C00064918F01662361F0772767FD70958FE2F7
:1062D0009CE00E94CA130F5F1F4FF8016491F2CF38
:1062E0002CDF19C06AE270E0C7010E94BCD8892B7C
:1062F00039F1E2EBFAE064918F01662361F07727D0
:1063000067FD70958FE29CE00E94CA130F5F1F4FDC
:10631000F8016491F2CF10929A0A1092990AB8C7C4
:106320008091D1079091D207A091D307B091D40763
:106330008093CD079093CE07A093CF07B093D0075B
:106340008091A00A9091A10A20E6289F7001299FC0
:10635000F00C1124C7018A55954F6C0161E470E07F
:106360000E94BCD8009709F4C3C49093970A809305
:10637000960A8C199D098E0D9F1D60E070E089556D
:10638000954F0E948DD40E945DD1CB01AA2797FD25
:10639000A095BA2F8232910508F0AAC4FC01EE58EC
:1063A000FF4F0C946AD4E6E5FAE064917F0166231E
:1063B00069F0772767FD70958FE29CE00E94CA1311
:1063C0009FEFE91AF90AF7016491F1CF20E030E07C
:1063D00040E05FE36091DD147091DE148091DF1482
:1063E0009091E01437C0E1E5FAE064917F01662303
:1063F00069F0772767FD70958FE29CE00E94CA13D1
:10640000FFEFEF1AFF0AF7016491F1CF6091D51405
:106410007091D61445C0ECE4FAE064917F016623E4
:1064200069F0772767FD70958FE29CE00E94CA13A0
:10643000FFEFEF1AFF0AF7016491F1CF20E030E09F
:1064400040E05FE36091D9147091DA148091DB141D
:106450009091DC140E9415D00E945DD17A836983EB
:10646000C8010E94F0BFBC018FE29CE00E94E3CA19
:1064700055C0E7E4FAE064917F01662369F077276D
:1064800067FD70958FE29CE00E94CA13FFEFEF1A40
:10649000FF0AF7016491F1CF6091D1147091D21489
:1064A000882777FD8095982F0E9490D120E030E0DA
:1064B00040E05FE3CFCF20911D0630911E0644E6F9
:1064C000429FC001439F900D112462EB70E00E9437
:1064D00005D47B01FFEFEF1AFF0A85E6E816F10409
:1064E00018F0E4E6EE2EF12CE2E4FAE064916F019C
:1064F000662369F0772767FD70958FE29CE00E9424
:10650000CA139FEFC91AD90AF6016491F1CF4AE084
:1065100050E0B7018FE29CE00E9493CB6DE070E009
:106520008FE29CE00E94CA136AE070E08FE29CE078
:106530000E94CA13DDC3EEE3FAE064917F01662393
:1065400069F0772767FD70958FE29CE00E94CA137F
:10655000FFEFEF1AFF0AF7016491F1CF60E270E0FC
:106560008FE29CE00E94CA13EAE3FAE064917F01A3
:10657000662369F0772767FD70958FE29CE00E94A3
:10658000CA13FFEFEF1AFF0AF7016491F1CF4091B0
:10659000EB075091EC076091ED077091EE0722E058
:1065A00030E08FE29CE00E9471CC60E270E08FE20C
:1065B0009CE00E94CA13E6E3FAE064917F0166233F
:1065C00069F0772767FD70958FE29CE00E94CA13FF
:1065D000FFEFEF1AFF0AF7016491F1CF4091EF0747
:1065E0005091F0076091F1077091F20722E030E0DE
:1065F0008FE29CE00E9471CC60E270E08FE29CE050
:106600000E94CA13E2E3FAE064917F01662369F015
:10661000772767FD70958FE29CE00E94CA13FFEF19
:10662000EF1AFF0AF7016491F1CF4091F3075091FF
:10663000F4076091F5077091F60722E030E08FE2F1
:106640009CE00E9471CC60E270E08FE29CE00E94CE
:10665000CA1364CF8091FE078823D9F0EDE2FAE0F7
:1066600064917F01662369F0772767FD70958FE25B
:106670009CE00E94CA13FFEFEF1AFF0AF701649132
:10668000F1CF81E080938E0A8CEF97E00E94345F17
:1066900045CFE5E2FAE064917F01662309F43ECF3D
:1066A000772767FD70958FE29CE00E94CA13FFEF89
:1066B000EF1AFF0AF7016491F0CFE0E2FAE064918B
:1066C0007F01662369F0772767FD70958FE29CE074
:1066D0000E94CA13FFEFEF1AFF0AF7016491F1CF8E
:1066E0008091920A9091930AA091940AB091950A90
:1066F000892B8A2B8B2B09F46CC00E9424C8A30120
:1067000092010E942CD469017A016091920A7091E1
:10671000930A8091940A9091950AA30192010E9494
:106720002CD47601E21AF30AC7016CE370E00E94F0
:1067300005D46983C8010E94D8BFBC018FE29CE0E8
:106740000E94E3CA60E270E08FE29CE00E94CA13FC
:10675000EEE1FAE064916F01662369F0772767FD47
:1067600070958FE29CE00E94CA13FFEFCF1ADF0AF8
:10677000F6016491F1CF60E270E08FE29CE00E944C
:10678000CA13C7016CE370E00E9405D48983C80175
:106790000E94D8BFBC018FE29CE00E94E3CA60E285
:1067A00070E08FE29CE00E94CA13ECE1FAE0649191
:1067B0007F01662309F4B2CE772767FD70958FE2DB
:1067C0009CE00E94CA13FFEFEF1AFF0AF7016491E1
:1067D000F0CF60E270E08FE29CE00E94CA13E4E137
:1067E000FAE064917F01662309F498CE772767FD6C
:1067F00070958FE29CE00E94CA13FFEFEF1AFF0A28
:10680000F7016491F0CF1092E90E1092E80E80919A
:10681000090180FF14C0E0E1FAE064917F01662382
:1068200009F47CCE772767FD70958FE29CE00E948B
:10683000CA13FFEFEF1AFF0AF7016491F0CF0E942D
:10684000D3161092380283E50E94B716882341F0D0
:106850000E94AE160E9462D17093280C6093270CA0
:10686000ECE0FAE064917F01662369F0772767FD29
:1068700070958FE29CE00E94CA13FFEFEF1AFF0AA7
:10688000F7016491F1CF6DE070E08FE29CE00E942F
:10689000CA136AE070E08FE29CE00E94CA138CEF9A
:1068A00097E00E94985DE8E0FAE064917F0166233A
:1068B00009F434CE772767FD70958FE29CE00E9443
:1068C000CA13FFEFEF1AFF0AF7016491F0CF80912E
:1068D000FE078823E9F081E080938F0A8093BD054D
:1068E0008093EA0E1092FE07E4E0FAE064917F01E3
:1068F000662309F413CE772767FD70958FE29CE03D
:106900000E94CA13FFEFEF1AFF0AF7016491F0CF5C
:10691000E0E0FAE064917F01662309F4FFCD772778
:1069200067FD70958FE29CE00E94CA13FFEFEF1A9B
:10693000FF0AF7016491F0CF8091EA0E882309F4F1
:10694000D7C18CEF97E00E94135FECEFF9E0649100
:106950007F01662309F4E2CD772767FD70958FE20A
:106960009CE00E94CA13FFEFEF1AFF0AF70164913F
:10697000F0CF8091FE07811105C08091EA0E882337
:1069800009F4B6C1109289158CEF97E00E946862F5
:1069900088EF99E016C10E94DC138111A9C1809192
:1069A000EA0E882309F44FC2A3C10E94DC138111AF
:1069B0009FC18091EA0E882309F461C299C10E94A7
:1069C000DC138111ABCD8091EA0E882309F479C2E2
:1069D000A5CD83E50E94B71681116EC183E40E94A4
:1069E000B716882309F484C10E94DC13882309F4B4
:1069F00063C17EC183E50E94B716882309F478C17C
:106A00000E94AE1620E030E0A9010E94EED087FD82
:106A10000FC00E94AE1620E030E046E153E40E9431
:106A2000F1D2181644F00E94AE160E9462D105C041
:106A300060E070E002C066E970E07093D214609389
:106A4000D11456C183E50E94B7168823D1F00E9465
:106A5000AE1620E030E042E353E40E942CD320E065
:106A600030E048EC52E40E94F5D00E9462D1633BD2
:106A7000710510F062EB70E070931E0660931D06C6
:106A80004DCD82EB90E090931E0680931D0646CD7F
:106A90008091260C811142CD8091FE0781113ECD5F
:106AA0000E94602A5F9A1092D5078A9A479A10929C
:106AB000D6079FB7F8948091080181608093080100
:106AC0009FBF479A1092D707129A28CD83E50E945C
:106AD000B716882319F10E94AE1620E030E040E29C
:106AE00052E40E94EED087FD0FC00E94AE1620E057
:106AF00030EC49E754E40E94F1D2181644F00E94A9
:106B0000AE160E945DD105C068E270E002C067EE7B
:106B100073E07093300260932F02EAC0EEEEF9E06A
:106B200064917F01662369F0772767FD70958FE296
:106B30009CE00E94CA13FFEFEF1AFF0AF70164916D
:106B4000F1CF60912F02709130024AE050E08FE265
:106B50009CE00E9480CBE2CC0E94DC138111C8C073
:106B60008091EA0E8111C4C088E50E94B716811198
:106B700006C089E50E94B716882309F4D6C188E5C6
:106B80000E94B716882341F088EE99E0909343065F
:106B9000809342060E949C1889E50E94B7168823BC
:106BA00041F082EE99E090934306809342060E9462
:106BB0009C188AE50E94B716882309F499C08CEDC9
:106BC00099E090934306809342060E949C1890C0DF
:106BD0000E94DC138111A2CC8091EA0E882309F473
:106BE000B2C19CCC0E94DC13811182C08091EA0E5C
:106BF000882309F4EDC27CC00E94DC13811178C0A7
:106C00008091EA0E882309F405C372C00E94DC1348
:106C100081116EC08091EA0E882309F41DC368C0FB
:106C20008CEF97E00E94075E8091090180FF60C0B1
:106C3000E3E4F9E064917F01662309F46FCC7727E0
:106C400067FD70958FE29CE00E94CA13FFEFEF1A78
:106C5000FF0AF7016491F0CF8FE40E94B71681110B
:106C60005DCC83E40E94B71659CCEEE3F9E0649161
:106C70007F01662369F0772767FD70958FE29CE0BE
:106C80000E94CA13FFEFEF1AFF0AF7016491F1CFD8
:106C9000E7E3F9E064917F01662309F43FCC7727AD
:106CA00067FD70958FE29CE00E94CA13FFEFEF1A18
:106CB000FF0AF7016491F0CF0E94AE1620E030E0A9
:106CC000A9010E94EED087FD2DC10E94AE1620E0E2
:106CD00030E849E853E40E94F1D218160CF41FC1C1
:106CE0000E94AE160E9462D17093D6146093D514A0
:106CF0008091A00A9091A10A019664E070E00E9440
:106D000019D49093A10A8093A00A8091A40A90912B
:106D1000A50A01969093A50A8093A40A10929A0A54
:106D20001092990A3BCA8B3319F491E09093980A18
:106D30009091980A911132CA4091A00A5091A10AEB
:106D4000B9016F5F7F4F70939A0A6093990A90E63A
:106D5000949FF001959FF00D1124E20FF31FEA5567
:106D6000F54F80831BCA80E68C9D70018D9DF00CD1
:106D70001124C7018A55954F6C016AE270E00E94A8
:106D8000BCD8009799F4E2EBFAE064918F01662396
:106D900009F4A6CA772767FD70958FE29CE00E94F0
:106DA000CA130F5F1F4FF8016491F1CF20E0912CBF
:106DB000F701E20FF11DEA55F54F30813A3219F033
:106DC0002F5F9326F5CF9093970A8093960A8C199C
:106DD0009D098E0D9F1D60E070E08955954F0E94C2
:106DE0008DD40E945DD1292D30E02617370709F494
:106DF00097CAF2EBEF2EFAE0FF2EF70164918701BC
:106E0000662361F0772767FD70958FE29CE00E9412
:106E1000CA130F5F1F4FF8016491F2CF8ED9F701AB
:106E2000E49002EB1AE0EE2009F45ACA6E2D77279F
:106E300067FD70958FE29CE00E94CA130F5F1F4FA1
:106E4000F801E490F0CFE090960AF090970A94E071
:106E5000E90EF11C6AE270E0C7010E94BCD80097FD
:106E600019F0FC013197108220E041E0B7018CEF6E
:106E700097E00E94F36281E080938D0A4FCB8CEF04
:106E800097E00E94135F0E9424C86093920A709357
:106E9000930A8093940A9093950AE4EFF9E0649141
:106EA0007F01662309F43ACB772767FD70958FE25F
:106EB0009CE00E94CA13FFEFEF1AFF0AF7016491EA
:106EC000F0CF8091FF07882319F081E08093891526
:106ED00081E08093900A8CEF97E00E94135F0E94FC
:106EE00024C86093920A7093930A8093940A9093B3
:106EF000950AF50164917FEAE72E7AE0F72E662382
:106F000009F40CCB772767FD70958FE29CE00E9417
:106F1000CA13FFEFEF1AFF0AF7016491F0CF63E1A4
:106F200071E0E2CE60E070E0DFCE8AE50E94B71645
:106F3000811125CE83E40E94B716882309F4D8CEA8
:106F400088ED99E03ECE86E40E94B716882309F4C6
:106F50003CC10E94AE160E9462D14B0130924306A2
:106F6000209242060E949C1888E50E94B71688234A
:106F700009F43EC00E94AE166B017C012DEC3CEC86
:106F80004CE45EE30E94EED0181674F020E030E08E
:106F9000A901C701B6010E94F1D218162CF49F92E4
:106FA0008F9289EC99E0FAC02DEC3CEC4CEC5DEB57
:106FB000C701B6010E94EED018167CF020E030E048
:106FC00040E85FEBC701B6010E94F1D218162CF41D
:106FD0009F928F928DEB99E0E1C09F928F92C701B3
:106FE000B6010E945DD17F936F9383EB99E087C0D8
:106FF00089E50E94B716882309F43EC00E94AE16A8
:107000006B017C012DEC3CEC4CE45EE30E94EED085
:10701000181674F020E030E0A901C701B6010E9403
:10702000F1D218162CF49F928F9288EA99E0B6C09C
:107030002DEC3CEC4CEC5DEBC701B6010E94EED0B0
:1070400018167CF020E030E040E85FEBC701B601A5
:107050000E94F1D218162CF49F928F928CE999E03D
:107060009DC09F928F92C701B6010E945DD17F9310
:107070006F9382E999E043C08AE50E94B71688239E
:1070800009F44BC00E94AE166B017C012DEC3CEC68
:107090004CE45EE30E94EED0181674F020E030E07D
:1070A000A901C701B6010E94F1D218162CF49F92D3
:1070B0008F9287E899E072C02DEC3CEC4CEC5DEBD4
:1070C000C701B6010E94EED018167CF020E030E037
:1070D00040E85FEBC701B6010E94F1D218162CF40C
:1070E0009F928F928BE799E059C09F928F92C70130
:1070F000B6010E945DD17F936F9381E799E09F93E2
:107100008F931F930F930E940ED9C80169D10FB6B8
:10711000F894DEBF0FBECDBF4FC085E40E94B71606
:10712000882309F449C00E94AE166B017C012DEC46
:107130003CEC4CE45EE30E94EED0181674F020E0C4
:1071400030E0A901C701B6010E94F1D218162CF453
:107150009F928F9286E699E021C02DEC3CEC4CEC9E
:107160005DEBC701B6010E94EED018167CF020E05E
:1071700030E040E85FEBC701B6010E94F1D218167B
:107180002CF49F928F928AE599E008C0C701B6015E
:107190000E945DD17F936F938FE499E09F938F93CB
:1071A0001F930F930E940ED9C8011AD10F900F9010
:1071B0000F900F900F900F908BE499E090934306FF
:1071C000809342060E949C18A9C9812C912CC6CE9E
:1071D000E2E3F0E0F093D214E093D1148EEB90E070
:1071E0009093D6148093D514F50164915FEAE52E4F
:1071F0005AE0F52E662309F491C9772767FD70954B
:107200008FE29CE00E94CA139FEFE91AF90AF70186
:107210006491F0CF80E590E09093D2148093D114E4
:10722000E0EFF0E0F093D614E093D514F50164910B
:107230004FEAE42E4AE0F42E662309F46FC977275B
:1072400067FD70958FE29CE00E94CA13FFEFEF1A72
:10725000FF0AF7016491F0CF1092D6141092D51462
:107260001092D2141092D114E7E4F9E064917F01F6
:10727000662309F453C9772767FD70958FE29CE078
:107280000E94CA13FFEFEF1AFF0AF7016491F0CFD3
:107290006E960FB6F894DEBF0FBECDBFDF91CF91D3
:1072A0001F910F91FF90EF90DF90CF90BF90AF9024
:1072B0009F908F907F906F905F904F903F902F9016
:1072C0000895CF92DF92EF92FF92CF93DF93809158
:1072D000A40A9091A50A039714F40E94A330809108
:1072E000A40A9091A50A009791F001979093A50A9E
:1072F0008093A40A8091A20A9091A30A019664E067
:1073000070E00E9419D49093A30A8093A20AC090BF
:10731000DD14D090DE14E090DF14F090E01420E053
:1073200030E040EA50E4C701B6010E94EED087FD8C
:1073300038C020E030E84EE853E4C701B6010E94AF
:10734000F1D2181674F18091B0059091B10589348D
:107350009E4E88F11092B1051092B005E3E3F9E07A
:107360006491EF01662359F0772767FD70958FE2EE
:107370009CE00E94CA132196FE016491F3CF6DE058
:1073800070E08FE29CE00E94CA136AE070E08FE236
:107390009CE0DF91CF91FF90EF90DF90CF900C9425
:1073A000CA138091B0059091B10501969093B105F3
:1073B0008093B005C8CFDF91CF91FF90EF90DF9021
:1073C000CF9008957EDF0E943FA00E94121780E0B8
:1073D0000E940A2E0E94109184EE95E00C94751381
:1073E000CF93DF93EC0160E0CE010E947918811108
:1073F00002C0E8DFF8CFDF91CF9108958F929F927E
:10740000AF92BF92CF92DF92EF92FF9280E50E94FF
:107410008D1B882329F00E94FA1A4B015C0103C0DE
:10742000812C912C540183E50E948D1B882321F02F
:107430000E94841B4B015C010E946D8C0E94D11341
:10744000C0901406D0901506E0901606F09017062E
:10745000C80CD91CEA1CFB1C0E94DD9F811105C0D1
:1074600060E084E597E00E9428A00E9424C86C197F
:107470007D098E099F0997FF02C0A4DFF6CFFF9018
:10748000EF90DF90CF90BF90AF909F908F90089536
:107490008F929F92AF92BF92CF92DF92EF92FF9224
:1074A0001F93CF93DF93C0914606D091470680E5A6
:1074B0000E948D1B882361F00E94FA1A6B017C01E7
:1074C00011E0611571058105910531F410E004C0EA
:1074D00010E0C12CD12C760183E50E948D1B8823FE
:1074E00099F00E94841B6B017C0111110FC0611582
:1074F00071058105910551F48881882339F061E097
:10750000CE010E94E49F07C01123B1F360E08EE03A
:1075100097E00E9428A081E080931A060E946D8C5B
:107520000E94D113C114D104E104F104C9F0809088
:10753000140690901506A0901606B09017068C0CB5
:107540009D1CAE1CBF1C0E9424C8681979098A09B9
:107550009B0997FF17C080911A06811121C012C0A4
:1075600080911A06882311F02DDFFACF8091FE0753
:1075700060E0882319F08FEF96E002C08DEE96E070
:107580000E9428A010921A06DF91CF911F91FF90C0
:10759000EF90DF90CF90BF90AF909F908F90089525
:1075A00011DFD1CF2F923F924F925F926F927F92D5
:1075B0008F929F92AF92BF92CF92DF92EF92FF9203
:1075C0000F931F93CF93DF93CDB7DEB72E970FB6F0
:1075D000F894DEBF0FBECDBF8DE690E00E94A11BE8
:1075E000811109C28091FB0783FD05C283E50E94DA
:1075F0008D1B482E8111B1C182E50E948D1B811126
:10760000ACC10CC06DE070E08FE29CE00E94CA1338
:107610006AE070E08FE29CE00E94CA130E945985E4
:1076200081E080930B0219821A821B821C821D82C8
:107630001E821F821886512C1986FCE3FA872CE1E2
:107640002B8736E43C87E12CF12C90E8C92E2FEBF8
:10765000D22E812C912C54018091D5149091D61466
:10766000BC01882777FD8095982F0E9490D1162F16
:10767000072F782E692E262F372F482F592FB70125
:10768000C6010E94EED0882309F12091DD143091CB
:10769000DE144091DF145091E014612F702F872D7C
:1076A000962D0E94EED0582E551C5524551C442072
:1076B00089F0552079F080910B02882309F4DEC00F
:1076C00060E081EE95E00E9428A0D8C01E2D0F2D0D
:1076D0007C2C6D2C0E9424C86B017C01DC01CB0149
:1076E0002D813E814F815885821B930BA40BB50BD6
:1076F000B7FD45C0D701C60188519C4FAF4FBF4F62
:107700008D839E83AF83B8870E940722E2EFF5E066
:1077100084911F019FEF291A390A882321F00E94C2
:10772000B311F101F5CF81149104A104B104D1F09A
:10773000C501B401605F784D8F4F9F4F6C197D0973
:107740008E099F0928EE33E040E050E00E942CD4DF
:10775000CA01B9014AE050E00E9449128AE00E9441
:10776000B3110DC0EFEEF5E084911F01AFEF2A1ABF
:107770003A0A882321F00E94B311F101F5CF22DEED
:107780000E94D1132090DD143090DE14B091DF14EC
:10779000BE87E091E014ED8791014B2F5E2F612FA2
:1077A000702F872D962D0E9414D09F7781149104FD
:1077B000A104B10449F420E030E040E85FE30E9416
:1077C000EED087FF0BC008C020E030E040E450E47A
:1077D0000E94F1D2181614F446015701552091F178
:1077E00029813A814B815C81211531054105510583
:1077F00041F0D701C601821B930BA40BB50BB7FD5B
:1078000021C091014E855D8569857A858B859C8532
:107810000E9414D020E030E040EC5FE30E94EED004
:1078200087FD49CFD701C601805A9541AF4FBF4F61
:1078300089839A83AB83BC8329863A869E859B87FE
:10784000AD85AC8780910B02882309F434CF811475
:107850009104A104B10429F4E12EF02EC72CD62CFA
:10786000FBCEB0E1CB1AB7E2DB0AE108F108C81899
:10787000D908EA08FB08F7FE1ECFEECFEDEDF5E0E4
:1078800064918F01662361F0772767FD70958FE221
:107890009CE00E94CA130F5F1F4FF8016491F2CF62
:1078A0006DE070E08FE29CE00E94CA136AE070E035
:1078B0008FE29CE00E94CA138091FE078823B1F1F9
:1078C000E9EDF5E064918F01662361F0772767FDAC
:1078D00070958FE29CE00E94CA130F5F1F4FF80162
:1078E0006491F2CF6DE070E08FE29CE00E94CA13D9
:1078F0006AE070E08FE29CE02E960FB6F894DEBF4F
:107900000FBECDBFDF91CF911F910F91FF90EF90F0
:10791000DF90CF90BF90AF909F908F907F906F90AF
:107920005F904F903F902F900C94CA138091260C3B
:10793000882309F460C0E5EDF5E064918F016623CA
:1079400089F2772767FD70958FE29CE00E94CA1349
:107950000F5F1F4FF8016491F2CF0E94D41A0E946A
:107960005DD17093D6146093D5140E94D41A20E090
:1079700030E04AEA52E40E94EED0181654F082E059
:1079800096E00E94C68D60E085E096E00E9428A007
:1079900004C082E096E00E94208E6091D514709120
:1079A000D614882777FD8095982F0E9490D120913A
:1079B000DD143091DE144091DF145091E0140E94E8
:1079C000F1D218162CF460E08AEF95E00E9428A00E
:1079D000E6EFF5E064918F01662309F413CE772773
:1079E00067FD70958FE29CE00E94CA130F5F1F4FE6
:1079F000F8016491F1CF2E960FB6F894DEBF0FBE5A
:107A0000CDBFDF91CF911F910F91FF90EF90DF904D
:107A1000CF90BF90AF909F908F907F906F905F902E
:107A20004F903F902F9008952F923F924F925F92E8
:107A30006F927F928F929F92AF92BF92CF92DF927E
:107A4000EF92FF920F931F93CF93DF93CDB7DEB7E3
:107A50002E970FB6F894DEBF0FBECDBF8091FB0707
:107A600083FDACC1E1EDF5E064918F01662361F027
:107A7000772767FD70958FE29CE00E94CA130F5F25
:107A80001F4FF8016491F2CF6DE070E08FE29CE04F
:107A90000E94CA136AE070E08FE29CE00E94CA1361
:107AA00060E084EC95E00E9428A083E50E948D1B95
:107AB000482E811105C082E50E948D1B8823B1F0FC
:107AC0000E94D41A0E945DD17093D2146093D11495
:107AD0000E94D41A20E030E040EA50E40E94F1D243
:107AE000181624F482E096E00E94208E81E08093B4
:107AF0000B0280911C068093E30519821A821B8277
:107B00001C821D821E821F821886512C1986FCE35E
:107B1000FA872CE12B8736E43C87E12CF12C30E806
:107B2000C32E4FEBD42E812C912C54018091D11473
:107B30009091D214BC01882777FD8095982F0E94E0
:107B400090D1162F072F782E692E262F372F482FEA
:107B5000592FB701C6010E94EED0882301F1209170
:107B6000D9143091DA144091DB145091DC14612F58
:107B7000702F872D962D0E94EED0582E551C55241F
:107B8000551C442081F0552071F080910B02882310
:107B900009F414C1E9EBF5E064918F01D8C01E2D02
:107BA0000F2D7C2C6D2C0E9424C86B017C01DC0104
:107BB000CB012D813E814F815885821B930BA40BF5
:107BC000B50BB7FD45C0D701C60188519C4FAF4FDB
:107BD000BF4F8D839E83AF83B8870E940722E0EC5E
:107BE000F5E084911F019FEF291A390A882321F0BB
:107BF0000E94B311F101F5CF81149104A104B104E5
:107C0000D1F0C501B401605F784D8F4F9F4F6C1963
:107C10007D098E099F0928EE33E040E050E00E9484
:107C20002CD4CA01B9014AE050E00E9449128AE00E
:107C30000E94B3110DC0EDEBF5E084911F01AFEF91
:107C40002A1A3A0A882321F00E94B311F101F5CFD4
:107C5000B9DB0E94D1132090D9143090DA14B0917E
:107C6000DB14BE87E091DC14ED8791014B2F5E2F72
:107C7000612F702F872D962D0E9414D09F7781142D
:107C80009104A104B10449F420E030E040E85FE34E
:107C90000E94EED087FF0BC008C020E030E040E437
:107CA00050E40E94F1D2181614F4460157015520F1
:107CB00091F129813A814B815C8121153105410582
:107CC000510541F0D701C601821B930BA40BB50BE4
:107CD000B7FD21C091014E855D8569857A858B85CB
:107CE0009C850E9414D020E030E040EC5FE30E94CD
:107CF000EED087FD4ACFD701C601805A9541AF4FDC
:107D0000BF4F89839A83AB83BC8329863A869E853D
:107D10009B87AD85AC8780910B02882309F435CF12
:107D200081149104A104B10429F4E12EF02EC72C92
:107D3000D62CFCCEB0E1CB1AB7E2DB0AE108F108A1
:107D4000C818D908EA08FB08F7FE1FCFEECF662354
:107D500061F0772767FD70958FE29CE00E94CA135F
:107D60000F5F1F4FF8016491F2CF6DE070E08FE27A
:107D70009CE00E94CA136AE070E08FE29CE00E94DF
:107D8000CA1360E08FEA95E02E960FB6F894DEBF36
:107D90000FBECDBFDF91CF911F910F91FF90EF905C
:107DA000DF90CF90BF90AF909F908F907F906F901B
:107DB0005F904F903F902F900C9428A02E960FB676
:107DC000F894DEBF0FBECDBFDF91CF911F910F9111
:107DD000FF90EF90DF90CF90BF90AF909F908F90EB
:107DE0007F906F905F904F903F902F900895FF92FB
:107DF0000F931F93CF93DF9380E50E948D1B882301
:107E000009F447C00E94101BEC0183E50E948D1B02
:107E1000882321F00E94101B8C0102C00FEF1FEF7E
:107E2000C80101960397A8F5D7FD33C0E0E8F3E059
:107E3000CE019927219131912817390751F123E07B
:107E4000E63DF207B9F70E946D8CFC2E60E08C2FA6
:107E50000E940FCA0F3F8FEF180759F48C2F0E9412
:107E60007DCA31E020E0892B09F030E0C32FD22F0A
:107E700005C00130110551F4C1E0D0E08F2D0E9402
:107E80007DCA8C179D0729F09DDAF8CFC0E0D0E0BD
:107E9000F5CFDF91CF911F910F91FF9008952F9211
:107EA0003F924F925F926F927F928F929F92AF928A
:107EB000BF92CF92DF92EF92FF920F931F93CF93D7
:107EC000DF93CDB7DEB7C654D1090FB6F894DEBF45
:107ED0000FBECDBF1C017AAB69AB142FDB01CD9077
:107EE000DD90ED90FC90139714968D909D90AD9041
:107EF000BC901797A7019601C701B6010E942CD329
:107F00002B013C01A5019401C501B4010E942CD3B1
:107F10009B01AC01C301B2010E9415D00E9499D30C
:107F20006FAB78AF89AF9AAF8091EB079091EC0778
:107F3000A091ED07B091EE07898F9A8FAB8FBC8F20
:107F4000A7019601BC01CD010E9415D06BAF7CAF9B
:107F50008DAF9EAF8091EF079091F007A091F10750
:107F6000B091F20789A39AA3ABA3BCA3A501940186
:107F7000BC01CD010E9415D023966CAF7DAF8EAFB2
:107F80009FAF23978091F3079091F407A091F50795
:107F9000B091F6078DA39EA3AFA3B8A79C01AD0136
:107FA000D10118966D917D918D919C911B970E94A6
:107FB00014D06D8F7E8F8F8F98A3D1011C968D91D9
:107FC0009D910D90BC91A02D27968CAF9DAFAEAF2B
:107FD000BFAF27978091F7079091F807A091F90715
:107FE000B091FA0789A79AA7ABA7BCA7D701C6018A
:107FF000B0588D8B9E8BAF8BB88FD501C401B05814
:10800000898B9A8BAB8BBC8BD1018D919D910D90FF
:10801000BC91A02D8DA79EA7AFA7B8AB2BAD3CAD53
:108020004DAD5EADBC01CD010E9414D06B017C0151
:10803000D10114968D919D910D90BC91A02D8BAB8B
:108040009CABADABBEAB23962CAD3DAD4EAD5FADA5
:108050002397BC01CD010E9414D04B015C01A70104
:1080600096016D897E898F89988D0E942CD32B0172
:108070003C01A501940169897A898B899C890E94B8
:108080002CD39B01AC01C301B2010E9415D02B017E
:108090003C01A50194016D897E898F89988D0E948C
:1080A0002CD34B015C01A701960169897A898B89E0
:1080B0009C890E942CD39B01AC01C501B4010E9494
:1080C00014D0A30192010E9488D06B017C0120E0B2
:1080D00030E0A9010E94EED087FF0AC02BED3FE0FF
:1080E00049EC50E4C701B6010E9415D06B017C0138
:1080F000112351F02BED3FE049EC50E4C701B601EC
:108100000E9414D06B017C0120E030E0A901C7017E
:10811000B6010E94EED0811122C02DA53EA54FA52B
:1081200058A9698D7A8D8B8D9C8D0E94EED081111E
:1081300016C02BA93CA94DA95EA969A17AA18BA162
:108140009CA10E94EED081110AC02BED3FE049ECCA
:1081500050E4C701B6010E9415D06B017C012FA924
:1081600038AD49AD5AADC701B6010E942CD39B0171
:10817000AC010E942CD34B015C012D8D3E8D4F8DA7
:1081800058A1CA01B9010E942CD39B01AC01C501C1
:10819000B4010E9415D00E9499D34B015C012FE6D7
:1081A00032E143E85AE30E94EED087FDD8C1C50111
:1081B000B4010E94CBD10E9462D17AA369A3FB01D2
:1081C000EF2B21F421E030E03AA329A3A9A1BAA121
:1081D000BD0180E090E00E948ED14B015C019B01CB
:1081E000AC01C701B6010E94F5D0698F7A8F8B8FE1
:1081F0009C8FA50194016D8D7E8D8F8D98A10E941D
:10820000F5D06BAB7CAB8DAB9EAB29A53AA54BA54E
:108210005CA527966CAD7DAD8EAD9FAD27970E9476
:1082200014D0A50194010E94F5D06FAB78AF89AF4F
:108230009AAF298D3A8D4B8D5C8DCA01B9010E9490
:108240002CD320E030E040E05FE30E942CD39B0180
:10825000AC0160E070E080E89FE30E9414D06DA75D
:108260007EA78FA798AB8DA19EA1AFA1B8A5898746
:108270009A87AB87BC8789A59AA5ABA5BCA58D8736
:108280009E87AF87B88B60912F027091300288274C
:1082900077FD8095982F0E9490D1209131023091E6
:1082A000320240913302509134020E942CD32AE0D2
:1082B00037ED43E25CE30E942CD36DA37EA38FA332
:1082C00098A70E9424C82B013C0198EC490E511C30
:1082D000611C711CA1E0B0E0BE8FAD8FB12C2D8D63
:1082E0003E8D89A19AA12817390708F024C10E9460
:1082F00010910E9424C8641975098609970997FD91
:108300000AC00E9424C82B013C01B8EC4B0E511C42
:10831000611C711C57D8B394E8E1EB150CF447C00D
:108320002DA53EA54FA558A969897A898B899C8975
:108330000E942CD36B017C01298D3A8D4B8D5C8D75
:108340006D897E898F89988D0E942CD3A701960113
:108350000E9415D0162FA72E982E892E2DA53EA54A
:108360004FA558A96D897E898F89988D0E942CD33D
:108370006B017C01298D3A8D4B8D5C8D69897A89E1
:108380008B899C890E942CD39B01AC01C701B6014B
:108390000E9414D06D8B7E8B8F8B988F812F9A2D9E
:1083A000A92DB82D898B9A8BAB8BBC8B6DC02D8D75
:1083B0003E8DB90180E090E00E948ED1298D3A8DEA
:1083C0004B8D5C8D0E942CD36B017C010E94F2D0FE
:1083D000698B7A8B8B8B9C8BC701B6010E948FD3E4
:1083E0004B015C01A9A9BAA9CD90DD90ED90FC905C
:1083F0001397F7FAF094F7F8F09414968D919D91F5
:108400000D90BC91A02D89A79AA7ABA7BCA72989DD
:108410003A894B895C89C701B6010E942CD36D8BC8
:108420007E8B8F8B988FA501940169A57AA58BA56A
:108430009CA50E942CD39B01AC016D897E898F89FC
:10844000988D0E9415D06D8B7E8B8F8B988FA50198
:108450009401C701B6010E942CD36B017C012989CC
:108460003A894B895C8969A57AA58BA59CA50E9450
:108470002CD39B01AC01C701B6010E9414D0698BBB
:108480007A8B8B8B9C8BB12C2D893E894F89588D93
:108490006BAD7CAD8DAD9EAD0E9415D069837A83A6
:1084A0008B839C8329893A894B895C8923966CAD9F
:1084B0007DAD8EAD9FAD23970E9415D06D837E83D9
:1084C0008F8398872BA93CA94DA95EA969857A85D8
:1084D0008B859C850E9415D069877A878B879C87BE
:1084E0002FA938AD49AD5AAD6D857E858F859889A8
:1084F0000E9415D06D877E878F87988BCE0101965D
:108500000E948429C0901C06EDA0FEA00FA118A512
:108510009E01235F3F4FAE01475F5F4FBE016B5F20
:108520007F4FCE0101960E94F678ED8DFE8D31963B
:10853000FE8FED8FD4CE9101245F3F4FA101485FA4
:108540005F4FB1016C5F7F4FC0901C06EDA0FEA095
:108550000FA118A5C1010E94F6780E94AD1DCA5B4B
:10856000DF4F0FB6F894DEBF0FBECDBFDF91CF91C6
:108570001F910F91FF90EF90DF90CF90BF90AF9041
:108580009F908F907F906F905F904F903F902F9033
:1085900008954F925F926F927F928F929F92AF92C7
:1085A000BF92CF92DF92EF92FF921F93CF93DF9310
:1085B000CDB7DEB7A4970FB6F894DEBF0FBECDBF20
:1085C000182F80913502882309F488C10E94C21EA9
:1085D00019821A821B821C821D821E821F821886AB
:1085E00082E50E948D1B882309F428C10E94D41AB9
:1085F0006B017C018091EB079091EC07A091ED0756
:10860000B091EE0789879A87AB87BC878090EF0788
:108610009090F007A090F107B090F2078091DB07EF
:108620009091DC07A091DD07B091DE078D879E87D2
:10863000AF87B88B8091DF079091E007A091E107A9
:10864000B091E207898B9A8BAB8BBC8B20E030E03A
:10865000A901C701B6010E94EED0882309F404C124
:1086600029853A854B855C856D857E858F859889C2
:108670000E94EED081110BC0A501940169897A890D
:108680008B899C890E94EED0882309F4EDC020E0FC
:1086900030E0A901C701B6010E94EED0881F8827EB
:1086A000881F181729F080E090E0A0E8BFEB04C015
:1086B00080E090E0A0E8BFE389A39AA3ABA3BCA3AA
:1086C00029853A854B855C856D857E858F85988962
:1086D0000E9414D0698F7A8F8B8F9C8FA501940193
:1086E00069897A898B899C890E9414D06D8F7E8FCD
:1086F0008F8F98A3298D3A8D4B8D5C8DCA01B9015E
:108700000E942CD32B013C012D8D3E8D4F8D58A105
:10871000CA01B9010E942CD39B01AC01C301B20173
:108720000E9415D00E9499D36D8B7E8B8F8B988F72
:1087300020E030E040E05FE30E942CD32B013C01BD
:10874000A7019601C701B6010E942CD36B017C01E1
:10875000A3019201C301B2010E942CD39B01AC0181
:10876000C701B6010E9414D00E9499D39B01AC01AD
:1087700069A17AA18BA19CA10E942CD36B017C01E1
:108780002D853E854F85588969857A858B859C85A1
:108790000E9415D020E030E040E05FE30E942CD33F
:1087A0002B013C016D8D7E8D8F8D98A190582D8968
:1087B0003E894F89588D0E94F5D09B01AC01C701BD
:1087C000B6010E942CD39B01AC01C301B2010E94EF
:1087D00015D029853A854B855C850E9414D0698324
:1087E0007A838B839C8329893A894B895C89C5016B
:1087F000B4010E9415D020E030E040E05FE30E9429
:108800002CD32B013C012D893E894F89588D698DD0
:108810007A8D8B8D9C8D0E94F5D09B01AC01C70198
:10882000B6010E942CD39B01AC01C301B2010E948E
:1088300015D0A50194010E9414D012C089E40E94B1
:108840008D1B882331F00E94D41A69837A838B832D
:108850009C838AE40E948D1B882331F00E94D41AE5
:108860006D837E838F83988720E030E0A901698142
:108870007A818B819C810E94EED081110BC020E017
:1088800030E0A9016D817E818F8198850E94EED0B4
:10889000882351F0412FBE016F5F7F4F8BED97E032
:1088A000FEDA0E94D1131AC0EDEBFAE084917F0149
:1088B0009FEFE91AF90A882321F00E94B311F7010A
:1088C000F5CFEDE5F7E084917F01AFEFEA1AFA0A00
:1088D000882321F00E94B311F701F5CFA4960FB6BB
:1088E000F894DEBF0FBECDBFDF91CF911F91FF90F7
:1088F000EF90DF90CF90BF90AF909F908F907F9040
:108900006F905F904F9008950F931F93CF93DF93D5
:1089100080914C0620E6829FC0011124835B994F11
:1089200090934906809348068091FB0780FF18C00A
:10893000E7EBFAE08491EF012196882321F00E9471
:10894000B311FE01F7CFC0914806D0914906899135
:10895000882319F00E94B311FACF8AE00E94B31164
:108960008091480690914906FC01208101962032B1
:10897000D9F3F0934906E09348062E3461F0C09194
:108980004806D09149066AE270E0CE010E94BCD848
:108990000097D1F420C0818190ED980F9A3010F0AB
:1089A0008D3269F73296DF0131962C9120532A30AF
:1089B000D0F3CD01FC01019620812032D9F3F09350
:1089C0004906E0934806DBCFFC0131968291803264
:1089D00029F08A3219F0FE01219102C01082F6CFEF
:1089E0003E2F9F2F81918032D9F380538A3008F037
:1089F000F0C3A32FB92FE0E0F0E09AE08D91AF0132
:108A0000949FF001959FF00D1124F097E80FF11D50
:108A100087FDFA958C9180538A3080F3CD011196B1
:108A2000EC0138813032D1F39093470680934606AB
:108A30002D3409F45CC0243509F4ABC3273409F0A4
:108A4000C8C3E430F10509F445C020F4E230F10573
:108A5000D8F518C0EA35F10509F442C048F4E5300C
:108A6000F105D9F17C9709F09BC30E94BF1F98C301
:108A7000EB35F105C1F1EC35F10509F091C30E9428
:108A800093208EC380913502882309F489C30E9404
:108A9000C21E8091900A8130A1F4809189158823AB
:108AA00081F020E030E040EA51E46091E707709106
:108AB000E8078091E9079091EA070E94EED087FDD0
:108AC0006FC30E94692A6CC381E0329709F080E08D
:108AD00060DD66C30E94FE3963C30E944A1F60C303
:108AE00010921B065DC381E080931B0659C3EF36CD
:108AF000F10509F4D2C108F09AC0EA32F10509F48F
:108B0000A9C108F053C0E731F10509F467C100F5C8
:108B1000E231F10509F455C278F4E230F10508F4C8
:108B200037C1719709F03CC360E084EE96E00E9483
:108B300028A00E94702C34C3E531F10509F444C12A
:108B400008F047C1749709F02BC3E3EDF6E023C1A9
:108B5000EB31F10509F45DC178F4E931F10509F46F
:108B600045C108F04BC18CEF97E00E94135F82E093
:108B700096E00E94208E14C3EE31F10509F44EC137
:108B800058F47C9709F00CC320E040E0BC018CEF66
:108B900097E00E94F36204C3EF31F10509F457C175
:108BA000B09709F0FDC20E947321FAC2E535F105C4
:108BB00009F40AC2D8F4E135F10509F4E6C168F414
:108BC000EC34F10509F44BC1ED34F10509F44CC165
:108BD000EB34F10509F0E4C23DC1E335F10509F4D8
:108BE000ECC108F0EEC110923B06DAC2EA36F1059C
:108BF00009F496C168F4E836F10509F43AC108F0C1
:108C000068C1EC35F10509F0CBC20E94BF23C8C290
:108C1000EC36F10509F444C108F4A7C1ED36F105BD
:108C200009F478C1EE36F10509F426C1B9C2E33D75
:108C3000F10509F44FC208F056C0EC38F10509F40B
:108C400035C120F5E537F10509F4DEC180F4E237DE
:108C5000F10509F4CAC1E337F10509F4C9C1E037E8
:108C6000F10509F09DC28AE196E00E94922CE83756
:108C7000F10509F4CDC1E937F10509F4CFC1E737B2
:108C8000F10509F08DC20E94C8718AC2E93CF10564
:108C900009F4CCC178F4EE3BF10509F43EC1E83C9F
:108CA000F10509F4C0C1E139F10509F079C20E946A
:108CB000012376C2EC3CF10509F4E7C148F4EB3C32
:108CC000F10509F06DC2C6EDD3E007EA1FE0D0C19F
:108CD000ED3CF10509F4DCC1EE3CF10509F060C2A0
:108CE0000E942C255DC2EA39D1E0FD0709F4DBC002
:108CF00030F5EC3241E0F40709F418C268F4ED3DB8
:108D0000F10509F4F7C1E23EF10509F40CC2EC3DAE
:108D1000F10509F045C2E1C1EE3281E0F80709F43E
:108D20000BC208F406C2EF32D1E0FD0709F407C216
:108D3000E039F14009F034C20E946D8C31C2E63F47
:108D400041E0F40709F404C270F4E43F81E0F8075D
:108D500009F4F8C108F0F9C1EC3AF14009F020C279
:108D60000E94B6271DC2EA3922E0F20709F493C136
:108D700028F4E73FF14009F4EEC112C2E03AC3E043
:108D8000FC0709F45EC0E73EF34009F4F3C108C2F2
:108D90000E94483A05C28491EF012196882321F070
:108DA0000E94B311FE01F7CF8CEF97E00E94D15DD6
:108DB000E4ECF6E08491EF012196882309F4F0C1F8
:108DC0000E94B311FE01F6CF8CEF97E00E94075E80
:108DD000E7C18CEF97E00E94B85EE2C120E041E07D
:108DE000BC018CEF97E00E94F362DAC181E08093CE
:108DF000BD058093EA0E1092FE07D2C18091FF0755
:108E0000882309F4CDC183E50E948D1B8111CEC159
:108E1000C7C18CEF97E00E94DC60C2C18091FF0760
:108E2000882309F4BDC160E08CEF97E00E94536293
:108E300060914606709147068CEF97E00E94E75FCD
:108E4000AFC1BC018CEF97E00E948565A9C10E946B
:108E50001221A6C182E096E00E94208EA1C182E08C
:108E600096E00E94DC8D9CC182E096E00E94C68D57
:108E700097C10E94CC2194C18EE40E948D1B88234F
:108E800009F48EC10E94051B6093D1077093D2072D
:108E90008093D3079093D40783C10E94922280C10C
:108EA00010920B027DC10E94602A7AC18091FB075B
:108EB00083FD76C183E50E948D1B882309F470C170
:108EC0000E94D41A0E945DD17093D2146093D11481
:108ED00067C189E690E00E94A11B81117DC180914C
:108EE000FE07811103C081E08093C605E7E1F6E04B
:108EF0008491EF012196882321F00E94B311FE0195
:108F0000F7CF0E9407228AE0DF91CF911F910F9146
:108F10000C94B3110E94D23A43C10E94143D40C147
:108F200083E50E948D1B882329F00E941D1BD82FEA
:108F3000C92F02C0D3EBC0E080E50E948D1B8823BF
:108F400019F00E941D1B02C080E090E02D2F3C2FE5
:108F5000233B310510F022EB30E0892B09F020C1D2
:108F600030931E0620931D061BC180E50E948D1BB9
:108F7000811105C010921E0610921D0611C10E949B
:108F80001D1B892B09F00CC1F5CF0E946A920E942B
:108F9000028D10921E0610921D0668EE73E080E0AE
:108FA00090E00E9453C860E08FE995E00E9428A0FD
:108FB0000E943FA00E946139F3C081E080933B068C
:108FC000EFC00E947323ECC083E50E948D1B8823B1
:108FD00009F4E6C00E94841B60931006709311068A
:108FE0008093120690931306DBC00E94DD12D8C056
:108FF000E5EDF4E08491EF012196882309F4D0C0D7
:109000000E94B311FE01F6CF60E00E94E49FC8C049
:1090100081E08093390280930B0FC2C01092390215
:1090200010920B0FBDC00E94232CBAC0C6EDD3E036
:1090300007E61FE089910E948D1B882349F00E945A
:10904000D41A0E9462D1F801608371838283938372
:109050000C5F1F4FF3E0CA3DDF0761F70E94CB842E
:109060009FC00C5F1F4FF3E0CA3DDF0709F498C0B3
:1090700089910E948D1B8823A1F30E94D41AF801C4
:109080006083718382839383ECCF0E94592488C0CC
:109090000E94C22485C08AE50E948D1B882351F05E
:1090A0000E94D41A6093DF057093E0058093E10578
:1090B0009093E2054091DF055091E0056091E10554
:1090C0007091E2058FE094E00E9429158AE00E94E9
:1090D000B31166C00E94852563C083E50E948D1B85
:1090E000882309F45DC00E94101B90933002809386
:1090F0002F0256C08DED90E00E94A11B811150C03F
:1091000083E50E948D1B882309F44AC0C091E305C2
:10911000D0E00E94101BFE01EE0FFF1FE35DFD4F2C
:10912000918380833DC00E94F73E3AC00E941B2677
:1091300037C00E945C2634C00E94FC2631C00E94C9
:109140006F272EC00E94C5672BC00E94746E28C076
:109150000E94806925C083E50E948D1B882329F029
:109160000E94591B91E0982701C090E0892F0E942E
:10917000EA6A16C081E0809335020E94A1A083E5CF
:109180000E948D1B882311F10E94591B811108C078
:109190001DC020E040E050E0BA018E2F0E94E1287F
:1091A000DF91CF911F910F910C94FC280E94051B19
:1091B000AB01BC0140937A0A50937B0A60937C0A0E
:1091C00070937D0A89EC99E0FAD7EACF0E941B29B7
:1091D000E7CF0E942D1FE4CFDF91CF911F910F9118
:1091E0000895CF93DF938091BD0581110E94FE18F1
:1091F00080914A06843010F40E94022E60E08CEFC9
:1092000097E00E94856180914A06882309F43FC057
:109210008091FC07882359F1C0914C0680E6C89FD5
:10922000E0011124C35BD94F6BEF71E0CE010E94C6
:109230006ED8892B81F060E08CEF97E00E9453623A
:10924000E8EEF1E08491EF012196882369F00E9415
:10925000B311FE01F7CFBE018CEF97E00E941F61B2
:109260008091FD07811103C00E94FC2801C04CDBE6
:1092700080914A06882359F0815080934A06809154
:109280004C0690E001968370992780934C060E94CB
:10929000E2390E941C1680918F0A882319F10E94DE
:1092A0006D8C10928F0AE4EEF1E06491EF01662379
:1092B00059F0772767FD70958FE29CE00E94CA13F2
:1092C0002196FE016491F3CF6DE070E08FE29CE0A7
:1092D0000E94CA136AE070E08FE29CE0DF91CF91B8
:1092E0000C94CA13DF91CF910895FC012485358534
:1092F000F901E05CFF4F80819181329620813181BC
:10930000805C9F4F821B930B60E470E00C9419D437
:10931000FC0184859585FC01E05CFF4F4081518113
:109320003296208131814217530741F00190F0813C
:10933000E02DE80FF91F808190E008958FEF9FEFF7
:109340000895FC0184859585FC01E05CFF4F408118
:1093500051813296208131814217530779F0A081E3
:10936000B181A80FB91F8C91208131812F5F3F4FB0
:109370002F7333273183208390E008958FEF9FEF81
:109380000895FC0181A1882329F0A489B5898C91D5
:1093900086FFFBCF11A20895CF93DF93FC012685B2
:1093A0003785D901A05CBF4F8D919C911197019693
:1093B0008F739927E901CE5BDF4F4881598184176C
:1093C0009507D9F30D90BC91A02DA20FB31F6C93FC
:1093D000A685B785A05CBF4F11969C938E93A689F6
:1093E000B7892C9181E090E0078C02C0880F991F0B
:1093F0000A94E2F7282B2C9381E081A30488F58955
:10940000E02D80818064808381E090E0DF91CF91C6
:1094100008951F920F920FB60F9211240BB60F9260
:109420002F933F934F938F939F93EF93FF9380914D
:10943000300182FD1CC0409136018091D50C909185
:10944000D60C01968F7399272091D70C3091D80CA8
:109450008217930771F0E091D50CF091D60CEB5682
:10946000F34F40839093D60C8093D50C02C080912B
:109470003601FF91EF919F918F914F913F912F91E5
:109480000F900BBE0F900FBE0F901F9018951F925C
:109490000F920FB60F9211240BB60F922F933F939A
:1094A0008F939F93EF93FF932091910C3091920CA7
:1094B0008091930C9091940C2817390731F4809186
:1094C00031018F7D8093310114C0E091930CF091B4
:1094D000940CEF5AF34F20818091930C9091940C4F
:1094E00001968F7399279093940C8093930C2093FB
:1094F0003601FF91EF919F918F913F912F910F90A6
:109500000BBE0F900FBE0F901F901895CF92DF9259
:10951000EF92FF92CF93DF93EC016A017B0141153B
:1095200081EE580761057105F9F0EC89FD8981E04C
:1095300090E008A002C0880F991F0A94E2F7808388
:1095400060E079E08DE390E0A70196010E942CD4C1
:10955000215031094109510956954795379527956D
:10956000211580E1380798F0EC89FD89108260E8C8
:1095700074E88EE190E0A70196010E942CD421505E
:109580003109410951095695479537952795E8893D
:10959000F9893083EA89FB89208319A2EE89FF8942
:1095A000408181E090E09C010C8C02C0220F331FAF
:1095B0000A94E2F7422B4083EE89FF8940819C01A7
:1095C0000D8C02C0220F331F0A94E2F7422B408316
:1095D000EE89FF8940819C010E8C02C0220F331F4F
:1095E0000A94E2F7422B4083EE89FF8920810F8C99
:1095F00002C0880F991F0A94E2F780958223808326
:10960000DF91CF91FF90EF90DF90CF90089510926F
:10961000320C1092310C88EE93E0A0E0B0E0809321
:10962000330C9093340CA093350CB093360C86EF2A
:1096300093E09093300C80932F0C85E99CE09093FD
:109640003C0C80933B0C81E59CE090933E0C809316
:109650003D0C85E391E09093400C80933F0C84E3B4
:1096600091E09093420C8093410C80E391E09093C1
:10967000440C8093430C81E391E09093460C8093DB
:10968000450C82E391E09093480C8093470C86E36D
:1096900091E090934A0C8093490C84E080934B0CAA
:1096A00083E080934C0C87E080934D0C85E08093A1
:1096B0004E0C81E080934F0C08958FEF8EBD0DB45A
:1096C00007FEFDCF8EB508958EBD0DB407FEFDCF0C
:1096D000089561E0FC0180810C9448CAFC0122815C
:1096E000322F306A36953CBD20FD06C031E0263071
:1096F00009F430E0232F01C020E02DBD60E0FC0123
:1097000080810C9448CACF92DF92EF92FF920F9320
:109710001F93CF93DF93EC018B017A010E9424C841
:109720006B01CBDF8B838F3F49F40E9424C86C19F7
:109730007D096D327140A8F381E103C08E3F41F095
:109740008FE08983CE01C5DF8FEFBEDF80E026C0CA
:10975000E114F104E1F081E0E81AF1088FEF8EBD29
:10976000F8012FEFCF01801B910B8E159F0538F468
:109770000DB407FEFDCF8EB581932EBDF3CF0DB492
:1097800007FEFDCF8EB5F801EE0DFF1D808395DF3E
:1097900094DFCE019EDF8FEF97DF81E0DF91CF91E5
:1097A0001F910F91FF90EF90DF90CF9008950F934E
:1097B0001F93CF93DF93EB010E9424C88B017DDFC1
:1097C0008F3F49F00E9424C8601B710B6C177D0706
:1097D000B0F380E001C081E0DF91CF911F910F9144
:1097E0000895CF92DF92FF920F931F93CF93DF9351
:1097F00000D01F92CDB7DEB76C01F62E29833A83D5
:109800004B835C836BDF6CE271E0C601D0DF8F2D90
:1098100080645ADF08E110E05C814B813A81298144
:10982000DA01C901002E04C0B695A79597958795D2
:109830000A94D2F729833A834B835C8345DF08502F
:10984000110929813A814B815C81083F8FEF18070C
:1098500039F7FF2029F0E8E0FE1621F08FEF03C072
:1098600085E901C087E830DFFCE0FF1201C025DF99
:1098700010E023DFF601838387FF04C01F3F11F050
:109880001F5FF7CF0F900F900F900F90DF91CF9148
:109890001F910F91FF90DF90CF900895BF92CF92CC
:1098A000DF92EF92FF920F931F93CF93DF93EC0120
:1098B000B62E1C82198248830E9424C88B0161E065
:1098C00088810E940FCACE0104DF2398229A219A30
:1098D000209A289A85E08A8382E58CBD1DBC2AE007
:1098E000F22E8FEFF1DEFA94E1F720E030E0A901EB
:1098F00060E0CE0176DFF82E8B8381E0F81649F028
:109900000E9424C8601B710B613D774070F381E0B9
:1099100046C02AEA31E040E050E068E0CE0161DF75
:1099200082FF02C0FC820CC094E0F92EC6DE8B835D
:10993000FA94E1F78A3A11F082E031C082E08C8338
:109940008C81823031F4C12CD12CE12C80E4F82EB2
:1099500003C0C12CD12C760120E030E0A90167E3DF
:10996000CE013FDFA701960169E2CE013ADF8B838A
:10997000882349F00E9424C8601B710B613D774029
:1099800058F38AE00CC08C818230B1F420E030E0E2
:10999000A9016AE3CE0125DF882329F088E08983C5
:1099A000CE0197DE14C089DE807C803C11F483E018
:1099B0008C8383DE82DE81DECE018BDE86E08B153A
:1099C00018F488E1898303C0BA8281E001C080E095
:1099D000DF91CF911F910F91FF90EF90DF90CF908B
:1099E000BF9008950F931F93CF93DF93EC018901EC
:1099F0008C81833039F039E0440F551F661F771F83
:109A00003A95D1F79A01AB0161E1CE01EADE81110D
:109A100009C040E052E0B801CE01DF91CF911F9123
:109A20000F9171CE84E08983CE0153DE80E0DF9117
:109A3000CF911F910F910895CF93DF93EC016EBDED
:109A400020E030E00DB407FEFDCFFA01E20FF31F76
:109A500080818EBD0DB407FEFDCF81818EBD2E5F4E
:109A60003F4F211582E0380769F70DB407FEFDCF9F
:109A70008FEF2ADE8FEF28DE20DE8B838F7185301B
:109A800031F083E18983CE0124DE80E001C081E0F2
:109A9000DF91CF9108950F931F93CF93DF93EC0144
:109AA00089018C81833039F089E0440F551F661F8E
:109AB000771F8A95D1F79A01AB0168E1CE0191DE5B
:109AC000882311F086E01EC0A8016EEFCE01B4DF3E
:109AD0008823C9F068E572E0CE0169DE182F811194
:109AE00002C087E10FC020E030E0A9016DE0CE01A7
:109AF00078DE811106C0E1DD811103C0CE01E9DD10
:109B000005C086E18983CE01E4DD10E0812FDF917D
:109B1000CF911F910F910895CF93DF93EC019C019A
:109B20002C5F3F4F41E050E060E070E0898D9A8DFE
:109B30000E946358882399F04D895E896F89788DDA
:109B4000452B462B472B59F44C815D816E817F81DB
:109B50004D8B5E8B6F8B788F998190689983DF91A5
:109B6000CF910895CF92DF92EF92FF920F931F93C0
:109B7000CF93DF93EC0189899A89AB89BC89803EB8
:109B80009F4FAF41B10510F080E06AC0CE01C4DF45
:109B90008823D1F30E947756182F8823A9F3E98DE3
:109BA000FA8DCC80DD80EE80FF8032E0C31AD108D0
:109BB000E108F108058404C0CC0CDD1CEE1CFF1C80
:109BC0000A94D2F786859785A089B189C80ED91ED7
:109BD000EA1EFB1E81E08093DF0CC092E20ED09261
:109BE000E30EE092E40EF092E50E80E092E0E2EE09
:109BF000FCE0DF019C011D9221503040E1F701E0C3
:109C0000E98DFA8D8481081788F422EE3CE0B701D3
:109C1000A601400F511D611D711D8091E00C9091B6
:109C2000E10C39DF8823E1F00F5FEACFC12C82E03D
:109C3000D82EE12CF12C058404C0CC0CDD1CEE1CCC
:109C4000FF1C0A94D2F749895A896B897C894C0D8B
:109C50005D1D6E1D7F1D498B5A8B6B8B7C8B812FFD
:109C6000DF91CF911F910F91FF90EF90DF90CF90F8
:109C70000895CF93DF93EC0141E0611101C040E012
:109C80006C857D858E859F850E94B756882341F01F
:109C9000888920E2829FC00111248E51934F02C017
:109CA00080E090E0DF91CF91089530E020E04EE237
:109CB000DC015C91503271F0383029F4FB01E20F85
:109CC000F11D40832F5FFB01E20FF11DDC015C9170
:109CD00050832F5F3F5F01963B3051F7FB01E20F4E
:109CE000F11D10820895CF93DF93EB01FC012381D6
:109CF000211102C080E00EC02250223020F48FE2F9
:109D00008883198206C060E0B4DF009799F3BE0132
:109D1000CCDF81E0DF91CF910895FB012BE030E2B1
:109D200031932150E9F7DC0190E027E03A2FEB2F47
:109D30008D9181110AC0DA013C931196EC9381E078
:109D4000FB019081903239F525C08F32A1F38E321C
:109D500019F0E4ECFAE008C02A30E1F098E02AE0DB
:109D6000E5CF31963817B1F034913111FACF291778
:109D700088F0813278F08F3769F031E0390FFB01DC
:109D8000E90FF11D9FE9980F9A3108F48052808302
:109D9000932FCCCF80E008950F931F93CF93DF9341
:109DA000EC018B018B81882311F080E042C0FB0124
:109DB0008789803139F18032C1F783E08B83F801E4
:109DC000428D538D648D758D4D8B5E8B6F8B788F2F
:109DD0009E012F5E3F4FC8010E946E57882329F3D2
:109DE0001A8F098F81E089831C821D821E821F8247
:109DF000188619861A861B861C861D861E861F8657
:109E0000188A17C082E08B831D8A1E8A1F8A188ECB
:109E1000FB01408D518D60E070E095E0440F551FCF
:109E2000661F771F9A95D1F7498B5A8B6B8B7C8B6A
:109E3000D7CFDF91CF911F910F9108952F923F922D
:109E40004F925F926F927F928F929F92AF92BF924A
:109E5000CF92DF92EF92FF920F931F93CF93DF93F6
:109E6000EC015B016A018B81811103C08FEF9FEFD1
:109E7000C6C0898180FFFACF49895A896B897C895C
:109E800088859985AA85BB852601612C712C8A015C
:109E90009B01081B190B2A0B3B0B04151505260506
:109EA000370518F46A01C81AD90A76013E0124E080
:109EB000620E711CE114F10409F476C048855985DD
:109EC0006A857B854A0181E098222B811A012B014A
:109ED000E9E05694479437942794EA95D1F7898D11
:109EE0009A8DFC01223049F4628D738D848D958D9D
:109EF000620D731D841D951D3CC0148111501221EB
:109F000081149104C1F4111116C0452B462B472B27
:109F100049F48D899E89AF89B88D8C839D83AE83EA
:109F2000BF8309C04C815D816E817F81930157D7CA
:109F3000882309F49BCFE98DFA8D6C817D818E8118
:109F40009F816250710981099109058404C0660FDF
:109F5000771F881F991F0A94D2F726853785408975
:109F60005189620F731F841F951F610F711D811D21
:109F7000911D20E032E02819390987012E153F058F
:109F800008F489010115F2E01F0761F52091E20E46
:109F90003091E30E4091E40E5091E50E6217730785
:109FA0008407950719F41EC0C60129C09501AB01AD
:109FB000BC018091E00C9091E10C14DD882309F440
:109FC00055CFA00EB11E88859985AA85BB85800FC7
:109FD000911FA11DB11D88879987AA87BB87E01AA9
:109FE000F10A68CF40E0C3D6882309F43FCFB4011B
:109FF0006E51734FA801C5010E9495D8E2CFDF9141
:10A00000CF911F910F91FF90EF90DF90CF90BF9075
:10A01000AF909F908F907F906F905F904F903F9008
:10A020002F900895CF93DF931F92CDB7DEB741E015
:10A0300050E0BE016F5F7F4F01DF019719F4898106
:10A0400090E002C08FEF9FEF0F90DF91CF910895C6
:10A05000AF92BF92CF92DF92EF92FF920F931F9336
:10A06000CF93DF936C01EB017A01DC0113968C91A5
:10A070001397823070F018960D911D912D913C919F
:10A080001B970F71112722273327012B022B032B3C
:10A0900011F08FEF58C04115510511F0F7011082F2
:10A0A0001DE040E250E0BE01C601C8DE9C018032E6
:10A0B000910531F081E0232B09F480E0819543C0C4
:10A0C00088818823C1F1853E61F38E3251F3E1141A
:10A0D000F10461F19B859F739F3041F54A8D5B8D43
:10A0E000452B21F58F719FEF980F9230F8F490E097
:10A0F0000197189F9001199F300D1124FE0180E0F7
:10A1000090E05701A20EB31E8530B8F46181A5011D
:10A11000480F591FDA016C93019632968D309105E4
:10A1200099F7888186FF02C0F50115868B8583FD2E
:10A13000B8CF822F08C080E006C08B3010F4648155
:10A14000E6CF6681E4CFDF91CF911F910F91FF9011
:10A15000EF90DF90CF90BF90AF9008951F93CF9373
:10A16000DF93EC018B81823018F480E090E023C013
:10A17000488559856A857B85A5E0769567955795CD
:10A180004795AA95D1F7142F1F70CE014BDF97FD8D
:10A19000ECCF488559856A857B85415E5F4F6F4F5F
:10A1A0007F4F488759876A877B8720E2129FC001CB
:10A1B00011248E51934FDF91CF911F9108954F92AB
:10A1C0005F926F927F92AF92BF92CF92DF92EF92A7
:10A1D000FF920F931F93CF93DF93EC016A017B01F2
:10A1E0002B81222349F089899A89AB89BC898417FC
:10A1F0009507A607B70710F480E06BC0223009F47A
:10A2000063C0C114D104E104F10449F41C821D822D
:10A210001E821F82188619861A861B8659C0888559
:10A220009985AA85BB85E98DFA8DE585F0E039969B
:10A23000AC01BD0141505109610971090E2E04C0E4
:10A2400076956795579547950A94D2F797018601B9
:10A25000015011092109310904C036952795179538
:10A260000795EA95D2F7041715072607370720F058
:10A27000892B8A2B8B2B49F48D899E89AF89B88DC8
:10A280008C839D83AE83BF8304C0041B150B260BF8
:10A29000370B280139015E0184E0A80EB11C41147E
:10A2A00051046104710481F04C815D816E817F8174
:10A2B0009501898D9A8D93D591E0491A51086108CD
:10A2C00071088111ECCF05C0C886D986EA86FB8665
:10A2D00081E0DF91CF911F910F91FF90EF90DF9080
:10A2E000CF90BF90AF907F906F905F904F90089508
:10A2F0000F931F93CF93DF93EC018B818823D1F1D0
:10A30000898187FF32C061E0CE01B3DC8C01009708
:10A3100089F1FC018081853E69F18B81823040F4B6
:10A3200049895A896B897C89448F558F668F778FCD
:10A330004D895E896F89788DF801538F428F758BB7
:10A34000648BE091D90CF091DA0C309759F0B80198
:10A350006A5E7F4FC80148961995F801808D918DEE
:10A36000938B828B89818F778983DF91CF911F9126
:10A370000F91BDC481E0888380E0DF91CF911F9170
:10A380000F910895CF93DF93EC01B2DF1B82DF9131
:10A39000CF910895FC0123812111F4CF08954F92AC
:10A3A0005F926F927F92AF92BF92CF92DF92EF92C5
:10A3B000FF920F931F93CF93DF9300D01F92CDB7DF
:10A3C000DEB75C016A017B01FC0183818130E9F425
:10A3D000818181FF1AC0F50181899289A389B4899D
:10A3E00084179507A607B70780F0892B8A2B8B2B3C
:10A3F00009F472C0F5014084518462847384B7010A
:10A40000A601C501DCDE811102C080E066C0F50155
:10A41000818D928DC114D104E104F10469F4458960
:10A4200056896789708D58D7882379F3F501158A85
:10A43000168A178A108E37C0F501448155816681CE
:10A4400077819E012F5F3F4FCAD48823F1F2498163
:10A450005A816B817C81F501818D928DFC01278968
:10A46000203139F4483FFFEF5F0761057105D8F4EB
:10A4700007C0483F2FEF520762072FE0720798F49A
:10A480002BD7882309F4C1CFF5014481558166811A
:10A4900077810FEF1FEF2FEF3FE0818D928D84D5F5
:10A4A000882309F4B2CFF501C18AD28AE38AF48AFB
:10A4B000818180688183C5011BDF882309F4A5CFD2
:10A4C000B701A6014C145D046E047F0410F4B301BF
:10A4D000A201C50174DE01C081E00F900F900F90C2
:10A4E0000F90DF91CF911F910F91FF90EF90DF9030
:10A4F000CF90BF90AF907F906F905F904F900895F6
:10A50000FF920F931F93CF93DF93EC01F42E80E221
:10A51000689FF0011124EE51F34F8385817121F082
:10A52000842F827109F04EC08091E20E9091E30E6B
:10A53000A091E40EB091E50E8C879D87AE87BF8712
:10A54000688B4489558960E070E0BA01552744273B
:10A55000028D138D20E030E0402B512B622B732BAA
:10A560004D8B5E8B6F8B788F8385887151F4048D52
:10A57000158D268D378D098B1A8B2B8B3C8B81E0AB
:10A580000BC08031F9F49E012F5E3F4F898D9A8D6B
:10A59000A5D48823B9F084E08B838F2D8F708983B5
:10A5A0001C821D821E821F82188619861A861B86AF
:10A5B000F4FE0BC040E050E0BA01CE01F0DE8111A4
:10A5C00004C011C01B8280E00EC0F5FE0BC049899B
:10A5D0005A896B897C89CE01DF91CF911F910F91B0
:10A5E000FF90EDCD81E0DF91CF911F910F91FF9012
:10A5F0000895AF92BF92CF92DF92EF92FF920F93A6
:10A600001F93CF93DF937C01EB016A01B22E898DFA
:10A610009A8DF701928F818F40E050E0BA01CE0110
:10A62000CEDDA12C088519852A853B8589899A89E3
:10A63000AB89BC89081719072A073B07A0F585E0F5
:10A6400036952795179507958A95D1F70F70CE0106
:10A6500085DD009709F481C0FC012081222311F0DF
:10A66000253EB9F4A1100EC04091E20E5091E30EC8
:10A670006091E40E7091E50EF70144875587668777
:10A680007787008BFC018081AA24A3948111CACF13
:10A690000AC04BE050E0BC01C6010E9488D8892B5B
:10A6A00009F0C0CF58C08B2D8274823409F055C098
:10A6B000AA2049F0F701008961E0C701DADAEC016C
:10A6C000009769F44AC08B81823009F446C0CE01FC
:10A6D00049DA882309F441C0C2EEDCE000E080E200
:10A6E000FE0111928A95E9F78BE0F601DE010190F7
:10A6F0000D928A95E1F7E091D90CF091DA0C309740
:10A7000039F0BE01625F7F4FCE014096199508C0B7
:10A7100081E298E2998B888B80E098E09F878E8712
:10A72000888999899B8B8A8B998F888F8E859F8545
:10A730009F8B8E8BDCD2882381F04B2D602FC7013D
:10A74000DF91CF911F910F91FF90EF90DF90CF900D
:10A75000BF90AF90D5CEB7FEF0CF80E0DF91CF9124
:10A760001F910F91FF90EF90DF90CF90BF90AF902F
:10A7700008953F924F925F926F927F928F929F9235
:10A78000AF92BF92CF92DF92EF92FF920F931F93FF
:10A79000CF93DF93CDB7DEB7C354D1090FB6F8948A
:10A7A000DEBF0FBECDBF5C016B0124965FAF4EAF25
:10A7B0002497522E1C8E1F8E19821C8261157105E2
:10A7C00011F410E073C0FC0183818111FACF24964B
:10A7D000EEADFFAD249780818F3211F076011DC060
:10A7E0002496EEADFFAD249780818F3231F43196FF
:10A7F0002496FFAFEEAF2497F3CFF601838182500A
:10A80000823060F3F601618D728DCE010196C4DA5B
:10A810008823B9F2CE0101967C018E01045E1F4FA0
:10A820003801FE0131964F01402E312E19C0882388
:10A83000A9F121E0AE01495C5F4FB701C801D9DE43
:10A84000882309F4BECFEC14FD0411F0C7019ADD92
:10A850000615170501F1942D832D7801092F182F66
:10A86000AE014E5B5F4FBE01695C7F4F24968EAD9B
:10A870009FAD249752DA882309F4A3CF2496EEAD36
:10A88000FFAD249780818F3291F631962496FFAFE9
:10A89000EEAF2497F3CF982D892DDFCF252DAE0174
:10A8A000495C5F4FB701C501A4DE182FCE010196A8
:10A8B00071DDCE014C966EDD812FCD5BDF4F0FB683
:10A8C000F894DEBF0FBECDBFDF91CF911F910F91E6
:10A8D000FF90EF90DF90CF90BF90AF909F908F90C0
:10A8E0007F906F905F904F903F900895CF93DF934C
:10A8F000EC0140E050E0BA0152DD882361F061E0F4
:10A90000CE01B7D9009739F025EEFC0120831B82D8
:10A91000DF91CF91ECC180E0DF91CF9108951F933B
:10A92000CF93DF93CDB7DEB76B970FB6F894DEBF4A
:10A930000FBECDBFAB0119821C8222E0BC01CE014B
:10A94000019617DF182F882321F0CE010196CEDF64
:10A95000182FCE0101961EDD812F6B960FB6F8944D
:10A96000DEBF0FBECDBFDF91CF911F9108952F9213
:10A970003F924F925F926F927F928F929F92AF928F
:10A98000BF92CF92DF92EF92FF920F931F93CF93DC
:10A99000DF9300D01F921F92CDB7DEB78C015B0111
:10A9A0003A01DC0113968C9113978130C1F4119612
:10A9B0008C9181FF14C082FF18C0F801418952892F
:10A9C0006389748980859185A285B38584179507ED
:10A9D000A607B70751F0C801F2DB811106C081E07C
:10A9E000F80180838FEF9FEF37C1630183C0D801E7
:10A9F00059968D919C915A97FC01F481F1501A015E
:10AA00002B0169E056944794379427946A95D1F7BF
:10AA1000F221FD834A0121E09222FF2309F476C04E
:10AA200080E092E08819990976018C159D0508F45B
:10AA30007C01D8015996ED91FC915A9714962D906E
:10AA40003D904D905C901797B2E02B1A3108410869
:10AA50005108058404C0220C331C441C551C0A9464
:10AA6000D2F786859785A089B189280E391E4A1E9E
:10AA70005B1EED812E0E311C411C511CE114F2E0D5
:10AA8000FF0609F089C08091E20E9091E30EA0913B
:10AA9000E40EB091E50E82159305A405B50569F4A1
:10AAA0001092DF0C8FEF9FEFDC018093E20E90930A
:10AAB000E30EA093E40EB093E50E9501B201A1015F
:10AAC0008091E00C9091E10C0E944B4D882309F499
:10AAD00086CFF80180859185A285B3858E0D9F1D57
:10AAE000A11DB11D80879187A287B387AE0CBF1CC3
:10AAF000CE18DF08D80118964D915D916D917C912B
:10AB00001B97C114D10409F072CF7AC0811491044B
:10AB100009F086CF14964D915D916D917C911797B8
:10AB2000411551056105710559F455968D919D9119
:10AB30000D90BC91A02D0097A105B10539F520C05D
:10AB40009E012F5F3F4F4BD1882309F448CF898165
:10AB50009A81AB81BC81F801218D328DF901278961
:10AB6000203139F4883FFFEF9F07A105B10540F47C
:10AB70000DC0883F2FEF9207A2072FE0B20730F0F9
:10AB8000C8010E948C4D81114BCF29CFF8018483DD
:10AB90009583A683B78344CF8114910411F5D8011E
:10ABA00018964D915D916D917C911B9751968D9169
:10ABB0009D910D90BC91A02D481759076A077B07FE
:10ABC00080F095D0882309F40ACF81E08093DF0CD0
:10ABD0002092E20E3092E30E4092E40E5092E50E87
:10ABE00007C041E0C201B101C2D0882309F4F7CE09
:10ABF000A701B501C4018E51934F0E9495D869CF2A
:10AC000051968D919D910D90BC91A02DF8012181BF
:10AC100084179507A607B70738F4418B528B638BCF
:10AC2000748B206821830CC08091D90C9091DA0C30
:10AC3000892B31F06114710419F02068F801218327
:10AC4000D80111968C9183FD02C0C30105C0C801D3
:10AC50004FDB8111FACFC3CE0F900F900F900F9062
:10AC60000F90DF91CF911F910F91FF90EF90DF90A8
:10AC7000CF90BF90AF909F908F907F906F905F909C
:10AC80004F903F902F900895CF93DF931F92CDB7B1
:10AC9000DEB72091C6153091C715CE01019621155A
:10ACA000310519F0821B930B02C08C5C95410F900B
:10ACB000DF91CF910895CF93DF931F92CDB7DEB789
:10ACC000698341E050E0BE016F5F7F4F04964FDE25
:10ACD0000F90DF91CF910895FB0101900020E9F7DB
:10ACE000AF0141505109461B570B049640CECF93FC
:10ACF0008091DF0C8823B9F14091E20E5091E30E70
:10AD00006091E40E7091E50E22EE3CE08091E00C43
:10AD10009091E10C0E944B4DC82F811102C0C0E000
:10AD200023C04091DB0C5091DC0C6091DD0C7091E4
:10AD3000DE0C411551056105710591F022EE3CE0F4
:10AD40008091E00C9091E10C0E944B4D882339F3E7
:10AD50001092DB0C1092DC0C1092DD0C1092DE0CC9
:10AD60001092DF0C01C0C1E08C2FCF910895CF92DB
:10AD7000DF92EF92FF92CF936B017C01C42F809101
:10AD8000E20E9091E30EA091E40EB091E50E8C15C9
:10AD90009D05AE05BF05C9F0AADF811102C080E0A4
:10ADA00018C022EE3CE0B701A6018091E00C909122
:10ADB000E10C0E94F24C882391F3C092E20ED092F3
:10ADC000E30EE092E40EF092E50E81E0C111809373
:10ADD000DF0CCF91FF90EF90DF90CF9008958F928E
:10ADE0009F92AF92BF92CF92DF92EF92FF920F931A
:10ADF0001F93CF93DF93EC016A017B018901898561
:10AE00009A85AB85BC850196A11DB11D8417950758
:10AE1000A607B70710F480E054C08F89803129F469
:10AE20009927872F762F652F0BC08032A1F7CB0192
:10AE3000BA0127E096958795779567952A95D1F77A
:10AE40008B889C88AD88BE88680D791D8A1D9B1DE6
:10AE50008090E20E9090E30EA090E40EB090E50E8C
:10AE6000681579058A059B0581F48F89803191F4F5
:10AE7000DD24EE24FF24F601EE0FFF1FEE51F34F09
:10AE800080819181A0E0B0E016C040E070DF8111C8
:10AE9000ECCFC1CFE894C7F8DD24EE24FF24F601FF
:10AEA000EE0FFF1FEE0FFF1FEE51F34F80819181D8
:10AEB000A281B381BF70F80180839183A283B383A1
:10AEC00081E0DF91CF911F910F91FF90EF90DF9084
:10AED000CF90BF90AF909F908F9008954F925F92C8
:10AEE0006F927F92AF92BF92CF92DF92EF92FF92DA
:10AEF0000F931F93CF93DF9300D01F92CDB7DEB790
:10AF00008C0149835A836B837C835901C12CD12CDA
:10AF10007601412C42E0542E612C712C49815A81DA
:10AF20006B817C819E012F5F3F4FC80158DF8823D2
:10AF300041F1D301C201F801058404C0880F991FB3
:10AF4000AA1FBB1F0A94D2F7C80ED91EEA1EFB1E09
:10AF500049815A816B817C818789803139F481E014
:10AF6000483F5F4F6105710538F4D8CF81E0483F15
:10AF70005F4F6F4F7F4090F2F501C082D182E28235
:10AF8000F3820F900F900F900F90DF91CF911F9150
:10AF90000F91FF90EF90DF90CF90BF90AF907F9098
:10AFA0006F905F904F9008954F925F926F927F9253
:10AFB0008F929F92AF92BF92CF92DF92EF92FF92C9
:10AFC0000F931F93CF93DF93EC014A015B0128019C
:10AFD0003901423051056105710508F462C04985A7
:10AFE0005A856B857C854F5F5F4F6F4F7F4F48154C
:10AFF00059056A057B0508F454C08F89803129F40E
:10B00000FF24EB2CDA2CC92C0CC0803209F049C08B
:10B010007501640177E0F694E794D794C7947A9524
:10B02000D1F74B895C896D897E89C40ED51EE61ED9
:10B03000F71E41E0C701B6019ADE882391F19F898E
:10B04000903159F49924AA24BB24F401EE0FFF1F78
:10B05000EE51F34F5182408210C0E89487F8992452
:10B06000AA24BB24F401EE0FFF1FEE0FFF1FEE51C9
:10B07000F34F40825182628273829A89923090F0BB
:10B080004D815E816F8178854C0D5D1D6E1D7F1D2C
:10B090004093DB0C5093DC0C6093DD0C7093DE0C62
:10B0A00001C080E0DF91CF911F910F91FF90EF9051
:10B0B000DF90CF90BF90AF909F908F907F906F90D8
:10B0C0005F904F9008952F923F924F925F926F92B0
:10B0D0007F928F929F92AF92BF92CF92DF92EF9228
:10B0E000FF920F931F93CF93DF93CDB7DEB72F97C8
:10B0F0000FB6F894DEBF0FBECDBF1C014C875D8735
:10B100006E877F873B872A87DC0119960D911D91F9
:10B110002D913C911C970F5F1F4F2F4F3F4F0D8379
:10B120001E832F833887EA85FB8580809180A280EB
:10B13000B38081149104A104B10431F0FFEF8F1AA0
:10B140009F0AAF0ABF0A10C0DC018D909D90AD90A0
:10B15000BC90B1E0B9870C851D852E853F850130F7
:10B1600011052105310509F0198675016401412C8D
:10B17000512C3201F10181859285A385B485481651
:10B1800059066A067B0608F04EC00D811E812F818C
:10B1900038850C151D052E053F0550F4F2E0CF2E25
:10B1A000D12CE12CF12CA2E08A2E912CA12CB12CD7
:10B1B0009E012F5F3F4FB701A601C10110DE88231A
:10B1C00091F149815A816B817C81D701C601019639
:10B1D000A11DB11D452B462B472B19F04C015D01DC
:10B1E0000FC0AC01BD01481959096A097B090C85DA
:10B1F0001D852E853F85401751076207730741F073
:10B200001FEF411A510A610A710A6C017D01B2CF28
:10B210000FEF1FEF2FEF3FE0B701A601C101C4DE22
:10B220008D83811113C01D823DC02601370121E0AD
:10B23000421A51086108710897018601B301A20101
:10B24000C101B2DE882379F3730162018C149D047D
:10B25000AE04BF0450F3AA85BB854D915D916D91FD
:10B260007C914115510561057105A9F4EA85FB85BD
:10B2700080829182A282B382F985FF2399F00FEF39
:10B28000801A900AA00AB00AD1018D929D92AD92C7
:10B29000BC92139707C095018401C10185DE81111D
:10B2A000E5CFC1CF8D812F960FB6F894DEBF0FBECC
:10B2B000CDBFDF91CF911F910F91FF90EF90DF9065
:10B2C000CF90BF90AF909F908F907F906F905F9046
:10B2D0004F903F902F900895AF92BF92CF92DF9200
:10B2E000EF92FF920F931F93CF93DF9300D01F92A3
:10B2F000CDB7DEB75C016A017B0182E090E0A0E09F
:10B30000B0E0F50180839183A283B3839E012F5F18
:10B310003F4FB701A601C50162DD811102C080E087
:10B3200023C000E010E09801B701A601C5013CDE92
:10B330008823A9F3C980DA80EB80FC80F501878936
:10B34000803149F481E0F8EFCF16FFEFDF06E1042A
:10B35000F10450F4DBCF81E098EFC9169FEFD906D6
:10B36000E9069FE0F90690F20F900F900F900F9072
:10B37000DF91CF911F910F91FF90EF90DF90CF90D1
:10B38000BF90AF9008957F928F929F92AF92BF929D
:10B39000CF92DF92EF92FF920F931F93CF93DF93A1
:10B3A000EC01142F7093E10C6093E00C1F8A82E093
:10B3B00090E0A0E0B0E088839983AA83BB831092D9
:10B3C000DF0C1092DB0C1092DC0C1092DD0C109252
:10B3D000DE0C8FEF9FEFDC018093E20E9093E30E83
:10B3E000A093E40EB093E50E442349F1453008F0F4
:10B3F000DEC040E060E070E0CB01B9DC882309F4F6
:10B40000D6C020E1129FF0011124E057F14F808156
:10B410008F7709F0CCC084859585A685B78584365D
:10B420009105A105B10508F4C2C0C084D184E284AD
:10B43000F384C114D104E104F10421F4B8C0C12C97
:10B44000D12C760140E0C701B60191DC782E88232B
:10B4500009F4ADC08091ED0C9091EE0C81159240F5
:10B4600009F0A5C03091F20C332309F4A0C08091FB
:10B47000F00C9091F10C892B09F499C02091EF0CFC
:10B48000222309F494C03A8B2C831D8630E041E0DE
:10B4900050E06D85062FCA01062E02C0880F991F45
:10B4A0000A94E2F72817390731F081E0860F8D877B
:10B4B000683078F37CC02091F80C3091F90C21159C
:10B4C000310519F040E050E008C02091060D3091A0
:10B4D000070D4091080D5091090D2D833E834F8338
:10B4E00058878091F00C9091F10C46015701880E1D
:10B4F000991EA11CB11C8B8A9C8AAD8ABE8AE091E0
:10B50000F30CF091F40CF98FE88FA091F20CB0E0FD
:10B510000E9470D4680D791D8A1D9B1D6A8F7B8FD8
:10B520008C8F9D8FB5E0EE0FFF1FBA95E1F7E150CC
:10B53000FE4FEF2FFF27E695DC01CB018E0F9F1FFB
:10B54000A11DB11D8E879F87A88BB98B8090F50CAC
:10B550009090F60C8114910419F0A12CB12C08C024
:10B560008090020D9090030DA090040DB090050DF9
:10B57000A7019601281B390B4A0B5B0BDA01C901A5
:10B58000880D991DAA1DBB1D04C0B695A79597955A
:10B5900087950A95D2F789879A87AB87BC87853FBD
:10B5A0003FE09307A105B10520F48CE08F8B712C4F
:10B5B00015C0853F9F4FA105B10510F480E10DC076
:10B5C00080910E0D90910F0DA091100DB091110D65
:10B5D0008A8F9B8FAC8FBD8F80E28F8B872DDF9101
:10B5E000CF911F910F91FF90EF90DF90CF90BF9080
:10B5F000AF909F908F907F900895FC0114821782E6
:10B600001382128286E094E0918380830895CF9222
:10B61000DF92EF92FF920F931F93CF93DF93EC0192
:10B620008F96EBDFCE01805B9F4FE7DF7E012FE639
:10B63000E20EF11C87016E013BE5C31A3EEFD30A0F
:10B64000C801DBDF015E1F4F0C151D05C9F7FE01A8
:10B65000EA55FE4F89E1818314823596178ACE011F
:10B6600087539E4FCADF198218821B821A82FE01FD
:10B67000E658FD4F10821182128213823496108296
:10B68000118212821382F8011082FE01E851FE4FEE
:10B69000108286E391E0F7019C0111922150304025
:10B6A000E1F7FE01EA57FD4F81E080831EA61DA64B
:10B6B0000E9424C8CE57DD4F68577C4E8F4F9F4F56
:10B6C000688379838A839B83DF91CF911F910F9148
:10B6D000FF90EF90DF90CF9008952BE1FB0134961F
:10B6E000DC01149601900D922A95E1F7FB0122816D
:10B6F0003381FC013383228326E034E031832083CD
:10B700000895FC0120E03EE2DB014C91403241F023
:10B71000283011F430833196DB014C91408331960F
:10B720002F5F6F5F7F4F2B3079F7108208952F9234
:10B730003F924F925F926F927F928F929F92AF92C1
:10B74000BF92CF92DF92EF92FF920F931F93CF930E
:10B75000DF93CDB7DEB7CA58D1090FB6F894DEBF74
:10B760000FBECDBF7C016B015A012901CA57DF4FC3
:10B770001882C658D0403C0122E1620E711C84E060
:10B78000A80EB11C87010B5F1F4FF701E957FD4F52
:10B79000C957DF4FF983E883C758D0401701F7E74F
:10B7A0002F1AFDEF3F0A80E490E08C0F9D1F049656
:10B7B000C757DF4F99838883C958D040A301BE0182
:10B7C0006F5F7F4FC5010E94285018160CF096C17C
:10B7D0002C85322F3871303161F4C957DF4FE88141
:10B7E000F981C758D040808191810197029708F074
:10B7F000F8C08981882309F481C1853EF9F28E322F
:10B80000E9F28F35D9F2F7018289882321F08E324F
:10B81000A9F28F3599F223FDD1CF81E0303109F0C3
:10B8200080E0F7018483811106C08985873431F671
:10B830008A858E3719F2BE016F5F7F4FC80161DFC5
:10B84000C957DF4FE881F981C758D0408081918185
:10B850008330910509F077C0809138028090E80E1E
:10B860009090E90E8823B9F060E274E0C8010E946C
:10B87000F4D8892B41F465E274E0C8010E94F4D841
:10B88000892B09F44FC0FFEF8F1A9F0A9092E90E9F
:10B890008092E80E47C08091270C9091280C881A5E
:10B8A000990A8091E60E9091E70E24E082169104A9
:10B8B00030F09401245031098217930750F1881514
:10B8C000990538F5B6018FE29CE00E94E3CAB80101
:10B8D0008FE29CE00E94E3CA6DE070E08FE29CE0A2
:10B8E0000E94CA136AE070E08FE29CE00E94CA13D3
:10B8F000B3018FE29CE00E94E3CA6DE070E08FE24A
:10B900009CE00E94CA136AE070E08FE29CE00E9413
:10B91000CA138091E60E9091E70E01969093E70E80
:10B920008093E60E2091E60E3091E70E8091E80EAE
:10B930009091E90E2817390708F440CF1092E70ECE
:10B940001092E60E3BCF0097B1F44601F4018191CD
:10B950004F01882319F00E94B311F8CF4801F40178
:10B9600081914F01882319F00E94B311F8CF8AE02A
:10B970000E94B31123CF8130910539F4F101808108
:10B98000918101969183808319CF029709F016CF98
:10B99000BE016F5F7F4FC801B4DE4114510439F01E
:10B9A000B801C2010E949ED8892B79F4A7C0CA575A
:10B9B000DF4FF881C658D0402F2F30E0F101808151
:10B9C00091812817390709F499C0CA57DF4FF881C8
:10B9D000C658D040FF5FCA57DF4FF883C658D040E3
:10B9E000EDCEBE016F5F7F4FCE0187589F4F89DE3E
:10B9F000A0961FAEA097F6018081811107C06AE072
:10BA000074E0CE01815A9F4F0E94B1D8B601CE0199
:10BA1000815A9F4F0E94B1D8BE0167587F4FCE0117
:10BA2000815A9F4F0E94B1D86AE074E0CE01815ADA
:10BA30009F4F0E94B1D8CE01805C9F4FDEDD21E098
:10BA4000AE0147585F4FB501C757DF4F88819981D5
:10BA5000C958D0400E94B953811136C0C957DF4F31
:10BA6000E881F981C758D04080819181892B61F5A7
:10BA7000E7EBFAE084914F012FEF821A920A8111CD
:10BA800005C08CE0882E84E0982E04C00E94B3117B
:10BA9000F401F0CFF40181914F01882319F00E9445
:10BAA000B311F8CF8AE00E94B311CE0187589F4F9F
:10BAB0004C01F40181914F01882319F00E94B311C8
:10BAC000F8CF8AE00E94B311BE01605C7F4FCE01C7
:10BAD000819603DE20E030E0AE014F5D5F4FBE0196
:10BAE000615A7F4FC70123DECE0181960E9422302A
:10BAF000CE01805C9F4F0E94223060CEC657DF4F40
:10BB00000FB6F894DEBF0FBECDBFDF91CF911F916E
:10BB10000F91FF90EF90DF90CF90BF90AF909F90EC
:10BB20008F907F906F905F904F903F902F900895EF
:10BB30000F931F93CF93DF93CDB7DEB76F970FB6F9
:10BB4000F894DEBF0FBECDBF8C01FC01E957FD4F5D
:10BB500083E090E09183808340E050E0BA01C80127
:10BB6000C3960E94DF50B801615D7F4FCE01019600
:10BB7000B4DD20E030E0AE014F5F5F4F61EB74E079
:10BB8000C801D5DDCE0101960E9422306F960FB616
:10BB9000F894DEBF0FBECDBFDF91CF911F910F9103
:10BBA00008950F931F93CF93DF93CDB7DEB76F97B1
:10BBB0000FB6F894DEBF0FBECDBF8C01FC01E95774
:10BBC000FD4F1182108240E050E0BA01C3960E94FE
:10BBD000DF50B801615D7F4FCE0101967EDD20E030
:10BBE00030E0AE014F5F5F4F61EB74E0C8019FDD55
:10BBF000CE0101960E9422306F960FB6F894DEBFF8
:10BC00000FBECDBFDF91CF911F910F910895EF929D
:10BC1000FF920F931F93CF93DF93EC011B828EA9AA
:10BC2000882321F0CE01C3960E94C2517E018AE58D
:10BC3000E81A8EEFF80A45E360E0C7010E944E4C17
:10BC4000811119C0E7EBFAE084918F010F5F1F4F5C
:10BC5000882321F00E94B311F801F6CFE1EDFCE05A
:10BC600084918F010F5F1F4F882309F465C00E94E4
:10BC7000B311F801F5CF8E0105551E4F41E0B70114
:10BC8000C80181DB81111FC040E0B701C8017BDB27
:10BC9000811119C0EDEBFAE084918F010F5F1F4F06
:10BCA000882321F00E94B311F801F6CFEDEBFCE000
:10BCB00084918F010F5F1F4F882309F43DC00E94BC
:10BCC000B311F801F5CFB801CE01C3960E94CC4E56
:10BCD000811118C0EDEBFAE084918F010F5F1F4FC7
:10BCE000882321F00E94B311F801F6CFECEAFCE0C2
:10BCF00084918F010F5F1F4F8823F1F00E94B311D1
:10BD0000F801F6CF81E08B83E7EBFAE084918F01B5
:10BD10000F5F1F4F882321F00E94B311F801F6CF67
:10BD2000E0EAFCE084918F010F5F1F4F882321F030
:10BD30000E94B311F801F6CFCE01805B9F4F2BE13B
:10BD4000FE01F396DC01149601900D922A95E1F71D
:10BD500029A93AA9FC01338322833297AF96D18374
:10BD6000C083DF91CF911F910F91FF90EF900895C5
:10BD7000FC01128213820895CF92DF92EF92FF921C
:10BD80000F931F93CF93DF93CDB7DEB7CDB6DEB65B
:10BD9000FB0101900020E9F7E61BF70B34968DB705
:10BDA0009EB78E1B9F0B0FB6F8949EBF0FBE8DBF24
:10BDB0000DB71EB70F5F1F4F7F936F9389E99CE00C
:10BDC0009F938F931F930F930E940ED9780194E055
:10BDD000E90EF11C0F900F900F900F900F900F90A5
:10BDE000F7018081882349F0992787FD90950E946B
:10BDF0003FD8F70181937F01F3CF60E0C8010E9433
:10BE0000791885E99CE00E94F9180FB6F894DEBE17
:10BE10000FBECDBEDF91CF911F910F91FF90EF909C
:10BE2000DF90CF900895FC012381222381F021E04F
:10BE300022838091EA0E882351F08DE89CE00E94D5
:10BE4000F91889E89CE00E94F9181092EA0E08950A
:10BE5000FC011282E053FE4F2081222321F0835304
:10BE60009E4F0C94C25108950F931F93CF93DF936D
:10BE70001F921F92CDB7DEB7FC0123812223A9F1C7
:10BE8000E053FE4F2081222311F1E655FF4F408100
:10BE90005181628173814115510561057105B9F0C8
:10BEA0008C0102581D4FCB01BA016D597F4F8F4F46
:10BEB0009F4F24E630E040E050E00E942CD4F8018F
:10BEC00060817181828193810E942CD401C020E025
:10BED00030E03A832983CE0101960E94F0BFBC0175
:10BEE0008FE29CE00E94E3CA12C0E1E8FCE06491AA
:10BEF0008F01662361F0772767FD70958FE29CE0E4
:10BF00000E94CA130F5F1F4FF8016491F2CF0F9088
:10BF10000F90DF91CF911F910F910895AF92BF9233
:10BF2000CF92DF92EF92FF920F931F93CF93DF9305
:10BF30001F92CDB7DEB78C018FE2FB0181935F01C9
:10BF4000D12C21E07801FBE5EF1AFEEFFF0A9FE11B
:10BF5000C92EF7018081D816C8F4B501C801CD9C5F
:10BF6000800D911D11248D589F4F29830E94734E7F
:10BF7000C50129815C010196F5013081332321F04F
:10BF80002D3810F42F5FF6CFD394E3CF27FD11C0E7
:10BF9000B501C80183539E4F0F90DF91CF911F9140
:10BFA0000F91FF90EF90DF90CF90BF90AF900C94E7
:10BFB000734EF50110820F90DF91CF911F910F9179
:10BFC000FF90EF90DF90CF90BF90AF9008954F9289
:10BFD0005F926F927F928F929F92AF92BF92CF9219
:10BFE000DF92EF92FF920F931F93CF93DF93CDB722
:10BFF000DEB7AC970FB6F894DEBF0FBECDBF7C01A5
:10C000005B01FC018381882309F4BFC0C70120DFE5
:10C01000CE0101966C01F1DA27019EE4490E511C14
:10C02000C7018F96F20191838083F50180818F3261
:10C0300009F05BC06FE270E0C5010E94BCD88C01C2
:10C040000F5F1F4F09F457C06FE270E0C8010E94F4
:10C05000BCD84C01009709F44FC00817190708F025
:10C060004BC03C01601A710AA301B801CE01809651
:10C070000E94E5D8E0E2F0E0EC0FFD1FE60DF71DB1
:10C0800010828E01005E1F4FF80181918F0188237D
:10C0900019F00E94B311F8CF8AE00E94B311F201A7
:10C0A000608171816115710519F06C5F7F4F02C06D
:10C0B00060E070E021E0AE01405E5F4FCE0105968A
:10C0C0000E94B95381110CC0BE01605E7F4F87E6AC
:10C0D0009BE00E94D0148EE20E94B3118AE050C00F
:10C0E000F201D182C0828401ABCFC701805B9F4F38
:10C0F000F201918380838501F20180819181009713
:10C1000011F0049602C080E090E0B8010E948F54C4
:10C11000882301F1E9E5FBE084915F019FEFA91A13
:10C12000B90A882321F00E94B311F501F5CFF80177
:10C1300081918F01882319F00E94B311F8CF8AE012
:10C140000E94B311F701E258FD4F10821182128252
:10C15000138218C0E1E4FBE084917F019FEFE91AAC
:10C16000F90A882321F00E94B311F701F5CFF801F5
:10C1700081918F01882319F00E94B311F8CF8EE2CC
:10C180000E94B311C6010E942230AC960FB6F894FB
:10C19000DEBF0FBECDBFDF91CF911F910F91FF90FA
:10C1A000EF90DF90CF90BF90AF909F908F907F9057
:10C1B0006F905F904F9008950F931F93CF93DF93ED
:10C1C000EC018B81882359F1EFE2FBE084918F0130
:10C1D0000F5F1F4F882321F00E94B311F801F6CFA3
:10C1E000FE01E258FD4F60817181828193814AE0B6
:10C1F00050E00E9429128FE20E94B311C658DD4F11
:10C20000688179818A819B814AE050E00E942912ED
:10C210008AE0DF91CF911F910F910C94B311EEE161
:10C22000FBE08491EF012196882321F00E94B31155
:10C23000FE01F7CFDF91CF911F910F910895AF923B
:10C24000BF92CF92DF92EF92FF920F931F93CF9303
:10C25000DF935C01EB01FB0101900020E9F78F0106
:10C2600001501109061B170B6C01F3E3CF1AFEEF07
:10C27000DF0AF60110826EE470E0CE010E94BCD8A5
:10C280007C01009729F4F8013197EC0FFD1F0DC0D8
:10C2900060E270E00E94BCD8EC0121966AE270E096
:10C2A000C7010E94BCD8FC0131978DE081838AE0F0
:10C2B00082831382BE01C50187539E4F0E946C5634
:10C2C000F60180818823B1F0EDEBFAE08491EF0173
:10C2D0002196882321F00E94B311FE01F7CFE7E0F9
:10C2E000FBE08491EF012196882321F00E94B31195
:10C2F000FE01F7CFDF91CF911F910F91FF90EF904B
:10C30000DF90CF90BF90AF9008956F927F928F9201
:10C310009F92AF92BF92CF92DF92EF92FF920F93D4
:10C320001F93CF93DF93CDB7DEB7AA970FB6F894DC
:10C33000DEBF0FBECDBF8C018A579D4F7C016111BE
:10C3400014C0FC018081882309F498C00E9424C88D
:10C35000F801EE57FD4F80809180A280B38068196C
:10C3600079098A099B0997FF89C0F7011082F801B2
:10C370008381811107C0C8014ADCF80183818823C9
:10C3800009F47CC0F80186A58F9385A58F938EEF65
:10C390009AE09F938F937E01F1E2EF0EF11CFF92E2
:10C3A000EF920E940ED90F900F900F900F900F9068
:10C3B0000F90B12CF70101900020E9F73197EE19A9
:10C3C000FF09BE1684F46701CB0CD11CB7FCDA94CC
:10C3D000F6018081992787FD90950E943FD8F6014C
:10C3E0008083B394E7CF4801F3E38F0E911C40E0C4
:10C3F00050E0BA01C4010E94DF50612CCE010196C9
:10C400005C0140E050E0B501C4010E9428501816BC
:10C410004CF5712CF50101900020E9F73197EA19EC
:10C42000FB097E1674F46501C70CD11C77FCDA9405
:10C43000F601808190E00E943FD8F60180837394DA
:10C44000E9CF8A858E37E9F245E050E0B701C501B2
:10C450000E94D7D8892BA9F6B701C8018DDC6624C4
:10C460006394CFCF611004C08FEF9FEFF80104C039
:10C47000F80185A596A5019696A785A7AA960FB659
:10C48000F894DEBF0FBECDBFDF91CF911F910F910A
:10C49000FF90EF90DF90CF90BF90AF909F908F90E4
:10C4A0007F906F9008950F931F93CF93DF93EC01CC
:10C4B0008C0103531E4FC8010E947851C8010E948D
:10C4C000C25119821882DF91CF911F910F91089567
:10C4D000CF93DF93FC0112821092EA0E10928D0A24
:10C4E00060E0E1DF0E94602AE5E8FCE06491EF0192
:10C4F000662359F0772767FD70958FE29CE00E94D4
:10C50000CA132196FE016491F3CF6DE070E08FE2D3
:10C510009CE00E94CA136AE070E08FE29CE00E94F7
:10C52000CA135F9A1092D5078A9A479A1092D60733
:10C530009FB7F894809108018160809308019FBFA4
:10C54000479A1092D707129ADF91CF910895CF9210
:10C55000DF92EF92FF920F931F93CF93DF93CDB7AC
:10C56000DEB76F970FB6F894DEBF0FBECDBF8C015C
:10C570006A017C018EE4E80EF11CC801805B9F4FCC
:10C58000F70191838083E75CFD4F22E030E0318347
:10C59000208332967183608340E050E0BA010496B4
:10C5A0000E94DF50F70160817181CE01019695D81C
:10C5B0009601AE014F5F5F4F61EB74E0C801B7D8E1
:10C5C000CE0101960E9422306F960FB6F894DEBF1E
:10C5D0000FBECDBFDF91CF911F910F91FF90EF90D4
:10C5E000DF90CF9008953F924F925F926F927F922B
:10C5F0008F929F92AF92BF92CF92DF92EF92FF9273
:10C600000F931F93CF93DF93CDB7DEB7AC970FB6E1
:10C61000F894DEBF0FBECDBF8C016B01342EFC0140
:10C620008381882309F459C2E053FE4F8081882317
:10C6300009F48CC0222309F422C27801F8E1EF1A30
:10C64000FEEFFF0AF7018081882331F1EDEBFAE07C
:10C6500084918F010F5F1F4F882321F00E94B31137
:10C66000F801F6CFEEE3FCE084918F010F5F1F4FDE
:10C67000882321F00E94B311F801F6CF6AE070E040
:10C6800081E090E00E9453128AE00E94B31185E39A
:10C690009CE00E94922C21C28FE29CE00E94E3CA9F
:10C6A000F7018081B801FDE88F9F600D711D112495
:10C6B00063517E4FC80132DCE7EBFAE084915F0101
:10C6C0002FEFA21AB20A882321F00E94B311F501BC
:10C6D000F5CFB6018CE19CE00E94D014F701808177
:10C6E000B801FDE88F9F600D711D112463517E4FCD
:10C6F00081E19CE00E94D014580122E8A21A2DEF9B
:10C70000B20AF50140815181628173818BE09CE026
:10C710000E9461158AE00E94B311F7012081F8019F
:10C7200084E0289FE00DF11D1124AF0147515E4FB9
:10C73000F50180819181A281B381FA018083918387
:10C74000A283B3832F5FF70120831FC0F801E85154
:10C75000FE4F10828FE29CE00E94E3CA6DE070E021
:10C760008FE29CE00E94CA136AE070E08FE29CE0D6
:10C770000E94CA1322E0B22E84C1B6018EEF9BE064
:10C780000E94D0148AE00E94B311C80161DBCE017F
:10C7900001965C010E94FD5A28019EE4490E511C3D
:10C7A000C8018F96F20191838083F60180818F32D8
:10C7B00009F079C07601FFEFEF1AFF0A09F479C09A
:10C7C0006FE270E0C7010E94BCD84C01009709F4E9
:10C7D00071C0E816F90608F06DC03C016E187F08BC
:10C7E000A301B701CE0180960E94E5D8E0E2F0E017
:10C7F000EC0FFD1FE60DF71D1082CE0180967C0127
:10C80000F70181917F01882319F00E94B311F8CFBD
:10C810008AE00E94B311F201608171816115710596
:10C8200019F06C5F7F4F02C060E070E021E0AE0164
:10C83000405E5F4FCE0105960E94B95381112EC014
:10C84000EAEEFBE084918F010F5F1F4F811104C05E
:10C850008E01005E1F4F04C00E94B311F801F2CF99
:10C86000F80181918F01882319F00E94B311F8CF4C
:10C870008EE20E94B311E6EEFBE064918F01662325
:10C8800009F4B1C0772767FD70958FE29CE00E94A4
:10C89000CA130F5F1F4FF8016491F1CFF201B1820B
:10C8A000A082740188CFC801805B9F4FF201918301
:10C8B00080837601C80183539E4F4C01F201608151
:10C8C0007181332009F49CC06115710519F06C5F0A
:10C8D0007F4F02C060E070E021E0A701C4010E9428
:10C8E000B953882309F462C0F40181899289A3892C
:10C8F000B4896801F6E8CF1AFDEFDF0AF6018083FC
:10C900009183A283B383B70188ED9BE00E94D0148A
:10C91000F601408151816281738180ED9BE00E942C
:10C9200061158AE00E94B311F801E258FD4F1082B0
:10C93000118212821382E1ECFBE084916F012FEFF0
:10C94000C21AD20A882321F00E94B311F601F5CF52
:10C95000EDEBFBE064916F01662369F0772767FDDB
:10C9600070958FE29CE00E94CA138FEFC81AD80A14
:10C97000F6016491F1CF6DE070E08FE29CE00E94DF
:10C98000CA136AE070E08FE29CE00E94CA13A7011C
:10C9900060E070E0C801DBDDF8018289882319F0CE
:10C9A000C801429601C0C70160E063C0B70189EACF
:10C9B0009BE00E94D0148EE20E94B3118AE00E9494
:10C9C000B311E5EAFBE064918F01662361F07727FC
:10C9D00067FD70958FE29CE00E94CA130F5F1F4FA6
:10C9E000F8016491F2CF6DE070E08FE29CE00E946C
:10C9F000CA136AE070E08FE29CE00E94CA133BC059
:10CA00006115710519F06C5F7F4F02C060E070E046
:10CA100026E5A701C4010E94B95381111DC0B701C9
:10CA200081E99BE00E94D0148EE20E94B3118AE05B
:10CA30000E94B311EDE8FBE064918F01662399F247
:10CA4000772767FD70958FE29CE00E94CA130F5F05
:10CA50001F4FF8016491F2CF81E0F8018083B601A5
:10CA60008BE79BE00E94D0148AE00E94B31160E043
:10CA7000C7010E94E49FC5010E9422302EC0BB2442
:10CA8000B394E7EBFAE084917F012FEFE21AF20A08
:10CA9000882321F00E94B311F701F5CFE6E0FCE016
:10CAA00084917F019FEFE91AF90A882321F00E94FF
:10CAB000B311F701F5CFE1E0BE1203C08AE294E0C2
:10CAC00002C080E394E07C01F70181917F0188231B
:10CAD00009F453CE0E94B311F7CFAC960FB6F89479
:10CAE000DEBF0FBECDBFDF91CF911F910F91FF90A1
:10CAF000EF90DF90CF90BF90AF909F908F907F90FE
:10CB00006F905F904F903F90089521E0FC0121834A
:10CB100020E040E068CDCF92DF92EF92FF920F933A
:10CB20001F93CF93DF93CDB7DEB76F970FB6F8940F
:10CB3000DEBF0FBECDBF8C016C012EE4C20ED11C36
:10CB4000805B9F4FF60191838083E75CFD4F21E07E
:10CB500030E0318320837801F7E7EF1AFDEFFF0A19
:10CB6000F7011182108240E050E0BA0104960E9461
:10CB7000DF50F60160817181CE0101960E946D5BEC
:10CB800020E030E0AE014F5F5F4F61EB74E0C80121
:10CB90000E94975BCE0101960E942230F7018081AE
:10CBA00091816F960FB6F894DEBF0FBECDBFDF91B7
:10CBB000CF911F910F91FF90EF90DF90CF9008954C
:10CBC000AF92BF92CF92DF92EF92FF920F931F939B
:10CBD000CF93DF93CDB7DEB76F970FB6F894DEBF74
:10CBE0000FBECDBF8C01B62EA72ECE0101960E949E
:10CBF000FD5AF801E95AFF4F80817801811104C084
:10CC00002FE2E20EF11C03C030E5E30EF11C6701D8
:10CC100044E0C40ED11C21E04B2D5A2DB601CE01AB
:10CC200005960E94B953811127C0E7EBFAE0849181
:10CC30008F010F5F1F4F882321F00E94B311F8016D
:10CC4000F6CFE8EEFAE084918F010F5F1F4F81115C
:10CC500003C00B2D1A2D04C00E94B311F801F3CFAD
:10CC6000F80181918F01882319F00E94B311F8CF48
:10CC70008AE00E94B31130C0F801EB55FE4F80816D
:10CC80008A30D0F491E0980F908398014FE1849F0F
:10CC9000200D311D1124C90181599F4F2BE1F6014F
:10CCA000DC01149601900D922A95E1F7F70122819B
:10CCB0003381FC0133832283005B1F4F8BE1FE0134
:10CCC0003596D801149601900D928A95E1F78B81E3
:10CCD0009C81F80193838283CE0101960E942230C9
:10CCE0006F960FB6F894DEBF0FBECDBFDF91CF9128
:10CCF0001F910F91FF90EF90DF90CF90BF90AF907A
:10CD00000895CF93DF93FC01EB55FE4F2081222342
:10CD1000D1F021502083EC013FE1239FC00DD11DB4
:10CD20001124C159DF4F805B9F4F2BE1FE013496E8
:10CD3000DC01149601900D922A95E1F72A813B813E
:10CD4000FC0133832283DF91CF910895EF92FF920C
:10CD50000F931F93CF93DF93EC010E946D8C7E01A4
:10CD600083E3E81A8EEFF80AC7010E94C2518E01D0
:10CD700008511E4FF8018081882371F18150808312
:10CD8000BE01FDE88F9F600D711D112463517E4F20
:10CD900021E041E0CE0127DCF8018081FE0194E032
:10CDA000899FE00DF11D1124E751FE4F4081518113
:10CDB00062817381FE01E258FD4F4083518362839B
:10CDC0007383C7010E94DF50CE01DF91CF911F9185
:10CDD0000F91FF90EF9027C81A828CED9AE00E9485
:10CDE000F91882E096E00E94C68D82E096E00E94EB
:10CDF000F38D6D3371058105910520F088ED9AE082
:10CE00000E94F9181092910A10922E0C8C98109290
:10CE10008915E4EDFAE06491EF01662359F0772774
:10CE200067FD70958FE29CE00E94CA132196FE0177
:10CE30006491F3CF6DE070E08FE29CE00E94CA1332
:10CE40006AE070E08FE29CE0DF91CF911F910F913B
:10CE5000FF90EF900C94CA13CF92DF92EF92FF9263
:10CE60000F931F93CF93DF938C01D42EC62FD72F10
:10CE7000D60EDC1609F43CC07E016991F801808170
:10CE800091810E9432DBF801808191810E942ADB2E
:10CE9000C82EF7018081C816D1F0E7EBFAE0849143
:10CEA0007F019FEFE91AF90A882321F00E94B3114C
:10CEB000F701F5CFE4EBFFE084917F019FEFE91AE2
:10CEC000F90A882321F00E94B311F701F5CF2091D0
:10CED000040F3091050F2C0D311D3093050F209359
:10CEE000040FF80180819181019691838083C1CFE5
:10CEF000DF91CF911F910F91FF90EF90DF90CF9036
:10CF00000895EF92FF920F931F93CF93DF931F9299
:10CF1000CDB7DEB78C017B01460FF801808191818E
:10CF200049830E942ADBF70181937F012091040F3E
:10CF30003091050F280F311D3093050F2093040FFA
:10CF4000F8018081918101969183808349814E11FE
:10CF5000E4CF0F90DF91CF911F910F91FF90EF9051
:10CF600008950E94CB840E9435850E94ED8E0E9418
:10CF7000112C80E090E00E94D81B81E090E00E949C
:10CF8000D81B82E090E00C94D81B8F929F92AF92B6
:10CF9000BF92CF92DF92EF92FF920F931F93CF93A6
:10CFA000DF93CDB7DEB767970FB6F894DEBF0FBE3D
:10CFB000CDBF19861A861B861C8680E390E3A0E30A
:10CFC000B0E08D839E83AF83B88784E690E09C8B2E
:10CFD0008B8B44E0BE016B5F7F4FCE0143963CDFFD
:10CFE0008B899C8902969C8B8B8B1092050F1092DB
:10CFF000040F40E167E97FE0CE0143962DDF40E179
:10D0000067EA7FE0CE01439627DF40E167E67FE0F5
:10D01000CE01439621DF44E06BE57FE0CE014396ED
:10D020001BDF44E067E57FE0CE01439615DF44E077
:10D0300063E57FE0CE0143960FDF44E06FE57FE0DC
:10D04000CE01439609DF44E06FE37FE0CE014396D3
:10D0500003DF44E063E67FE0CE014396FDDE40E17E
:10D0600063E47FE0CE014396F7DE4CE06FE176E0CB
:10D07000CE014396F1DE83E08F8B8E8B1D8A19865D
:10D080001A861B861C8641E0BE016B5E7F4FCE0177
:10D090004396E2DE44E0BE01675F7F4FCE014396D8
:10D0A000DBDE41E0BE01695E7F4FCE014396D4DEF8
:10D0B00041E0BE016A5E7F4FCE014396CDDE10E0B7
:10D0C0009F898E89212F30E0989FC0011124281755
:10D0D00039074CF444E0BE01675F7F4FCE014396B1
:10D0E000BBDE1F5FEDCF19821A821B821C8244E0D7
:10D0F000BE016F5F7F4FCE014396AEDE44E06FED21
:10D1000075E0CE014396A8DE19861A861B861C861A
:10D1100019E0115044E039F0BE01675F7F4FCE0146
:10D1200043969ADEF6CF65E875E1CE01439694DE2C
:10D1300044E061E875E1CE0143968EDE44E06DE7A0
:10D1400075E1CE01439688DEC12C80E8D82E8BE3B2
:10D15000E82E85E4F82E812C912C90E8A92E9FE3EF
:10D16000B92E11111EC044E060E972E0CE01439671
:10D1700073DE44E06CE872E0CE0143966DDE44E07D
:10D1800068E872E0CE01439667DE89869A86AB86B0
:10D19000BC8644E0BE01675F7F4FCE0143965CDEF4
:10D1A0001AC0C986DA86EB86FC8644E0BE01675F5A
:10D1B0007F4FCE01439650DE19861A861B861C8649
:10D1C00004E0015041F044E0BE01675F7F4FCE01B3
:10D1D000439642DEF6CF1F5F143009F0C2CF84E1E0
:10D1E00090E09A8B898B42E0BE016F5E7F4FCE014B
:10D1F000439632DE80E090E8ABE3B5E489879A8716
:10D20000AB87BC87115041F044E0BE01675F7F4FA0
:10D21000CE01439621DEF6CF80E290E0988B8F8797
:10D2200042E0BE01615F7F4FCE01439615DE41E0D3
:10D2300067E376E0CE0143960FDE11110CC08091BA
:10D24000290290912A02A0912B02B0912C02898789
:10D250009A87AB87BC8744E0BE01675F7F4FCE01F2
:10D260004396FADD1F5F143041F78091040F9091CF
:10D27000050F9E878D87EB88FC8884E690E09C8B69
:10D280008B8B44E066E374E0CE014396E5DD42E03B
:10D29000BE01635F7F4FCE014396DEDDE7EBFAE030
:10D2A00084916F019FEFC91AD90A882321F00E9447
:10D2B000B311F601F5CFB70182EA9FE00E94F614A0
:10D2C000E9E9FFE084917F019FEFE91AF90A8823D9
:10D2D00021F00E94B311F701F5CF67960FB6F894CD
:10D2E000DEBF0FBECDBFDF91CF911F910F91FF9099
:10D2F000EF90DF90CF90BF90AF909F908F90089568
:10D30000AF92BF92DF92EF92FF920F931F93CF9352
:10D31000DF93CDB7DEB7E0970FB6F894DEBF0FBE50
:10D32000CDBF80E1ECE2F3E0DE01919601900D9239
:10D330008A95E1F780E1ECE3F3E0DE01519601909C
:10D340000D928A95E1F780E1ECE4F3E0DE011196BD
:10D3500001900D928A95E1F77E0181E2E80EF11CC1
:10D3600007E91FE0BE016F5E7F4F47EA5FE09E0165
:10D370002F5F3F4FE7E6AE2EEFE0BE2ED12CF70138
:10D3800081919191A191B1917F01F8018193919344
:10D39000A193B1938F01FB0181919191A191B191E1
:10D3A000BF01FA0181939193A193B193AF01F90168
:10D3B00081919191A191B1919F01F50181939193F7
:10D3C000A193B1935F01D394F4E0DF12D8CF80E052
:10D3D00090E8ABE3B5E480935B0F90935C0FA09370
:10D3E0005D0FB0935E0F8093570F9093580FA093EB
:10D3F000590FB0935A0F8093530F9093540FA093EB
:10D40000550FB093560F10925F0F1092600F10924D
:10D41000610F1092620F80E29EE4A0E0B0E0809382
:10D42000630F9093640FA093650FB093660F1092F3
:10D430003F0F1092400F1092410F1092420F80E068
:10D4400090E0A0E2B1E48093430F9093440FA09347
:10D45000450FB093460F8093470F9093480FA093CA
:10D46000490FB0934A0F8DEC9CECACECBEE380937B
:10D470004B0F90934C0FA0934D0FB0934E0F80E045
:10D4800090E0A0EAB0E480934F0F9093500FA093E8
:10D49000510FB093520F1092270610922806109247
:10D4A000290610922A061092230610922406109242
:10D4B00025061092260610921F0610922006109242
:10D4C0002106109222061092DF051092E0051092BC
:10D4D000E1051092E20584EB90E09093861580932D
:10D4E000851580EF90E0909388158093871586E4EA
:10D4F00090E090938215809381158EE690E0909352
:10D5000084158093831510927E1510927D151092CC
:10D51000801510927F1584EA90E7A3E8B1E4809328
:10D52000900290939102A0939202B093930281E3B0
:10D5300091E6A1E5BEE380938C0290938D02A093C7
:10D540008E02B0938F028DE692E1ACE9B3E4809352
:10D55000880290938902A0938A02B0938B02109262
:10D56000370680E090E0A0EEBFE38093290290931D
:10D570002A02A0932B02B0932C021092390210922F
:10D580000B0FEFDCE7EBFAE084918F010F5F1F4F89
:10D59000882321F00E94B311F801F6CFE6E3FFE003
:10D5A00084918F010F5F1F4F882321F00E94B311D8
:10D5B000F801F6CFE0960FB6F894DEBF0FBECDBFF0
:10D5C000DF91CF911F910F91FF90EF90DF90BF906F
:10D5D000AF900895AF92BF92CF92DF92EF92FF92F9
:10D5E0000F931F93CF93C82F811124C0E7EBFAE06C
:10D5F00084918F010F5F1F4F882321F00E94B31188
:10D60000F801F6CFE5E2FFE084918F010F5F1F4F35
:10D61000882321F00E94B311F801F6CFE7EBFAE07E
:10D6200084918F010F5F1F4F882321F00E94B31157
:10D63000F801F6CF4091970F5091980F6091990F94
:10D6400070919A0F8DE19FE00E94291540919B0FE8
:10D6500050919C0F60919D0F70919E0F8AE19FE009
:10D660000E94291540919F0F5091A00F6091A10F2A
:10D670007091A20F87E19FE00E9429154091A30FAE
:10D680005091A40F6091A50F7091A60F84E19FE0C7
:10D690000E9429158AE00E94B311C11124C0E7EB52
:10D6A000FAE084918F010F5F1F4F882321F00E94C1
:10D6B000B311F801F6CFE9EFFEE084918F010F5F1F
:10D6C0001F4F882321F00E94B311F801F6CFE7EB3A
:10D6D000FAE084918F010F5F1F4F882321F00E9491
:10D6E000B311F801F6CF4091A70F5091A80F6091A8
:10D6F000A90F7091AA0F80EF9EE00E94291540911A
:10D70000AB0F5091AC0F6091AD0F7091AE0F8DEEDD
:10D710009EE00E9429154091AF0F5091B00F60918B
:10D72000B10F7091B20F8AEE9EE00E9429154091D0
:10D73000B30F5091B40F6091B50F7091B60F87EE93
:10D740009EE00E9429158AE00E94B311C11124C0F5
:10D75000E7EBFAE084918F010F5F1F4F882321F0E0
:10D760000E94B311F801F6CFE8ECFEE084918F013E
:10D770000F5F1F4F882321F00E94B311F801F6CFED
:10D78000E7EBFAE084918F010F5F1F4F882321F0B0
:10D790000E94B311F801F6CF4091670F5091680FC6
:10D7A0006091690F70916A0F8FEB9EE00E94611586
:10D7B00040916B0F50916C0F60916D0F70916E0FD7
:10D7C0008CEB9EE00E94611540916F0F5091700F9D
:10D7D0006091710F7091720F89EB9EE00E9461154C
:10D7E0004091730F5091740F6091750F7091760F87
:10D7F00086EB9EE00E9461158AE00E94B311C11180
:10D8000024C0E7EBFAE084918F010F5F1F4F88235C
:10D8100021F00E94B311F801F6CFE3E8FEE0849115
:10D820008F010F5F1F4F882321F00E94B311F80171
:10D83000F6CFE7EBFAE084918F010F5F1F4F88234B
:10D8400021F00E94B311F801F6CF40915B0F509187
:10D850005C0F60915D0F70915E0F8AE79EE00E9401
:10D8600029154091570F5091580F6091590F7091A1
:10D870005A0F87E79EE00E9429154091530F50915F
:10D88000540F6091550F7091560F84E79EE00E94EF
:10D8900029158AE00E94B311C11124C0E7EBFAE018
:10D8A00084918F010F5F1F4F882321F00E94B311D5
:10D8B000F801F6CFE0ECFDE084918F010F5F1F4F80
:10D8C000882321F00E94B311F801F6CFE7EBFAE0CC
:10D8D00084918F010F5F1F4F882321F00E94B311A5
:10D8E000F801F6CF40915F0F5091600F6091610F8A
:10D8F0007091620F87EB9DE00E94291540913F0FC8
:10D900005091400F6091410F7091420F84EB9DE068
:10D910000E9429154091630F5091640F6091650F2B
:10D920007091660F81EB9DE00E9461154091430F5D
:10D930005091440F6091450F7091460F8EEA9DE023
:10D940000E9429154091470F5091480F6091490F4F
:10D9500070914A0F8BEA9DE00E94291540914B0F70
:10D9600050914C0F60914D0F70914E0F88EA9DE0E1
:10D970000E94291540914F0F5091500F6091510F07
:10D980007091520F85EA9DE00E9429158AE00E945D
:10D99000B311C11124C0E7EBFAE084918F010F5F4E
:10D9A0001F4F882321F00E94B311F801F6CFE3E95D
:10D9B000FDE084918F010F5F1F4F882321F00E94AB
:10D9C000B311F801F6CFE7EBFAE084918F010F5F16
:10D9D0001F4F882321F00E94B311F801F6CF409128
:10D9E0001F065091200660912106709122068AE858
:10D9F0009DE00E94291540912306509124066091D4
:10DA000025067091260687E89DE00E942915409121
:10DA10002706509128066091290670912A0684E80D
:10DA20009DE00E9429158AE00E94B311C11124C013
:10DA3000E7EBFAE084918F010F5F1F4F882321F0FD
:10DA40000E94B311F801F6CFE7E6FDE084918F0163
:10DA50000F5F1F4F882321F00E94B311F801F6CF0A
:10DA6000E7EBFAE084918F010F5F1F4F882321F0CD
:10DA70000E94B311F801F6CF4091DF055091E00507
:10DA80006091E1057091E2058EE59DE00E94291507
:10DA90008AE00E94B311C11118C0E7EBFAE084914B
:10DAA0008F010F5F1F4F882321F00E94B311F801EF
:10DAB000F6CFE1E4FDE084918F010F5F1F4F8823D3
:10DAC00099F00E94B311F801F6CFF5E8AF2EF5E119
:10DAD000BF2EA1E8CA2EA5E1DA2EBDE7EB2EB5E1F7
:10DAE000FB2E00E010E00CC0E7EBFAE084918F0120
:10DAF0000F5F1F4F882349F30E94B311F801F6CF3F
:10DB0000B80188E39DE00E94F614F50161917191DE
:10DB10005F0185E39DE00E94F614F6016191719129
:10DB20006F0182E39DE00E94F614F701619171910B
:10DB30007F018FE29DE00E94F6148AE00E94B311FB
:10DB40000F5F1F4F02301105D9F6C11124C0E7EB5A
:10DB5000FAE084918F010F5F1F4F882321F00E940C
:10DB6000B311F801F6CFE0E2FDE084918F010F5F81
:10DB70001F4F882321F00E94B311F801F6CFE7EB85
:10DB8000FAE084918F010F5F1F4F882321F00E94DC
:10DB9000B311F801F6CF409190025091910260913B
:10DBA00092027091930287E19DE00E9429152CE971
:10DBB00033E549E45EE360918C0270918D028091BF
:10DBC0008E0290918F020E94F5D0AB01BC0184E1DE
:10DBD0009DE00E9445152CE933E549E45EE3609140
:10DBE00088027091890280918A0290918B020E9432
:10DBF0002CD3AB01BC0181E19DE00E9445158AE078
:10DC00000E94B311C1112CC0E7EBFAE084918F019F
:10DC10000F5F1F4F882321F00E94B311F801F6CF48
:10DC2000EEEFFCE084918F010F5F1F4F882321F0FE
:10DC30000E94B311F801F6CF80913706882321F0B6
:10DC40008AE00E94B3113AC0E3EFFCE084918F01B7
:10DC50000F5F1F4F882391F10E94B311F801F6CF97
:10DC60004091290250912A0260912B0270912C025E
:10DC70008AEE9CE00E9429158AE00E94B3118091EF
:10DC80003706811127C0CC2319F0EFEDFCE00CC062
:10DC9000E7EBFAE084918F010F5F1F4F8823A9F310
:10DCA0000E94B311F801F6CF84918F010F5F1F4FCF
:10DCB000882381F00E94B311F801F6CFE7EBFAE078
:10DCC00084918F010F5F1F4F882351F20E94B3117F
:10DCD000F801F6CFCF911F910F91FF90EF90DF9059
:10DCE000CF90BF90AF900895CF92DF92EF92FF92C6
:10DCF0000F931F93CF93DF93CDB7DEB767970FB620
:10DD0000F894DEBF0FBECDBF84E690E09C8B8B8B7A
:10DD100044E0BE01675F7F4FCE014396F2D842E0F8
:10DD2000BE016F5E7F4FCE014396EBD843E050E0DB
:10DD3000BE01675F7F4F86E394E00E94D7D8892BAE
:10DD400009F076C11D821E821F8218861092050F6F
:10DD50001092040F40E167E97FE0CE014396D1D8ED
:10DD600040E167EA7FE0CE014396CBD840E167E629
:10DD70007FE0CE014396C5D844E06BE57FE0CE015D
:10DD80004396BFD844E067E57FE0CE014396B9D81B
:10DD900044E063E57FE0CE014396B3D844E06FE50D
:10DDA0007FE0CE014396ADD844E06FE37FE0CE0143
:10DDB0004396A7D844E063E67FE0CE014396A1D81E
:10DDC00040E163E47FE0CE0143969BD84CE06FE1F5
:10DDD00076E0CE01439695D81F8A1E8A1D8A41E0BF
:10DDE000BE01695E7F4FCE0143968BD844E0BE01F1
:10DDF0006B5F7F4FCE01439684D841E0BE016A5EDF
:10DE00007F4FCE0143967DD841E0BE016B5E7F4FD0
:10DE1000CE01439676D810E09E898D89212F30E07F
:10DE2000989FC0011124281739074CF444E0BE0123
:10DE30006B5F7F4FCE01439664D81F5FEDCF198291
:10DE40001A821B821C8244E0BE016F5F7F4FCE01AD
:10DE5000439657D844E06FED75E0CE01439651D814
:10DE60001D821E821F82188619E0115044E039F08D
:10DE7000BE016B5F7F4FCE01439643D8F6CF65E876
:10DE800075E1CE0143963DD844E061E875E1CE01ED
:10DE9000439637D844E06DE775E1CE01439631D81B
:10DEA00044E0BE016B5F7F4FCE0143962AD811112B
:10DEB0000EC0CD80DE80EF80F88420E030E84BE3B8
:10DEC00055E4C701B6010E94EED0811102C004E002
:10DED0001DC0C0929002D0929102E0929202F09204
:10DEE000930244E06CE872E0CE0143960AD844E025
:10DEF00068E872E0CE01439604D844E0BE016B5F4F
:10DF00007F4FCE0143960E9481670BC0015049F0BC
:10DF100044E0BE016B5F7F4FCE0143960E94816754
:10DF2000F5CF1F5F143009F0BBCF42E0BE01615F47
:10DF30007F4FCE0143960E948167115029F044E043
:10DF4000BE016B5F7F4FF5CF42E0BE01635F7F4F45
:10DF5000CE0143960E94816741E067E376E0CE01FF
:10DF600043960E94816744E0BE016B5F7F4FCE0104
:10DF700043960E94816711110CC08D819E81AF81F3
:10DF8000B8858093290290932A02A0932B02B09324
:10DF90002C021F5F143039F72091040F3091050FC8
:10DFA00089899A892817390759F50E94B167E7EBE3
:10DFB000FAE084918F010F5F1F4F811103C006E3C8
:10DFC00014E004C00E94B311F801F3CFF80181916D
:10DFD0008F01882319F00E94B311F8CF6B897C89D7
:10DFE0008CE79FE00E94F614E3E7FFE084918F0145
:10DFF0000F5F1F4F8823E9F00E94B311F801F6CF9D
:10E00000EDEBFAE084918F010F5F1F4F882321F021
:10E010000E94B311F801F6CFE9E5FFE084918F018A
:10E020000F5F1F4F882321F00E94B311F801F6CF34
:10E0300067D980E0CFDA67960FB6F894DEBF0FBEDF
:10E04000CDBFDF91CF911F910F91FF90EF90DF90A7
:10E05000CF900895CF93DF9300D000D0CDB7DEB737
:10E0600080E390E3A0E3B0E089839A83AB83BC8331
:10E0700084E190E09E838D8344E0BE016F5F7F4F1B
:10E08000CE0105960E942C6780917A0A90917B0AB6
:10E09000A0917C0AB0917D0A8093F00E9093F10ECE
:10E0A000A093F20EB093F30E8091F7079091F807CA
:10E0B000A091F907B091FA078093F40E9093F50EB2
:10E0C000A093F60EB093F70E8091F3079091F407AA
:10E0D000A091F507B091F6078093F80E9093F90E92
:10E0E000A093FA0EB093FB0E8091EF079091F0078A
:10E0F000A091F107B091F2078093FC0E9093FD0E72
:10E10000A093FE0EB093FF0E8091EB079091EC0769
:10E11000A091ED07B091EE078093000F9093010F4F
:10E12000A093020FB093030F44E060EF7EE0CE01B6
:10E1300005960E942C6744E064EF7EE0CE010596D0
:10E140000E942C6744E068EF7EE0CE0105960E94B5
:10E150002C6744E06CEF7EE0CE0105960E942C67B0
:10E1600044E060E07FE0CE0105960E942C67269691
:10E170000FB6F894DEBF0FBECDBFDF91CF910895EB
:10E18000CF93DF9300D000D0CDB7DEB784E190E02D
:10E190009E838D8344E0BE016F5F7F4FCE01059665
:10E1A0000E94816744E060EF7EE0CE0105960E9408
:10E1B000816744E064EF7EE0CE0105960E948167AE
:10E1C00044E068EF7EE0CE0105960E94816744E05E
:10E1D0006CEF7EE0CE0105960E94816744E060E02E
:10E1E0007FE0CE0105960E94816726960FB6F894CF
:10E1F000DEBF0FBECDBFDF91CF910895CF93DF93E8
:10E2000000D000D0CDB7DEB780E390E3A0E3B0E06C
:10E2100089839A83AB83BC8385E590E09E838D835D
:10E220008AE58093EF0E44E0BE016F5F7F4FCE0121
:10E2300005960E942C6741E06FEE7EE0CE010596C8
:10E240000E942C6726960FB6F894DEBF0FBECDBF96
:10E25000DF91CF910895CF93DF9300D000D0CDB759
:10E26000DEB785E590E09E838D8344E0BE016F5F5D
:10E270007F4FCE0105960E94816741E06FEE7EE000
:10E28000CE0105960E94816726960FB6F894DEBFF0
:10E290000FBECDBFDF91CF910895CF93DF9300D014
:10E2A00000D0CDB7DEB780E390E3A0E3B0E0898390
:10E2B0009A83AB83BC8382E390E09E838D838091BD
:10E2C000290C90912A0CA0912B0CB0912C0C8093CE
:10E2D000EB0E9093EC0EA093ED0EB093EE0E44E097
:10E2E000BE016F5F7F4FCE0105960E942C6744E010
:10E2F0006BEE7EE0CE0105960E942C6726960FB647
:10E30000F894DEBF0FBECDBFDF91CF910895CF93BC
:10E31000DF9300D000D0CDB7DEB782E390E09E83DC
:10E320008D8344E0BE016F5F7F4FCE0105960E9452
:10E33000816744E06BEE7EE0CE0105960E94816726
:10E3400026960FB6F894DEBF0FBECDBFDF91CF91FA
:10E3500008956D98759AEAE0F1E080818F77808367
:10E360009FB7F894EBE0F1E08081806880839FBFE5
:10E3700053985B9AEAE0F1E080818F7B80839FB7BE
:10E38000F894EBE0F1E08081806480839FBF089582
:10E39000CF93DF93EFEEFFE08491EF012196882386
:10E3A00021F00E94B311FE01F7CFE7EEFFE0849168
:10E3B000EF012196882321F00E94B311FE01F7CFCF
:10E3C000659903C0CAE3D4E002C0C4E4D4E08991F3
:10E3D000882319F00E94B311FACF8AE00E94B3118A
:10E3E000EFEDFFE08491EF012196882321F00E9458
:10E3F000B311FE01F7CF8091090187FD03C0CAE385
:10E40000D4E002C0C4E4D4E08991882319F00E94CA
:10E41000B311FACF8AE00E94B311E7EDFFE08491D7
:10E42000EF012196882321F00E94B311FE01F7CF5E
:10E430004B9903C0CAE3D4E002C0C4E4D4E089919C
:10E44000882319F00E94B311FACF8AE00E94B31119
:10E45000EEECFFE08491EF012196882321F00E94E9
:10E46000B311FE01F7CF8091090186FD03C0CAE315
:10E47000D4E002C0C4E4D4E08991882319F00E945A
:10E48000B311FACF8AE0DF91CF910C94B311409190
:10E49000060F5091070F2091080F3091090F42236A
:10E4A000532321E030E002C0220F331F8A95E2F7A8
:10E4B0002423352371E0232B09F470E081E090E000
:10E4C00002C0880F991F6A95E2F784239523892B50
:10E4D00011F022E001C020E0272B21F1E0918E1401
:10E4E000F0918F1482859385A485B5851816190639
:10E4F0001A061B06BCF480910A0F846080930A0FF1
:10E5000080918D14882311F0233061F482899389DE
:10E51000A489B5898093741490937514A09376148C
:10E52000B093771408950F931F93CF93DF93809147
:10E530008C1480FF34C04CB18091080F9091090F6A
:10E5400042954695477051E04527242F217030E0D1
:10E550008E7F822B932B9093090F8093080F20912D
:10E56000060F3091070F2170332728233923232BDF
:10E57000B1F0E0918E14F0918F1482819381A48187
:10E58000B581181619061A061B064CF480910A0F5D
:10E59000816080930A0F80E090E00E94228D80913C
:10E5A0008C1481FF38C0809109012091080F3091AF
:10E5B000090F992787FD909580959095990F880B65
:10E5C000982F8227932782709927822793279093E9
:10E5D000090F8093080F2091060F3091070F2270CA
:10E5E000332728233923232BB1F0E0918E14F091A7
:10E5F0008F1486819781A085B185181619061A0691
:10E600001B064CF480910A0F826080930A0F81E010
:10E6100090E00E94228D80918C1482FF37C029B136
:10E620008091080F9091090F26952695269531E047
:10E630002327022F017010E0119501951109082779
:10E64000192704701127082719271093090F009321
:10E65000080F80910901829586958695837083279E
:10E660008170C82F80E0D82FD195C195D109C027DE
:10E67000D127C078DD27C027D127D093090FC093B9
:10E68000080F67E070E082E090E001DF8091080F02
:10E690009091090F9093070F8093060FDF91CF9110
:10E6A0001F910F910895CF92DF92EF92FF920F93F7
:10E6B0001F93CF93DF93CAE3D2E00AE412E098EE0F
:10E6C000E92E93E0F92E69917991C7010E9419D43E
:10E6D0006B01F801619171918F019601442737FD1B
:10E6E0004095542F8FE10E9472CCB601660F771FC0
:10E6F000882777FD8095982F0E9453C888E00E9454
:10E7000093CFF2E0CA34DF07F1F6DF91CF911F918A
:10E710000F91FF90EF90DF90CF900895CF92DF920E
:10E72000EF92FF920F931F93CF93DF93CAE5D2E04E
:10E7300002E612E058EEE52E53E0F52E699179914C
:10E74000C7010E9419D46B01F801619171918F0189
:10E750009601442737FD4095542F8FE10E9472CCDB
:10E76000B601660F771F882777FD8095982F0E9446
:10E7700053C888E00E9493CFF2E0C236DF07F1F67B
:10E78000DF91CF911F910F91FF90EF90DF90CF908D
:10E7900008951092B70F1092B80F80E1EEE2FFE0FB
:10E7A000DF01982F1D929A95E9F7EAE1FFE0DF017A
:10E7B0001D928A95E9F71092160F1092170F10927A
:10E7C000180F1092190F08952F923F924F925F9257
:10E7D0006F927F928F929F92AF92BF92CF92DF9271
:10E7E000EF92FF920F931F93CF93DF93CDB7DEB7D6
:10E7F00068970FB6F894DEBF0FBECDBF1C015B015A
:10E800008A01DC01D7966D917D918D919C91DA976B
:10E810000E948ED16B017C01F50120813181428102
:10E8200053810E942CD30E94DBD00E9462D1698761
:10E830007A878B879C87D8012D913D914D915C9172
:10E84000C701B6010E942CD30E94DBD00E9462D186
:10E850006D877E878F87988B29853A854B855C8568
:10E86000283731054105510540F488E790E0A0E0E4
:10E87000B0E089879A87AB87BC872D853E854F8519
:10E880005889283731054105510540F488E790E063
:10E89000A0E0B0E08D879E87AF87B88B91012D5B9C
:10E8A0003F4FD9018D919D910D90BC91A02D8D83ED
:10E8B0009E83AF83B887BC01CD010E9490D169834C
:10E8C0007A838B839C8369857A858B859C850E945E
:10E8D0008ED1698B7A8B8B8B9C8B20E030E0A901E9
:10E8E00069817A818B819C810E94EED0882339F1E5
:10E8F000A7019601C701B6010E942CD34B015C0110
:10E9000029893A894B895C89CA01B9010E942CD3B3
:10E910009B01AC01C501B4010E9414D04B015C0104
:10E9200029813A814B815C81CA01B9010E9415D0CD
:10E930009B01AC01C501B4010E94F5D003C060E0A9
:10E9400070E0CB010E94DBD00E945DD12B013C0125
:10E950006D817E818F819885909580957095619568
:10E960007F4F8F4F9F4F0E9490D14B015C016D856F
:10E970007E858F8598890E948ED16D837E838F835B
:10E98000988720E030E0A901C501B4010E94EED0D3
:10E99000882349F12D813E814F815885CA01B901F3
:10E9A0000E942CD36D8B7E8B8F8B988FA701960145
:10E9B000C701B6010E942CD39B01AC016D897E89F1
:10E9C0008F89988D0E9414D06B017C01A501940160
:10E9D000C501B4010E9415D09B01AC01C701B6016D
:10E9E0000E94F5D003C060E070E0CB010E94CBD163
:10E9F000F10182889388A488B58875016401C418E0
:10EA0000D508E608F7080E945DD1C61AD70AE80AB9
:10EA1000F90AF7FE6BC020E030E0A90169817A8134
:10EA20008B819C810E94EED0882309F447C0298104
:10EA30003A814B815C81CA01B9010E9415D06B01FA
:10EA40007C01C501B4010E948ED19B01AC01C701BC
:10EA5000B6010E942CD36B017C0129893A894B892C
:10EA60005C89CA01B9010E942CD39B01AC01C7018A
:10EA7000B6010E9414D06B017C012D813E814F8133
:10EA80005885CA01B9010E942CD39B01AC01C70172
:10EA9000B6010E9415D06B017C0120E030E040E817
:10EAA00050E469817A818B819C810E942CD39B01E7
:10EAB000AC01C701B6010E94F5D003C060E070E070
:10EAC000CB010E94DBD00E945DD12B013C0197FF5E
:10EAD00003C0412C512C3201481459046A047B04B0
:10EAE00010F024013501C12CD12C76018FB7F89498
:10EAF000D1019C9193FD22C0F101468A578A608E14
:10EB0000718EC40CD51CE61CF71C5A96CD92DD9272
:10EB1000ED92FC925D9729853A854B855C85DB9665
:10EB20002D933D934D935C93DE97FF962D853E8507
:10EB30004F85588920833183428353838FBF6896E2
:10EB40000FB6F894DEBF0FBECDBFDF91CF911F91FE
:10EB50000F91FF90EF90DF90CF90BF90AF909F907C
:10EB60008F907F906F905F904F903F902F9008957F
:10EB70004F925F926F927F929F92AF92BF92CF928D
:10EB8000DF92EF92FF920F931F93CF93DF93EC01ED
:10EB90007B01009709F45EC06115710509F45AC044
:10EBA0009BA4BCA40DA51EA5292D3B2DA8016FA1DA
:10EBB00078A589A59AA50E94EED0882309F44AC0B9
:10EBC000A880A1FC3DC0F70147A050A461A472A495
:10EBD000A3019201692D7B2DC8010E94EED0181669
:10EBE0007CF5A3019201C301B2010E942CD36B01F9
:10EBF0007C018BA99CA9ADA9BEA9BC01CD019058EF
:10EC00009B01AC010E9415D02FA538A949A95AA98A
:10EC10000E942CD39B01AC01C701B6010E9414D005
:10EC20000E9499D36B017C019B01AC01692D7B2D66
:10EC3000C8010E94EED087FD03C09C2CBD2C87012B
:10EC4000492D5B2DB8014FA358A769A77AA78A2D34
:10EC500081608883DF91CF911F910F91FF90EF909A
:10EC6000DF90CF90BF90AF909F907F906F905F901C
:10EC70004F900895CF92DF92EF92FF920F931F93E0
:10EC8000CF93DF931F92CDB7DEB78091B80F9091ED
:10EC9000B70F891B8F70843018F1F090B70F209157
:10ECA000B80F23502F7060E070E0C12CD12C89E4A4
:10ECB000E82E2F15A9F0C114D10421F0F6018081AE
:10ECC00082FD0EC021502F70E29E80011124075456
:10ECD000104FC60129834CDFB60168012981E9CFB5
:10ECE0000F90DF91CF911F910F91FF90EF90DF90E8
:10ECF000CF9008954F925F926F927F92AF92BF92A2
:10ED0000CF92DF92EF92FF920F931F93CF93DF93F7
:10ED10008C01EB01009709F454C0FC01808181FD56
:10ED200050C047A050A461A472A4AFA0B8A4C9A4C5
:10ED3000DAA49501A601C301B2010E94EED087FFBB
:10ED400040C0A3019201C301B2010E942CD32B0148
:10ED50003C01F80183A994A9A5A9B6A9BC01CD01DC
:10ED600090589B01AC010E9415D0F80127A530A94D
:10ED700041A952A90E942CD39B01AC01C301B2014D
:10ED80000E9414D00E9499D37B018C019B01AC019D
:10ED9000B501C6010E94EED087FF02C07501860151
:10EDA0009701A801B501C6010E94EED0882349F061
:10EDB000A701B8014FA358A769A77AA788818160E6
:10EDC0008883DF91CF911F910F91FF90EF90DF909B
:10EDD000CF90BF90AF907F906F905F904F900895CD
:10EDE000EF92FF920F931F93CF93DF931091B70F82
:10EDF000F12C00E080E090E029E4E22E2091B80FB1
:10EE0000121779F0E19EE0011124C754D04F6F2D05
:10EE1000702F70DF1F5F1F708F2D902FFC2E0D2F16
:10EE2000EDCF6F2D702FDF91CF911F910F91FF903C
:10EE3000EF9060CF8F929F92AF92BF92CF92DF926E
:10EE4000EF92FF920F931F93CF93DF93CDB7DEB76F
:10EE500028970FB6F894DEBF0FBECDBF9090B70FC6
:10EE600000E010E039E4832E892D992787FD9095E5
:10EE70002091B80F30E08217930709F445C0889EAF
:10EE80005001899EB00C1124C5018754904F5C013C
:10EE90000115110599F1F801808180FD04C0F5018B
:10EEA000808180FF2BC0F801C3A0D4A0E5A0F6A00C
:10EEB000A7019601F50167A170A581A592A50E9401
:10EEC000F5D069837A838B839C83A7019601F8012F
:10EED00067A170A581A592A50E94F5D06D837E8360
:10EEE0008F839887AE014F5F5F4FBE016B5F7F4F8F
:10EEF000C8016ADCF80180818E7F80839394F92DAC
:10EF0000FF709F2E8501B0CF0115110551F1F80159
:10EF1000C3A0D4A0E5A0F6A0A70196016DEC7CECFF
:10EF20008CE49DE30E94F5D069837A838B839C8374
:10EF3000A7019601F80167A170A581A592A50E947D
:10EF4000F5D06D837E838F839887AE014F5F5F4FCF
:10EF5000BE016B5F7F4FC80137DCF80180818E7F77
:10EF6000808328960FB6F894DEBF0FBECDBFDF9129
:10EF7000CF911F910F91FF90EF90DF90CF90BF90B6
:10EF8000AF909F908F90089575DE2ADF53CF4F92F8
:10EF90005F926F927F928F929F92AF92BF92CF9229
:10EFA000DF92EF92FF920F931F93CF93DF938091A5
:10EFB0003E0F882309F4EBC000916E0210916F029E
:10EFC000D0917002C09171026091D5147091D614E5
:10EFD000882777FD8095982F0E9490D120E030E01F
:10EFE00040E050E40E9415D098014D2F5C2F0E9404
:10EFF000EED087FDCCC05090B70F612C712C812CC6
:10F00000912C49E4442E8091B80F581609F44EC053
:10F01000459C50011124C5018754904F5C01FC01AF
:10F0200082819381A481B581892B8A2B8B2B81F4DA
:10F0300086819781A085B185892B8A2B8B2B41F402
:10F0400082859385A485B585892B8A2B8B2B49F1E5
:10F05000F50166857785808991890E9490D16B0141
:10F060007C01F50162897389848995890E948ED11A
:10F070009B01AC01C701B6010E94F5D0F50123A1A7
:10F0800034A145A156A10E942CD36B017C019B01A8
:10F09000AC01B301C4010E94EED087FF02C036016B
:10F0A00047015394F52DFF705F2EADCF20916A027A
:10F0B00030916B0240916C0250916D02B301C4011A
:10F0C0000E942CD39B01AC01B8018D2F9C2F0E9474
:10F0D00015D06B017C0198014D2F5C2F0E94EED062
:10F0E00087FD14C00091720210917302D0917402D6
:10F0F000C091750298014D2F5C2FB601C7010E9487
:10F10000F1D218161CF08601DE2DCF2D8090110F44
:10F110009090120FA090130FB090140F98014D2FE4
:10F120005C2FC501B4010E94F1D21816E4F420E06E
:10F1300037ED43EA5CE3B8018D2F9C2F0E942CD35E
:10F140006B017C0128E431EE4AE75FE3C501B401BD
:10F150000E942CD39B01AC01C701B6010E9415D0BF
:10F160008B01D82FC92FC801AD2FBC2F8093110F51
:10F170009093120FA093130FB093140FB8018D2F1B
:10F180009C2F0E945DD17093D6146093D514DF91AB
:10F19000CF911F910F91FF90EF90DF90CF90BF9094
:10F1A000AF909F908F907F906F905F904F90089559
:10F1B00080911D062091B80F9091B70F291799F0F3
:10F1C000E091B70F89E4E89FF0011124E050F04F7F
:10F1D00090818091B70F2091B80F821719F08F5F3F
:10F1E0008F70F9CF892F8093CF14D1CE2F923F9279
:10F1F0004F925F926F927F928F929F92AF92BF9247
:10F20000CF92DF92EF92FF920F931F93CF93DF93F2
:10F21000CDB7DEB7C557D1090FB6F894DEBF0FBE24
:10F22000CDBF5B014A013901EFAEFBAA24960FAFB7
:10F23000249728961FAF28973C2C2091970F309148
:10F24000980F4091990F50919A0FDC016D917D912B
:10F250008D919C910E942CD30E94FCD2AE966CAFF3
:10F260007DAF8EAF9FAFAE9720919B0F30919C0FDB
:10F2700040919D0F50919E0FF501608171818281B7
:10F2800093810E942CD30E94FCD2E2966CAF7DAF9A
:10F290008EAF9FAFE29720919F0F3091A00F4091CA
:10F2A000A10F5091A20FD4016D917D918D919C91F0
:10F2B0000E942CD30E94FCD2E6966CAF7DAF8EAF3D
:10F2C0009FAFE6972091A30F3091A40F4091A50F17
:10F2D0005091A60FF30160817181828193810E9418
:10F2E0002CD30E94FCD268966CAF7DAF8EAF9FAFDF
:10F2F000689780912E0F90912F0FA091300FB091B1
:10F30000310FAE96CCACDDACEEACFFACAE97C81A0C
:10F31000D90AEA0AFB0A8091320F9091330FA0912B
:10F32000340FB091350FE2968CAC9DACAEACBFAC57
:10F33000E297881A990AAA0ABB0A8091360F90911F
:10F34000370FA091380FB091390FE6960CAD1DAD77
:10F350002EAD3FADE697081B190B2A0B3B0B0FA7F1
:10F3600018AB29AB3AAB8091FB0783FF0EC06896C0
:10F370002CAD3DAD4EAD5FAD689720933A0F309305
:10F380003B0F40933C0F50933D0F80913A0F90916B
:10F390003B0FA0913C0FB0913D0F68964CAC5DAC1B
:10F3A0006EAC7FAC6897481A590A6A0A7B0A09F45E
:10F3B000B4C08091CE1481115EC02091840230913E
:10F3C000850240918602509187026091DD14709110
:10F3D000DE148091DF149091E0140E94EED087FF3C
:10F3E0004AC068968CAD9DADAEADBFAD68978093B9
:10F3F0003A0F90933B0FA0933C0FB0933D0FE7EB78
:10F40000FAE084913F019FEF691A790A882321F07D
:10F410000E94B311F301F5CFECE2F0E184913F01DA
:10F42000AFEF6A1A7A0A882321F00E94B311F30120
:10F43000F5CFE8E2F0E164913F01662369F07727B8
:10F4400067FD70958FE29CE00E94CA13BFEF6B1AB4
:10F450007B0AF3016491F1CF6DE070E08FE29CE0F4
:10F460000E94CA136AE070E08FE29CE00E94CA1317
:10F47000412C512C32014BA65CA66DA67EA677FED0
:10F480000BC000271127980104191509260937090F
:10F490000BA71CA72DA73EA76091A30F7091A40FE7
:10F4A0008091A50F9091A60F0E945DD19B01AC01A8
:10F4B000A8ECB0E00E9470D42BA53CA54DA55EA59C
:10F4C00062177307840795075CF568968CAD9DAD50
:10F4D000AEADBFAD689780933A0F90933B0FA0936A
:10F4E0003C0FB0933D0FE7EBFAE084913F019FEFB3
:10F4F000691A790A882321F00E94B311F301F5CF2C
:10F50000E9E0F0E184913F01AFEF6A1A7A0A8823BB
:10F5100021F00E94B311F301F5CF412C512C32019F
:10F52000D701C6018827B7FD83959927AA27BB274E
:10F53000182FB7FC12602FA538A949A95AA957FD61
:10F54000146077FC1860432D50E02D965FAF4EAFEE
:10F550002D97C301B2010E9490D12D96EEADFFAD63
:10F560002D97EE0FFF1FEE0FFF1FEB5DFD4F20816C
:10F570003181428153810E942CD32B013C012D9675
:10F58000EEADFFAD2D97EE0FFF1FE35DFD4F6081E8
:10F590007181882777FD8095982F0E9490D19B01DB
:10F5A000AC01C301B2010E942CD32AE037ED43E243
:10F5B0005CE30E942CD36BAF7CAF8DAF9EAF20E09D
:10F5C00030E0A9010E94F1D218165CF420E030E08E
:10F5D00040E05FE36BAD7CAD8DAD9EAD0E9415D07C
:10F5E0000AC02BAD3CAD4DAD5EAD60E070E080E09B
:10F5F0009FE30E9414D00E945DD16FAB78AF89AFBA
:10F600009AAF0091B80F0F5F0F7060960FAF6097C1
:10F61000602E772467FC70948091B70F90E0861578
:10F62000970519F40E94E239F7CF8091B80F49E4A9
:10F63000849F900111242754304F3CA72BA7D90158
:10F640001C9292961C9326013701F7FE07C04424B2
:10F65000552432014C185D086E087F08EBA5FCA507
:10F660004282538264827582B501A401B7FE07C04D
:10F6700044275527BA01481959096A097B09ABA5DE
:10F68000BCA516964D935D936D937C9319978FA5AA
:10F6900098A9A9A9BAA9B7FF07C0B095A095909558
:10F6A00081959F4FAF4FBF4FEBA5FCA582879387F6
:10F6B000A487B5870FA918AD29AD3AAD068717877E
:10F6C000208B318B441555056605770514F4B3017D
:10F6D000A201481759076A077B0714F4AC01BD0162
:10F6E0000FA918AD29AD3AAD40175107620773074E
:10F6F00014F4B901A801ABA5BCA552964D935D9336
:10F700006D937C935597463051056105710510F452
:10F710000C949A8380911D0690911E06FD01E95B71
:10F72000FF4F9183808311963C92452846284728B5
:10F7300009F05F98EBA5FCA586819781A085B1852E
:10F74000892B8A2B8B2B11F08A984798EBA5FCA567
:10F7500082859385A485B585892B8A2B8B2B49F0CF
:10F760009FB7F894809108018E7F809308019FBF16
:10F7700047980FA918AD29AD3AAD012B022B032BE9
:10F78000B1F08091150F882319F081508093150FE7
:10F79000311004C0129880E28093150F30905F0FF3
:10F7A0002090600F0091610F1091620F08C030909F
:10F7B0003F0F2090400F0091410F1091420F232DD9
:10F7C000322DA8016FAD7BA924968FAD2497289682
:10F7D0009FAD28970E94EED087FFA3C7C701B6014F
:10F7E0000E9490D12091870F3091880F4091890F0E
:10F7F00050918A0F0E942CD32B013C01698B7A8B8C
:10F800008B8B9C8BC501B4010E9490D120918B0FF2
:10F8100030918C0F40918D0F50918E0F0E942CD300
:10F820004B015C016D8B7E8B8F8B988F6FA578A9B8
:10F8300089A99AA90E9490D120918F0F3091900FA1
:10F840004091910F5091920F0E942CD36B017C013B
:10F85000698F7A8F8B8F9C8F2091930F3091940FAB
:10F860004091950F5091960F6BAD7CAD8DAD9EADD7
:10F870000E942CD36D8F7E8F8F8F98A3ABA5BCA5D4
:10F8800012962D913D914D915C9115972FA738AB14
:10F8900049AB5AAB263031054105510504F51696A2
:10F8A0002D913D914D915C9119972630310541057F
:10F8B0005105ACF41A962D913D914D915C911D9797
:10F8C000263031054105510554F4DC01CB01BF77E9
:10F8D000EBA5FCA587A790ABA1ABB2AB2CC0A30155
:10F8E0009201C301B2010E942CD32B013C01A5015E
:10F8F0009401C501B4010E942CD39B01AC01C3014A
:10F90000B2010E9415D04B015C01A7019601C7010D
:10F91000B6010E942CD39B01AC01C501B4010E9429
:10F9200015D00E9499D3ABA5BCA59F966D937D93EE
:10F930008D939C93D297ABA5BCA59F962D913D919D
:10F940004D915C91D297A2962CAF3DAF4EAF5FAF79
:10F95000A29760E070E080E89FE30E94F5D02796D0
:10F960006CAF7DAF8EAF9FAF27979B01AC01632D2E
:10F97000722DC8010E942CD32B013C011091B80FAD
:10F980008091B70F181B1F70E12FF0E02F96FFAF8B
:10F99000EEAF2F97A301920160E074E284E799E44F
:10F9A0000E94F5D00E94FCD26B017C012F968EAD97
:10F9B0009FAD2F970297069798F58091630F9091CE
:10F9C000640FA091650FB091660FC816D906EA06BC
:10F9D000FB0630F5BC01CD016C197D098E099F092C
:10F9E000660F771F881F991F212F30E040E050E0FD
:10F9F0000E942CD4CA01B9010E948ED10E94FCD26F
:10FA00006C0D7D1D8E1D9F1D0E948ED19B01AC0132
:10FA100060E074E284E799E40E94F5D02B013C0198
:10FA2000A3019201A2966CAD7DAD8EAD9FADA29764
:10FA30000E942CD32B966CAF7DAF8EAF9FAF2B97D0
:10FA4000ABA5BCA593966D937D938D939C93969750
:10FA500052960D911D912D913C9155970BAF1CAF76
:10FA60002DAF3EAFC901B8010E948ED123966CAF75
:10FA70007DAF8EAF9FAF2397A30192010E942CD33D
:10FA80000E94DBD00E9462D16B017C01EBA5FCA53A
:10FA900067AB70AF81AF92AF8E010F5E1F4F1CAB93
:10FAA0000BAB07EA1FE06E961FAF0EAF6E978E018D
:10FAB0000F5D1F4F1AA709A7005211096A961FAFC1
:10FAC0000EAF6A97212C312C00E81FE3ABA9BCA92B
:10FAD0006D917D918D919D91BCABABABA3019201DA
:10FAE0000E942CD36A96EEADFFAD6A976193719335
:10FAF000819391936A96FFAFEEAF6A979B01AC0139
:10FB00005F7764962CAF3DAF4EAF5FAF64976E9654
:10FB1000AEADBFAD6E978D909D90AD90BD906E9641
:10FB2000BFAFAEAF6E97A501940164966CAD7DAD8D
:10FB30008EAD9FAD64970E94F1D21816E4F46496DE
:10FB40002CAD3DAD4EAD5FAD6497C501B4010E94D3
:10FB5000F5D0B62EA72E982E892E262F372F482F78
:10FB6000592FB101C8010E94F1D2181624F42B2C90
:10FB70003A2C092D182DEBA9FCA929A53AA5E217C5
:10FB8000F30709F0A3CF20E030E040E85FE3B101E4
:10FB9000C8010E94EED087FF3CC04E0131E1830EC8
:10FBA000911CAE014F5F5F4F5A019101A801D50131
:10FBB0006D917D918D919C910E942CD3F501619363
:10FBC0007193819391935F01E815F90571F79101A4
:10FBD000A8012B966CAD7DAD8EAD9FAD2B970E948D
:10FBE0002CD3ABA5BCA593966D937D938D939C93DD
:10FBF0009697C701B6010E948ED19101A8010E947B
:10FC00002CD30E9462D1EBA5FCA567AB70AF81AF8E
:10FC100092AF27962CAD3DAD4EAD5FAD27972396A5
:10FC20006CAD7DAD8EAD9FAD23970E942CD32796F2
:10FC30006CAF7DAF8EAF9FAF2797ABA5BCA51696D7
:10FC40000D911D912D913C9119970BAB1CAB2DABD8
:10FC50003EAB1A964D905D906D907C901D970FA5D0
:10FC600018A929A93AA9012B022B032BD1F42BA9FE
:10FC70003CA94DA95EA9232B242B252B91F44114DB
:10FC800051046104710469F42091570F3091580FA9
:10FC90004091590F50915A0F0E942CD30E94DBD0F3
:10FCA00026C28FA998ADA9ADBAAD892B8A2B8B2B13
:10FCB00049F060915B0F70915C0F80915D0F9091A6
:10FCC0005E0F08C06091530F7091540F8091550FD3
:10FCD0009091560F27962CAD3DAD4EAD5FAD279759
:10FCE0000E942CD30E94DBD00E9462D16B017C0168
:10FCF00080912A0F90912B0FA0912C0FB0912D0F76
:10FD0000EBA5FCA506851785208931890FAB18AFB7
:10FD100029AF3AAF0BAD1CAD2DAD3EAD80179107AD
:10FD2000A207B30708F4D3C02FA538A949A95AA937
:10FD3000232B242B252B61F12091770F3091780F05
:10FD40004091790F50917A0F2C153D054E055F05B6
:10FD5000F8F46BAD7CAD8DAD9EAD0E94F6D34B013A
:10FD60005C01A70196016FA578A989A99AA90E94AB
:10FD7000F6D386169706A806B90650F4C501B40155
:10FD80002FA538A949A95AA90E942CD469017A0142
:10FD90008BA99CA9ADA9BEA9892B8A2B8B2B61F1BC
:10FDA00020917B0F30917C0F40917D0F50917E0F01
:10FDB0002C153D054E055F05F8F46BAD7CAD8DADA2
:10FDC0009EAD0E94F6D34B015C01A70196016BA981
:10FDD0007CA98DA99EA90E94F6D386169706A8062F
:10FDE000B90650F4C501B4012BA93CA94DA95EA9DF
:10FDF0000E942CD469017A014114510461047104F8
:10FE000041F120917F0F3091800F4091810F5091EF
:10FE1000820F2C153D054E055F05D8F46BAD7CAD0A
:10FE20008DAD9EAD0E94F6D34B015C01A7019601FA
:10FE3000C301B2010E94F6D386169706A806B9063A
:10FE400040F4C501B401A30192010E942CD46901C0
:10FE50007A010FA918AD29AD3AAD012B022B032B66
:10FE600009F449C12D96EEADFFAD2D97EE0FFF1FA2
:10FE7000EE0FFF1FED57F04F2081318142815381FA
:10FE80002C153D054E055F0508F035C16BAD7CAD09
:10FE90008DAD9EAD0E94F6D34B015C01A70196018A
:10FEA0006FA978AD89AD9AAD0E94F6D386169706F4
:10FEB000A806B90608F01FC1C501B4012FA938ADC5
:10FEC00049AD5AAD0E942CD469017A0114C12FA505
:10FED00038A949A95AA9232B242B252B09F43FC063
:10FEE0006091770F7091780F8091790F90917A0FD0
:10FEF0006C157D058E059F0590F50E948ED1239689
:10FF00002CAD3DAD4EAD5FAD23970E942CD34B0180
:10FF10005C016FA578A989A99AA90E9490D16FA7C1
:10FF200078AB89AB9AABC701B6010E948ED12FA5E1
:10FF300038A949A95AA90E942CD3A50194010E946D
:10FF4000F1D2181664F42FA538A949A95AA9C501F8
:10FF5000B4010E94F5D00E9462D16B017C018BA993
:10FF60009CA9ADA9BEA9892B8A2B8B2B09F43FC074
:10FF700060917B0F70917C0F80917D0F90917E0F2F
:10FF80006C157D058E059F0590F50E948ED12396F8
:10FF90002CAD3DAD4EAD5FAD23970E942CD34B01F0
:10FFA0005C016BA97CA98DA99EA90E9490D16FA725
:10FFB00078AB89AB9AABC701B6010E948ED12FA551
:10FFC00038A949A95AA90E942CD3A50194010E94DD
:10FFD000F1D2181664F42FA538A949A95AA9C50168
:10FFE000B4010E94F5D00E9462D16B017C014114E2
:10FFF000510461047104B9F160917F0F7091800F19
:020000021000EC
:100000008091810F9091820F6C157D058E059F0563
:1000100050F50E948ED123962CAD3DAD4EAD5FAD17
:1000200023970E942CD34B015C01C301B2010E94B3
:1000300090D12B013C01C701B6010E948ED1A301D2
:1000400092010E942CD3A50194010E94F1D21816AE
:1000500054F4A3019201C501B4010E94F5D00E949D
:1000600062D16B017C010FA918AD29AD3AAD012B0E
:10007000022B032B09F43FC02D96EEADFFAD2D975B
:10008000EE0FFF1FEE0FFF1FED57F04F60817181E4
:10009000828193816C157D058E059F0560F50E9418
:1000A0008ED123962CAD3DAD4EAD5FAD23970E9412
:1000B0002CD34B015C016FA978AD89AD9AAD0E943C
:1000C00090D12B013C01C701B6010E948ED1A30142
:1000D00092010E942CD3A50194010E94F1D218161E
:1000E00054F4A3019201C501B4010E94F5D00E940D
:1000F00062D16B017C01EBA5FCA5ED5BFF4FC082DB
:10010000D182E282F382C701B6010E948ED16B01D7
:100110007C0127962CAD3DAD4EAD5FAD27970E947B
:10012000F5D06C966CAF7DAF8EAF9FAF6C97ABA5E3
:10013000BCA5D3966D937D938D939C93D69720E029
:1001400030E040E85BE4C701B6010E942CD320E018
:1001500034E244EF59E40E94F5D00E945DD1EBA552
:10016000FCA5668F778F80A391A303A10FA714A18D
:100170001FAB05A10BAF16A11FAF2E0121E1420E4F
:10018000511C63E4262E6FE0362EAE014F5F5F4FA9
:100190003A010FA50BAB1FA92C961FAF2C970BADE7
:1001A00024960FAF24971FAD28961FAF289710E015
:1001B000D3018D909D90AD90BD903D01E894B7F82E
:1001C000F101C190D190E190F1901F01A70196013A
:1001D000C501B4010E94F1D218160CF04FC01123D2
:1001E00009F441C02BA92C963FAD2C9724964FAD16
:1001F000249728965FAD2897C501B4010E942CD39F
:100200004B015C012FA53FA94BAD5FADC701B60106
:100210000E942CD36B017C019B01AC01C501B40190
:100220000E94F1D2181654F5A5019401C701B60138
:100230000E94F5D09B01AC016BA92C967FAD2C9749
:1002400024968FAD249728969FAD28970E942CD393
:100250006BAB2C967FAF2C9724968FAF2497289664
:100260009FAF28970BC0CBAA2C96DFAE2C97249675
:10027000EFAE24972896FFAE289711E0641475041A
:1002800009F096CF2F960EAD1FAD2F9702301105B6
:100290000CF458C12090160F3090170F1091180FC2
:1002A0000091190F27E137EB41ED58E3B101812FA0
:1002B000902F0E94F1D218160CF044C121E06D96E7
:1002C0002FAF6D972FA53FA94BAD5FADB101812F2A
:1002D000902F0E94F1D218169CF06D961FAE6D976C
:1002E0002FA53FA94BAD5FADB101812F902F0E948B
:1002F000F5D0A6966CAF7DAF8EAF9FAFA69713C01B
:100300009101412F502F6FA57FA98BAD9FAD0E940A
:10031000F5D0A6966CAF7DAF8EAF9FAFA6972FA4FA
:100320003FA81BAD0FAD4AE15FE062965FAF4EAFF5
:10033000629783E49FE0A8969FAF8EAFA897DE01F7
:100340001196AA96BFAFAEAFAA97412C512C50E898
:10035000652E5FE3752E2E961FAE2E976296EEAD3C
:10036000FFAD629781909190A190B1906296FFAF9E
:10037000EEAF6297AA96AEADBFADAA97CD90DD90D5
:10038000ED90FD90AA96BFAFAEAFAA976D96BFADA8
:100390006D97BB2361F0A6962CAD3DAD4EAD5FAD24
:1003A000A697C501B4010E942CD34B015C012E9687
:1003B000EFAD2E97EE2381F0A3019201C501B401A8
:1003C0000E942CD34B015C01A3019201C701B6012D
:1003D0000E942CD36B017C01A7019601C501B401D9
:1003E0000E94F1D220E030E0A9011816CCF4C70138
:1003F000B6010E94F1D218164CF020E030E0A901BD
:10040000C501B4010E94EED087FF05C0A701960187
:10041000C501B40118C0F7FAF094F7F8F0941CC0C5
:10042000C701B6010E94EED087FD09C020E030E090
:10043000A901C501B4010E94F1D218164CF4A5011E
:100440009401C701B6010E9414D06B017C010EC05B
:10045000B7FAB094B7F8B094A7019601C501B401FA
:100460000E94F1D2181614F475016401A896AEAD7D
:10047000BFADA8978D909D90AD90BD90A896BFAF51
:10048000AEAFA897A5019401C701B6010E94F1D2B1
:10049000181694F4A7019601C501B4010E94F5D085
:1004A0009B01AC01C301B2010E942CD32B013C0182
:1004B000B1E02E96BFAF2E976296EEADFFAD62977C
:1004C000EA52FF4009F04ACF2E963FAD2E973323D4
:1004D00051F0A3019201B101812F902F0E942CD3E2
:1004E0001B01182F092F24EA30E74DE75FE3B10124
:1004F000812F902F0E942CD36B017C019B01AC01BA
:1005000060910D0F70910E0F80910F0F9091100F51
:100510000E94F1D218162CF5A70196016BA92C9612
:100520007FAD2C9724968FAD249728969FAD289762
:100530000E94F1D21816ACF4ABA5BCA58C918460D6
:100540008C9305C0EBA5FCA58081846080832BA8DB
:100550002C963FAC2C9724961FAD249728960FAD70
:100560002897C101A12FB02FEBA5FCA583A794A7C5
:10057000A5A7B6A76C966CAD7DAD8EAD9FAD6C9703
:1005800090589B01AC010E9415D0A2962CAD3DADB8
:100590004EAD5FADA2970E942CD39B01AC016BE0E6
:1005A00077ED83E29BE30E9414D00E9499D3F62E4C
:1005B000E72ED82EC92E262F372F482F592FB101BD
:1005C000812F902F0E94EED087FD03C02F2C3E2C50
:1005D0008601C101A12FB02FEBA5FCA587A390A791
:1005E000A1A7B2A7B0802F2D3E2D4D2D5C2D6FA55C
:1005F0007FA98BAD9FAD0E94EED0181614F083E05A
:1006000001C081E0B82AABA5BCA5BC9280E1FE0187
:100610003196AAE1BFE001900D928A95E1F78FA58E
:100620009FA9ABADBFAD8093160F9093170FA0930A
:10063000180FB093190F8BA92C969FAD2C97249669
:10064000AFAD24972896BFAD289780930D0F909358
:100650000E0FA0930F0FB093100F2FA53FA94BAD16
:100660005FADBC01CD010E94F5D069A37AA38BA335
:100670009CA32FA53FA94BAD5FADB101812F902F5A
:100680000E94F5D06DA37EA38FA398A7AE014F5D06
:100690005F4FBE016B5D7F4F8BA59CA50E94E473ED
:1006A00060960FAD60970093B80FAE962CAD3DAD40
:1006B0004EAD5FADAE9720932E0F30932F0F40932A
:1006C000300F5093310FE2968CAD9DADAEADBFAD06
:1006D000E2978093320F9093330FA093340FB0932F
:1006E000350FE6960CAD1DAD2EAD3FADE6970093F0
:1006F000360F1093370F2093380F3093390F6896C9
:100700002CAD3DAD4EAD5FAD689720933A0F309361
:100710003B0F40933C0F50933D0F0E94C4770AD289
:1007200009C03FAC2BA824960FAD249728961FAD87
:10073000289754C8CB58DF4F0FB6F894DEBF0FBED2
:10074000CDBFDF91CF911F910F91FF90EF90DF9080
:10075000CF90BF90AF909F908F907F906F905F9061
:100760004F903F902F900895CF92DF92EF92FF929B
:100770000F931F93CF93DF93CDB7DEB760970FB67C
:10078000F894DEBF0FBECDBF6B017A0189012091C5
:10079000970F3091980F4091990F50919A0FDC016B
:1007A0006D917D918D919C910E942CD30E94FCD2E1
:1007B00060932E0F70932F0F8093300F9093310F13
:1007C0006D877E878F87988B20919B0F30919C0F30
:1007D00040919D0F50919E0FF60160817181828141
:1007E00093810E942CD30E94FCD26093320F7093AD
:1007F000330F8093340F9093350F69877A878B87F7
:100800009C8720919F0F3091A00F4091A10F509194
:10081000A20FD7016D917D918D919C910E942CD357
:100820000E94FCD26093360F7093370F8093380F7D
:100830009093390F6D837E838F8398872091A30FC8
:100840003091A40F4091A50F5091A60FF80160813F
:100850007181828193810E942CD30E94FCD260938B
:100860003A0F70933B0F80933C0F90933D0F698339
:100870007A838B839C839E012F5F3F4FAE014B5F3A
:100880005F4FBE01675F7F4FCE010D960E94778C50
:100890001092160F1092170F1092180F1092190F36
:1008A00080E1EAE1FFE0DF011D928A95E9F76096B9
:1008B0000FB6F894DEBF0FBECDBFDF91CF911F9171
:1008C0000F91FF90EF90DF90CF9008959C01245FEF
:1008D0003F4FAC01485F5F4FBC016C5F7F4F44CF1F
:1008E000CF92DF92EF92FF920F931F93CF93DF93FC
:1008F00000D000D0CDB7DEB79E838D838C01FB0185
:10090000C080D180E280F380FC01FF27EE0FFF1F43
:10091000EE0FFF1FE956F04F208131814281538154
:10092000C701B6010E942CD30E94FCD2F801EE0F41
:10093000FF1FEE0FFF1FE25DF04F60837183828324
:100940009383C701B6010E945DD169837A838B834B
:100950009C83BE016F5F7F4FCE0105960E94C38CC2
:10096000ED81FE81EE0FFF1FEE0FFF1FE65EF04FE1
:10097000108211821282138226960FB6F894DEBF7F
:100980000FBECDBFDF91CF911F910F91FF90EF90E0
:10099000DF90CF9008958F929F92AF92BF92CF92A7
:1009A000DF92EF92FF920F931F93CF93DF9300D0CC
:1009B0001F92CDB7DEB767E6862E6FE0962E77E9F9
:1009C000A72E7FE0B72E07E71FE0C12CD12C7601C0
:1009D000C394F40161917191819191914F01F5015D
:1009E00021913191419151915F0129833A834B8348
:1009F0005C830E948ED129813A814B815C810E9467
:100A00002CD30E9462D1F8016193719381939193E9
:100A10008F01C616D706E806F90610F46B017C01B3
:100A2000F7E78F16FFE09F06A1F66FEF7FEFCB0190
:100A3000A70196010E942CD420932A0F30932B0FEC
:100A400040932C0F50932D0F0F900F900F900F90FD
:100A5000DF91CF911F910F91FF90EF90DF90CF909A
:100A6000BF90AF909F908F9008950F931F93CF9357
:100A7000DF93C7E9DFE007E81FE029913991499149
:100A8000599160E070E080E89FE30E94F5D0F801A2
:100A900061937193819391938F01FFE0C73ADF07D0
:100AA00061F78BEE97E012DFDF91CF911F910F91ED
:100AB00072CF86E40E948D1B80933E0F882351F0F5
:100AC0000E94831B60936A0270936B0280936C0296
:100AD00090936D0283E50E948D1B882351F00E9444
:100AE000821B60936E0270936F02809370029093EA
:100AF000710282E40E948D1B882351F00E94821BA8
:100B000060937202709373028093740290937502E3
:100B1000089589E494E10C94C9739091B80F809181
:100B2000B70F981731F08091B70F8F5F8F70809358
:100B3000B70F0895EFE6F0E080818260808308952A
:100B400080918C1480FF03C0899A8FEF02C089982E
:100B500081E08093770280918C1481FF03C08F988D
:100B60008FEF02C08F9A81E08093780280918C147D
:100B70009FB782FF0AC0F89480910B018D7F80930C
:100B80000B019FBF43988FEF09C0F89480910B0130
:100B9000826080930B019FBF439A81E0809379022A
:100BA00080918C1483FF03C016988FEF02C0169AB1
:100BB00081E080937A020895EF92FF920F931F9342
:100BC000CF93DF9380916E008B7F80936E00809136
:100BD0006F008D7F80936F00789480918A1490913C
:100BE0008B140097B9F0019790938B1480938A141B
:100BF00010928F1410928E1490DF80918A1490912D
:100C00008B14892B21F48AE590E10E94F91888EC75
:100C100090E08FC180918E1490918F14892B09F0F0
:100C20008DC19091B80F8091B70F981761F0E09146
:100C3000B70F29E4E29FF0011124E754F04F8081BF
:100C40008860808302C0E0E0F0E0F0938F14E093CE
:100C50008E14309709F46BC152A180918C1441819C
:100C600058130AC0242F30E080917602992787FD1F
:100C700090952817390729F050938C1440937602E9
:100C80005FDF10926C1410926D1410926E1410921B
:100C90006F14E0918E14F0918F1487A990AD813478
:100CA000ECE99E0728F48132FEE49F0748F002C079
:100CB00080E49CE9969587959695879524E007C0F2
:100CC000813127E2920730F09695879522E02093B4
:100CD000591408C021E0209359148032910510F472
:100CE00080E290E08C0100521109011588E018079C
:100CF000D0F0812F9927880F991F880F991F8A5943
:100D00009B4EFC01329645915491AA27059F900174
:100D1000049F210D3A1F06942A1F3A1F1124FC013B
:100D2000859194911DC0C801969587958C7F8A59AD
:100D30009F4EFC01459154910296FC01859194913E
:100D4000B80167707727869F9001879F300D969F27
:100D5000300D1124D3E036952795DA95E1F7CA01D5
:100D6000821B930B8436910578F4C9E4D4E0899111
:100D7000882319F00E94B311FACF6AE070E0C8012D
:100D80000E945E1284E690E090935714809356146C
:100D90008091591480935814E0918E14F0918F141F
:100DA00083AD94AD90935B1480935A148134ECE935
:100DB0009E0728F48132FEE49F0748F002C080E4D9
:100DC0009CE9969587959695879524E007C0813193
:100DD00027E2920730F09695879522E020935914E8
:100DE00008C021E0209359148032910510F480E26C
:100DF00090E08C0100521109011588E01807E0F01D
:100E0000812F9927880F991F880F991F8A599B4E08
:100E1000FC01329625913491AA27039FA001029FDD
:100E2000410D5A1F06944A1F5A1F1124FC01259197
:100E30003491241B350B1EC0C801969587958C7F75
:100E40008A599F4EFC01259134910296FC014591EF
:100E50005491B80167707727469FC001479F900D56
:100E6000569F900D112473E0969587957A95E1F73A
:100E7000281B390B2436310578F4C9E4D4E0899174
:100E8000882319F00E94B311FACF6AE070E0C8011C
:100E90000E945E1224E630E0C901A0E0B0E0809339
:100EA000701490937114A0937214B09373143093D0
:100EB000890020938800E0918E14F0918F1482892C
:100EC0009389A489B589B695A79597958795B09587
:100ED000A095909581959F4FAF4FBF4F8093781409
:100EE00090937914A0937A14B0937B1480937C141C
:100EF00090937D14A0937E14B0937F1480938014FC
:100F000090938114A0938214B093831480938414DB
:100F100090938514A0938614B09387141092741440
:100F200010927514109276141092771407C080ED09
:100F300097E0909389008093880008C480913902DB
:100F400081110E94937220E08091591490E0422F09
:100F5000552747FD5095481759070CF0EBC1E09114
:100F60008E14F0918F148091841490918514A09127
:100F70008614B09187144281538164817581840FF6
:100F8000951FA61FB71F8093841490938514A09378
:100F90008614B0938714181619061A061B060CF44B
:100FA000889AE0918E14F0918F1480918014909122
:100FB0008114A0918214B091831446815781608579
:100FC0007185840F951FA61FB71F8093801490937F
:100FD0008114A0938214B0938314181619061A066C
:100FE0001B060CF48E9AE0918E14F0918F14809170
:100FF0007C1490917D14A0917E14B0917F14428551
:10100000538564857585840F951FA61FB71F809330
:101010007C1490937D14A0937E14B0937F141816C3
:1010200019061A061B063CF580918D148823D1F011
:101030008091060F82FF04C08091790287FD05C070
:1010400080918914882309F492C38091060F87FF49
:1010500004C08091790287FD0EC0809188148111AF
:101060000AC008C09FB7F89480910B0188608093F4
:101070000B019FBF419AE0918E14F0918F148091E3
:10108000781490917914A0917A14B0917B144685CC
:10109000578560897189840F951FA61FB71F80939C
:1010A000781490937914A0937A14B0937B14181643
:1010B00019061A061B060CF4149A80918414909158
:1010C0008514A0918614B0918714181619061A0673
:1010D0001B0684F5E0918E14F0918F144289538998
:1010E00064897589841B950BA60BB70B80938414B8
:1010F00090938514A0938614B0938714409177023F
:1011000080915C1490915D14A0915E14B0915F1475
:10111000552747FD5095652F752F840F951FA61FE6
:10112000B71F80935C1490935D14A0935E14B093EA
:101130005F1488988091801490918114A0918214FA
:10114000B0918314181619061A061B0684F5E0914F
:101150008E14F0918F144289538964897589841B98
:10116000950BA60BB70B8093801490938114A093DA
:101170008214B0938314409178028091601490910E
:101180006114A0916214B0916314552747FD5095E6
:10119000652F752F840F951FA61FB71F80936014AE
:1011A00090936114A0936214B09363148E9880910D
:1011B0007C1490917D14A0917E14B0917F14181628
:1011C00019061A061B060CF056C0E0918E14F09119
:1011D0008F144289538964897589841B950BA60BEA
:1011E000B70B80937C1490937D14A0937E14B093DE
:1011F0007F14409179028091641490916514A091BC
:101200006614B0916714552747FD5095652F752FCB
:10121000840F951FA61FB71F8093641490936514C5
:10122000A0936614B093671480918D148823D1F035
:101230008091060F82FF04C08091790287FD05C06E
:1012400080918914882309F49BC28091060F87FF3F
:1012500004C08091790287FD0EC0809188148111AD
:101260000AC008C09FB7F89480910B01877F8093D4
:101270000B019FBF41988091781490917914A091AF
:101280007A14B0917B14181619061A061B0684F5F9
:10129000E0918E14F0918F14428953896489758985
:1012A000841B950BA60BB70B80937814909379143D
:1012B000A0937A14B0937B1440917A0280916814C1
:1012C00090916914A0916A14B0916B14552747FD51
:1012D0005095652F752F840F951FA61FB71F8093FC
:1012E000681490936914A0936A14B0936B141498C3
:1012F0008091741490917514A0917614B091771424
:101300000196A11DB11D8093741490937514A09340
:101310007614B0937714E0918E14F0918F14428973
:1013200053896489758984179507A607B70720F440
:101330002F5F0ACEC0E001C0C1E04091741450910B
:1013400075146091761470917714E0918E14F09179
:101350008F1486899789A08DB18D84179507A6076C
:10136000B70708F4DDC0409170145091711460917A
:10137000721470917314068D178D20A131A1AA27C4
:10138000419FB12D529FC001629F900D619F800DC2
:10139000911D429FB00D811D9A1F519FB00D811D5F
:1013A0009A1F609FB00D811D9A1F509FB10D8A1F1B
:1013B0009A1FB6958A1F9A1F349F800D911D359FE5
:1013C000900D112443AD54AD480F591F50935B1439
:1013D00040935A1487A990ADA1ADB2AD60E070E022
:1013E00084179507A607B70720F490935B148093A2
:1013F0005A1480915A1490915B148134ECE99E0741
:1014000028F48132FEE49F0748F002C080E49CE9A2
:10141000969587959695879524E007C0813127E2B8
:10142000920730F09695879522E02093591408C0D2
:1014300021E0209359148032910510F480E290E06D
:101440008C0100521109011588E01807E0F0812F86
:101450009927880F991F880F991F8A599B4EFC0165
:10146000329625913491AA27039FA001029F410D36
:101470005A1F06944A1F5A1F1124FC0125913491CA
:10148000241B350B1EC0C801969587958C7F8A5901
:101490009F4EFC01259134910296FC014591549197
:1014A000B80167707727469FC001479F900D569FF0
:1014B000900D1124B3E096958795BA95E1F7281B16
:1014C000390B2436310598F4F9E4EF2EF4E0FF2EC1
:1014D000F70181917F01882319F00E94B311F8CFA1
:1014E0006AE070E0C8010E945E1224E630E03093AA
:1014F0008900209388008091701490917114A091BC
:101500007214B0917314820F931FA11DB11D8093AB
:10151000701490937114A0937214B0937314FAC062
:1015200040917414509175146091761470917714F1
:10153000828D938DA48DB58D84179507A607B70767
:1015400008F0DCC040916C1450916D1460916E14E1
:1015500070916F14068D178D20A131A1AA27419F8C
:10156000B12D529F7001629FF00C619FE00CF11C45
:10157000429FB00DE11CFA1E519FB00DE11CFA1EF6
:10158000609FB00DE11CFA1E509FB10DEA1EFA1EBD
:10159000B695EA1EFA1E349FE00CF11C359FF00C44
:1015A000112480915A1490915B14FF96E816F90665
:1015B00080F48E199F0940815181628173818C0171
:1015C00020E030E0041715072607370720F4CA018A
:1015D00002C0808191818134FCE99F0728F4813227
:1015E0002EE4920748F002C080E49CE99695879526
:1015F0009695879524E007C08131E7E29E0730F099
:101600009695879522E02093591408C021E02093F5
:1016100059148032910510F480E290E08C01005260
:1016200011090115F8E01F07E0F0812F9927880FB5
:10163000991F880F991F8A599B4EFC01329625915C
:101640003491AA27039FA001029F410D5A1F0694BF
:101650004A1F5A1F1124FC0125913491241B350B7C
:101660001EC0C801969587958C7F8A599F4EFC01B4
:10167000259134910296FC0145915491B80167700F
:101680007727469FC001479F900D569F900D1124CC
:1016900043E0969587954A95E1F7281B390B243648
:1016A000310598F489E4E82E84E0F82EF701819161
:1016B0007F01882319F00E94B311F8CF6AE070E02F
:1016C000C8010E945E1224E630E030938900209326
:1016D000880080916C1490916D14A0916E14B0915B
:1016E0006F14820F931FA11DB11D80936C149093F2
:1016F0006D14A0936E14B0936F140CC080915614A7
:101700009091571490938900809388008091581489
:101710008093591420918800309189008091840031
:101720009091850040962817390748F480918400ED
:101730009091850040969093890080938800CC23F7
:1017400029F010928F1410928E14E7D980916E00B8
:10175000846080936E0080916F00826080936F0040
:10176000DF91CF911F910F91FF90EF9008959FB758
:10177000F89480910B01886080930B019FBF65CC2A
:101780009FB7F89480910B01877F80930B019FBFD7
:101790005CCD1F920F920FB60F9211240BB60F92D1
:1017A0002F933F934F935F936F937F938F939F9369
:1017B000AF93BF93EF93FF93FFD9FF91EF91BF9149
:1017C000AF919F918F917F916F915F914F913F91D9
:1017D0002F910F900BBE0F900FBE0F901F9018957A
:1017E000819A879AEAE0F1E08081826080833B9A67
:1017F0000E9A3B9A579A5F9A829A8A9AE7E0F1E0AA
:101800008081816080839FB7F894E8E0F1E0808177
:10181000816080839FBF3F9A479A0A9A129A3F9AA3
:10182000479A8CE09FE00E94A971809A88985F9AFD
:101830001092D507869A8E988A9A479A1092D60760
:10184000399A4198EAE0F1E08081886080839FB70F
:10185000F894EBE0F1E08081877F80839FBF9FB7A2
:10186000F894E8E0F1E08081816080839FBF479A2F
:101870001092D7070C9A1498129A399A4198A1E8B5
:10188000B0E08C918F7E8C938C9188608C93E0E893
:10189000F0E080818D7F808380818E7F8083808156
:1018A0008F73808380818F7C80838C91887F82601E
:1018B0008C9380E090E4909389008093880010924C
:1018C000850010928400EFE6F0E0808182608083E2
:1018D00081E080933902789433C99091B80F809158
:1018E000B70F981719F00E94E239F7CF0895CF92F9
:1018F000DF92EF92FF920F931F93CF93DF936C01D0
:101900007B018A01E901E9DF2FB7F894F6018081B4
:101910009181A281B38180935C1490935D14A09314
:101920005E14B0935F14F70180819181A281B3812D
:101930008093601490936114A0936214B093631425
:10194000F80180819181A281B38180936414909386
:101950006514A0936614B093671488819981AA8155
:10196000BB818093681490936914A0936A14B09318
:101970006B142FBFDF91CF911F910F91FF90EF90CC
:10198000DF90CF900895CF93DF932FB7F894DC01C9
:10199000ED91FC91EB0188819981AA81BB81EE0FC9
:1019A000FF1FEE0FFF1FE45AFB4E80839183A2833B
:1019B000B3832FBFDF91CF9108952FB7F894880F8D
:1019C000991F880F991F845A9B4EFC016081718179
:1019D000828193812FBF0895CF93DF93EC01EDDFD8
:1019E0000E9490D1FE01EE0FFF1FEE0FFF1FE9577F
:1019F000F04F20813181428153810E942CD3DF91AD
:101A0000CF9108956ADF0C947E2C88E893E190933F
:101A10008B1480938A1480916F008D7F80936F0068
:101A20009091B80F8091B70F981711F076D8F8CF32
:101A300010928F1410928E1480916F0082608093A8
:101A40006F000895880F991F880F991FFC01E45AB1
:101A5000FB4E4081518162817381FC01E65BFB4E4C
:101A60004083518362837383E0918E14F0918F14CD
:101A700082899389A489B58980937414909375148D
:101A8000A0937614B093771408954F925F926F925B
:101A90007F928F929F92AF92BF92CF92DF92EF92FE
:101AA000FF92CF93DF938FB7F89440905C145090DF
:101AB0005D1460905E1470905F148090601490903C
:101AC0006114A0906214B0906314C0906414D0901C
:101AD0006514E0906614F09067148FBFEFE4F0E1B6
:101AE0008491EF012196882321F00E94B311FE0119
:101AF000F7CF4AE050E0C301B2010E944912EBE483
:101B0000F0E184913F019FEF691A790A882321F05F
:101B10000E94B311F301F5CF4AE050E0C501B401D2
:101B20000E944912E7E4F0E184915F019FEFA91A56
:101B3000B90A882321F00E94B311F501F5CF4AE0DC
:101B400050E0C701B6010E9449128AE0DF91CF91AF
:101B5000FF90EF90DF90CF90BF90AF909F908F90CD
:101B60007F906F905F904F900C94B311FC011182A5
:101B700010821682178210861186128613861486AA
:101B8000158612821382148215820895CF93DF93F3
:101B9000EC01888199810197029710F080E009C0DB
:101BA000198218820E9424C86A877B878C879D8748
:101BB00081E0DF91CF910895CF93DF93EC0188818D
:101BC0009981019761F482E090E0998388830E9473
:101BD00024C86A877B878C879D8781E001C080E06D
:101BE000DF91CF9108950F931F93CF93DF93EC0173
:101BF00088819981019719F40E9424C804C06A85DC
:101C00007B858C859D850E811F8128853985601B8C
